:020000040800F2
:1000000000040020E1010008090E00080D0E0008A0
:10001000610E00080D0E0008350E0008E30100080F
:10002000E3010008E3010008E3010008392F00089C
:10003000E3010008E3010008E3010008E301000810
:10004000E3010008E3010008E3010008E301000800
:10005000E3010008E301000899310008C5310008F8
:10006000F13100081D32000849320008E3010008A0
:10007000E3010008E3010008E3010008E3010008D0
:10008000E3010008E3010008E3010008E3010008C0
:10009000E3010008E3010008E301000875320008ED
:1000A000E3010008E3010008E3010008E3010008A0
:1000B000B52F0008E3010008E3010008E301000890
:1000C000E3010008E3010008E3010008E301000880
:1000D000E3010008E3010008E3010008E301000870
:1000E000DD320008E3010008E3010008E301000835
:1000F000E3010008E3010008E3010008E301000850
:10010000E3010008E3010008E3010008E30100083F
:10011000E3010008E3010008E3010008E30100082F
:10012000E3010008E3010008E3010008E30100081F
:10013000E3010008E3010008E3010008E30100080F
:10014000E3010008E3010008E30100088D26000830
:10015000E3010008E3010008E3010008E3010008EF
:10016000E3010008E3010008E3010008E3010008DF
:10017000E3010008E3010008E3010008E3010008CF
:10018000E3010008E3010008E3010008E3010008BF
:10019000E3010008E3010008E3010008E3010008AF
:1001A000E3010008E3010008E3010008E30100089F
:1001B000E3010008E3010008E3010008E30100088F
:1001C000E3010008E3010008E3010008E30100087F
:1001D000E3010008E3010008E3010008E30100086F
:1001E00002E000F000F8FEE772B6394880F30888B4
:1001F000384880F3098838484EF60851CEF200019D
:10020000086040F20000CCF200004EF63471CEF2ED
:1002100000010860BFF34F8FBFF36F8F40F2000003
:10022000C0F2F0004EF68851CEF200010860BFF334
:100230004F8FBFF36F8F4FF00000E1EE100A4EF6C4
:100240003C71CEF200010860062080F31488BFF3F1
:100250006F8F01F0E3FE02F005FE4FF055301F49AD
:100260001B4A91423CBF41F8040BFAE71C49194A6A
:1002700091423CBF41F8040BFAE71A491A4A1B4B5A
:100280009A423EBF51F8040B42F8040BF8E70020F5
:100290001749184A91423CBF41F8040BFAE701F0B4
:1002A000C1FE02F03BFE144C144DAC4203DA54F88C
:1002B000041B8847F9E700F03FF8114C114DAC42A0
:1002C00003DA54F8041B8847F9E701F0A9BE0000DF
:1002D000000400200024002000000008000000208E
:1002E00000040020F036000800240020282400200C
:1002F0002824002018300020E0010008E001000858
:10030000E0010008E00100082DE9F04F2DED108A12
:10031000C1F80CD0C3689D46BDEC108ABDE8F08FD3
:10032000002383F311882846A047002001F0FAFA41
:1003300001F0AAFA00DFFEE71A4B6FF0790270B500
:1003400000241A700F225C709C70DC701C715C7150
:100350009C71DC711C725C729A72DC7201F030FE6E
:10036000064601F055FE054650B90F4B9E4217D088
:1003700001339E4241F2883412BF05460024012514
:10038000002001F027FE0DB100F0B4F800F010FDE0
:1003900000F0F4FB204600F00BF900F0ABF8F9E7B1
:1003A0000446EDE728240020010007B008B500F05E
:1003B00087FBA0F120035842584108BD07B5054B03
:1003C00002211B88ADF8043001A800F0C7FB03B080
:1003D0005DF804FBC0330008064991F8243033B1BE
:1003E00000230822086A81F8243000F0E9BB0120CC
:1003F000704700BF482400202DE9F84F234C94F8A3
:1004000024300546884617468BBB2E46DFF87C9085
:10041000002F38D094F824A0BAF1000F05D1202283
:10042000FF214846266200F0B1FCCAF10805BD4232
:1004300028BF3D465FFA85FBAD0041462A4604EBE6
:100440008A0000F079FC94F82430A7EB0B079B445A
:100450005FFA8BFBBBF1080F2E44A844FFB284F86F
:1004600024B0D5D1FFF7B8FF0028D1D108E0266A23
:1004700006EB8306B042C9D0FFF7AEFF0028C4D117
:100480000020BDE8F88F0120BDE8F88F4824002047
:1004900010B5202383F311881248C3680BB101F013
:1004A000C7FA0023104A0F484FF47A7101F084FA1A
:1004B000002383F311880D4C236813B12368013B9B
:1004C0002360636813B16368013B6360084B1B786A
:1004D00033B9636823B9022000F024FC322363603F
:1004E00010BD00BF342400209104000878250020AE
:1004F0007024002010B5254B254953F8042F0132F4
:1005000000D110BD8B42F8D1224C234B22689A4275
:100510003AD9224B9B6803F1006303F580339A427A
:1005200032D2002000F044FB1D4B0220187000F076
:10053000F1FB1C4B1A6C00221A64196E1A66196EB4
:10054000596C5A64596E5A665A6E5A6942F0800262
:100550005A615A6922F080025A615A691A6942F056
:1005600000521A611A6922F000521A611B6972B6B0
:100570000D4A0E4B13601B682268202181F31188FD
:100580009D4683F30888104710BD00BFFCFF00089C
:100590001C00010804000108FFFF000828240020B7
:1005A000702400200038024008ED00E0000001083F
:1005B0002DE9F04F99B0B34C01902022FF2110A8F3
:1005C000A66800F0E3FBB04A1378A346A3B9AF488E
:1005D0000121C3601170202383F31188C3680BB11C
:1005E00001F026FA0023AA4AA8484FF47A7101F0D4
:1005F000E3F9002383F31188019B13B1A54B019A02
:100600001A60A54AA349019F0292002313704B6010
:1006100099461C461D469846012000F07BFB002FA2
:1006200000F012829B4B1B68002B40F00D8219B02A
:10063000BDE8F08F0220FFF7B9FE002840F0FB81F3
:10064000019BB9F1000F08BF1F46944B1B88ADF802
:100650002C3002210BA800F081FADDE74FF47A700C
:1006600000F02EFA031E0393EADB0220FFF79EFE42
:1006700082460028E4D0039B581E042800F2DD8146
:10068000DFE800F0030E1114170018A8052340F846
:10069000343D042100F062FA54464FF0000856E061
:1006A00004217848F6E704217D48F3E704217D48DA
:1006B000F0E71C24204600F07DFA04340B9004215E
:1006C0000BA800F04BFA2C2CF4D1E5E7002DB7D0A5
:1006D000002CB5D00220FFF769FE0546002800F087
:1006E000AF8101206C4C00F063FA0220207000F012
:1006F00011FB4FF000095FFA89FA504600F068FAE2
:10070000074658B1504600F073FA09F10109002874
:10071000F1D12C46A9460027634B97E7012302201D
:10072000237000F0EDFA3E46DBF808309E4206D218
:10073000304600F03FFA0130EBD10436F4E7029B7B
:1007400000261E70534BA9465E602C46374600F0CB
:1007500025FB15B1002C18BF0027FFF72FFE5BE724
:10076000002D3FF46DAF002C3FF46AAF029B0220D6
:10077000187000F0CFFA322000F0A2F9B0F1000AB0
:10078000C0F25E811AF0030540F05A81DBF80820C0
:1007900006EB0A03934200F25381BAF5807F00F220
:1007A0004F8155450DDA4FF47A7000F089F90490C5
:1007B000049B002BC0F244813C4A049BAB5401359E
:1007C000EFE7C820FFF7F2FD0546002800F038816A
:1007D0001F2E11D8C6F12004544528BF544610AB33
:1007E00026F0030022463149184400F0A5FA2246BB
:1007F000FF212E4800F0CAFA4FEAAA0A5FFA8AF2ED
:100800002A493046FFF7F8FD0446002800F01A8117
:1008100006EB8A0605469AE70220FFF7C7FD002887
:100820003FF40EAFFFF7D8FD00283FF409AF4FF0BB
:10083000000A5346DBF8082092451CD2BAF11F0F7C
:1008400012D8109A01320FD02AF0030218A90A44D4
:1008500052F8202C0B92184604220BA900F014FB2E
:100860000AF1040A0346E5E75046039300F0A2F9B3
:10087000039B0B90EFE718A8042140F84C3D00F0D3
:100880006DF964E72824002074250020342400201A
:10089000910400087825002070240020C23300084D
:1008A0002C24002030240020C433000874240020AD
:1008B00018A8002340F8343D642100F02BF90028EB
:1008C0007FF4BEAE0220FFF771FD00283FF4B8AE02
:1008D0000B9800F09FF918AB43F8480D0421184617
:1008E000CDE718A8002340F8343D642100F012F948
:1008F00000287FF4A5AE0220FFF758FD00283FF442
:100900009FAE0B9800F094F918AB43F8440DE5E75F
:100910000220FFF74BFD00283FF492AE00F08EF965
:1009200018AB43F8400DD9E70220FFF73FFD002840
:100930003FF486AE0BA9142000F086F9824618A871
:10094000042140F83CAD00F009F951460BA896E7A8
:10095000322000F0B5F8B0F1000AFFF671AE1AF0DF
:10096000030F7FF46DAEDBF808200AEB0803934217
:100970003FF666AE0220FFF719FD00283FF460AE97
:100980002AF0030AC244D0453FF4E1AE404600F0ED
:1009900011F904210A900AA800F0E0F808F104080F
:1009A000F1E74FF47A70FFF701FD00283FF448AEFD
:1009B000FFF712FD00283FF4AFAE109B01330CD0BF
:1009C000082210A90020FFF717FD00283FF4A4AE6D
:1009D0002022FF2110A800F0D9F9FFF7EFFC3748DB
:1009E00000F0A6FF23E6002D3FF42AAE002C3FF4D2
:1009F00027AE18A8002340F8343D642100F08AF89F
:100A0000824600287FF41CAE0220FFF7CFFC0028AE
:100A10003FF416AE0390FFF7D1FC41F2883000F0AE
:100A200087FF0B9800F0EEF900F0B8F9039B5746EA
:100A30001C461D46F0E5054689E64FF00008FFE537
:100A40002546FDE52C4667E6002000F039F80490C5
:100A5000049B002BFFF6E3AD012000F051F9049B4D
:100A6000213B122B3FF6D8AD01A252F823F000BF74
:100A7000350600085D060008CD06000819060008C6
:100A80001906000819060008610700085109000846
:100A900019080008B1080008E30800081109000857
:100AA000190600082909000819060008A30900080A
:100AB0004F07000819060008E7090008A086010092
:100AC00037B5114B1A780132D2B20024012A0146FF
:100AD0008DF8074011D80D4803681D6A4FF47A73EA
:100AE0004B4301220DF10701A847012805D1084B0E
:100AF0009DF807001C7003B030BD4FF4FA7000F091
:100B000017FF4FF0FF30F6E70024002048260020B2
:100B10008425002038B50E4B1A780132D2B2012A52
:100B200005460ED80B4803681C6A4FF47A734B4392
:100B300004222946A047042803D1074B002018703F
:100B400038BD4FF4FA7000F0F3FE4FF0FF3038BDBF
:100B500000240020482600208425002030B4054CC5
:100B60002368DD69044B0A46AC460146204630BC8A
:100B7000604700BF48260020A086010070B501F044
:100B800023F9094C094E20700025306823788342F0
:100B900008D901F013F9336805440133B5F5803FF6
:100BA0003360F2D370BD00BF852500208025002072
:100BB00001F0B8B900F1006000F5803000687047BE
:100BC00000F10060920000F5803001F043B90000B0
:100BD000054B1A68054B1B789B1A834202D91044B7
:100BE00001F0ECB80020704780250020852500200A
:100BF00038B5074D04462868204401F0E7F828B9C5
:100C000028682044BDE8384001F0F8B838BD00BF7E
:100C10008025002010F0030308D1B0F5007F05D82F
:100C200000F10050A0F508400068704700207047B0
:100C3000014BC058704700BF107AFF1F014B186866
:100C4000704700BF002004E070B52A4B1C68C4F355
:100C50000B03240C63B140F21342934231D040F2B3
:100C6000194293422FD040F2214293422DD10323C7
:100C7000214A0C2505FB03235D6893F9082042F205
:100C800001039C4224D0B4F5805F23D041F20103DC
:100C90009C4221D041F203039C421FD041F2070342
:100CA0009C4208BF3122441E0C44013D0B46A34226
:100CB0001ED215F9016F581C96B1034600F8016C5D
:100CC000F5E70123D4E70223D2E73F220B4DD6E715
:100CD0003322E3E74122E1E75A22E4E75922E2E73F
:100CE0002C2584421D7001D9981C5A70401A70BD81
:100CF0001846FBE7002004E0D4330008C83300089E
:100D0000022802BF024B4FF400129A61704700BFE5
:100D100000040240022802BF014B20229A61704762
:100D200000040240022801BF024A536983F02003F5
:100D3000536170470004024010B50023934203D072
:100D4000CC5CC4540133F9E710BD000030B5441E3B
:100D500014F9010F0B4660B193F90050854201F17F
:100D6000010106D11AB993F90020801A30BD013A69
:100D7000EEE7002AF7D1104630BD000002460346D8
:100D8000981A13F9011B0029FAD17047024403464F
:100D9000934202D003F8011BFAE77047024B1A781E
:100DA000024B1A70704700BF8425002000240020E9
:100DB00038B5104D104C284600F002F9214628465F
:100DC00000F02AF924680D48626DD2F8043843F027
:100DD0000203C2F8043800F0ABFD0949204600F0D8
:100DE00027FA626DD2F8043823F00203C2F80438FF
:100DF00038BD00BF48260020A034000840420F0044
:100E0000C834000870470000FEE7000000B59BB042
:100E1000EFF3098168226846FFF78EFFEFF3058341
:100E2000034B9A6B9A6A9A6A9A6A9A6A9B6AFEE775
:100E300000ED00E000B59BB0EFF309816822684641
:100E4000FFF77AFFEFF30583044B9A6B9A6A9A6A6D
:100E50009A6A9A6A9A6A9B6AFEE700BF00ED00E010
:100E600000B59BB0EFF3098168226846FFF764FF85
:100E7000EFF30583034B5A6B9A6A9A6A9A6A9A6AE5
:100E80009B6AFEE700ED00E030B5084D0A44914250
:100E90000BD011F8013B09245840013CF7D040F336
:100EA00000032B4083EA5000F7E730BD2083B8ED04
:100EB000002304491A465A50C8180833802B426050
:100EC000F9D170478825002002684368114301600A
:100ED00003B118477047000013B5446BD4F894343D
:100EE0001A681178042915D1217C022912D11979A7
:100EF000128901238B4013420CD101A904F14C004B
:100F000001F02AFED4F89444019B2179024620681E
:100F100000F0DAF902B010BD143001F0ADBD0000F0
:100F20004FF0FF33143001F0A7BD00004C3001F04A
:100F30007FBE00004FF0FF334C3001F079BE00005F
:100F4000143001F07BBD00004FF0FF31143001F090
:100F500075BD00004C3001F04BBE00004FF0FF3279
:100F60004C3001F045BE0000D0F8942438B5136829
:100F700019780429054601D0012038BD017C0229D9
:100F8000FAD112795C89012090400440F4D105F136
:100F9000140001F00DFD02460028EDD0D5F8945460
:100FA0004FF480732868697900F07CF9204638BDD9
:100FB000406BFFF7D9BF000000207047704700006A
:100FC0007FB5124B0360002343608360C36001253B
:100FD00002260F4B057404460290019300F184022F
:100FE000294600964FF48073143001F0BDFC094B84
:100FF0000193029400964FF4807304F523722946FE
:1010000004F14C0001F084FD04B070BD24340008EC
:10101000B10F0008D90E00080B68202282F3118856
:101020000A7903EB820290614A79093243F822007F
:101030008A7912B103EB8203986102230374C0F82A
:101040009414002383F311887047000038B5037FA0
:10105000044613B190F85430ABB9201D012502218C
:10106000FFF732FF04F1140025776FF0010100F063
:1010700087FC84F8545004F14C006FF00101BDE886
:10108000384000F07DBC38BD10B501210446043065
:10109000FFF71AFF0023237784F8543010BD0000B7
:1010A00038B504460025143001F076FC04F14C00FC
:1010B000257701F045FD201D84F854500121FFF7EC
:1010C00003FF2046BDE83840FFF74EBF90F844309C
:1010D00003F06003202B19D190F84520212A0AD073
:1010E000222A4FF000030ED0202A0FD1084A826333
:1010F0000722C26304E0064B83630723C363002314
:101100000364012070478363C363F9E700207047DD
:1011100001240020D0F8943437B51A6811780429D6
:1011200004461AD1017C022917D1197912890123A9
:101130008B40134211D100F14C05284601F0C0FD4F
:1011400058B101A9284601F007FDD4F89444019B49
:1011500021790246206800F0B7F803B030BD0000E6
:1011600000EB8103F7B59C6905460E46F4B12023D8
:1011700083F3118805EB8607201D0821FFF7A4FEE5
:10118000FB685B691B684C3413B1204601F0F2FC2C
:1011900001A9204601F0E0FC024648B1019B31461E
:1011A000284600F091F8002383F3118803B0F0BDC6
:1011B000FB685A691268002AF5D01B8A013B13406C
:1011C000F1D105F14402EAE7093138B550F8214080
:1011D000DCB1202383F31188D4F894241368527966
:1011E00003EB8203DB689B695D6845B104216018ED
:1011F000FFF76AFE294604F1140001F0E3FB2046E4
:10120000FFF7B2FE002383F3118838BD704700005A
:1012100000F08EBF0123037000234360C36183622B
:101220000362C3624362036303814381704700002A
:1012300038B50446202383F3118800254160C5603A
:1012400005614561856100F083FF0223237085F30A
:10125000118838BD70B500EB810305465069DA602E
:101260000E46144618B110220021FFF78FFDA06929
:1012700018B110220021FFF789FD31462846BDE84C
:10128000704001F02FB80000028902F001020281D3
:10129000428902F0010242810022026142618261C0
:1012A00001F0B4B8F0B400EB81044789E46801258B
:1012B000A4698D403D43458123600023A2606360A3
:1012C000F0BC01F0CFB80000F0B400EB8104078956
:1012D000E468012564698D403D4305812360002356
:1012E000A2606360F0BC01F049B9000070B5022350
:1012F000002504460370A0F84C5080F84E5080F84A
:101300004F5005814581C56005614561856180F863
:10131000345000F083FF63681B6823B129462046E0
:10132000BDE87040184770BD436802781B6880F8BC
:101330005020052202700BB10421184770470000AD
:10134000436890F850201B6802700BB105211847C4
:101350007047000090F8343070B5044613B1002394
:1013600080F8343004F14402204601F071F86368DB
:101370009B6863BB94F8445015F0600615D194F84F
:10138000453005F07F0545EA032540F202339D42D2
:1013900000F00E815BD8022D00F0DC803FD8002DDC
:1013A00000F08780012D00F0CF800021204601F061
:1013B000A7FA0021204601F099FA63681B6813B16F
:1013C000062120469847062384F8343070BD204615
:1013D00098470028CED094F84B2094F84A3043EA3E
:1013E0000223E26B934238BFE36394F94430E56B28
:1013F000002B4FF0200380F2FD80002D00F0EC80E8
:10140000092284F8342083F311880021E36BA26B56
:101410002046FFF759FF002383F3118870BDB5F50F
:10142000817F00F0B180B5F5407F49D0B5F5807F70
:10143000BBD194F84630012BB7D1B4F84C3023F02F
:101440000203A4F84C30A663E6632664C3E740F2C7
:1014500001639D421ED8B5F5C06F3BD2B5F5A06FB4
:10146000A3D1B4F84430B3F5A06F0ED194F8463050
:1014700084F84E30204600F029FF63681B6813B1E2
:10148000012120469847032323700023A363E363CD
:101490002364A0E7B5F5106F32D040F602439D42B9
:1014A00052D0B5F5006F80D104F14F03A36301233F
:1014B00024E004F14C03A3630223E36325648AE779
:1014C00094F84630012B7FF470AFB4F84C3043F001
:1014D0000203B6E794F84920616894F848304D68F3
:1014E00094F8471043EA0223204694F84620A84780
:1014F00000283FF45AAF4368A3630368E363A4E79B
:101500002378042B10D1202383F311882046FFF782
:10151000BBFE86F31188636884F84F601B68032163
:1015200021700BB12046984794F84630002BACD080
:1015300084F84F300423237063681B68002BA4D009
:10154000022120469847A0E7374BA3630223E363B9
:1015500000239DE794F8481011F0800F204601F019
:101560000F010ED000F066FF012806D002287FF49C
:101570001CAF2E4BA363E06367E72D4BA363E563CA
:1015800063E700F049FFEFE794F84630002B7FF463
:101590000CAF94F8483013F00F013FF476AF1A0601
:1015A000204602D501F0C0F96FE701F0B3F96CE70E
:1015B00094F84630002B7FF4F8AE94F8483013F0DE
:1015C0000F013FF462AF1B06204602D501F098F9E7
:1015D0005BE701F08BF958E7142284F8342083F399
:1015E00011882B462A4629462046FFF75BFE85F3E5
:1015F000118870BD5DB1152284F8342083F3118801
:101600000021E36BA26B2046FFF74CFE03E70B22A1
:1016100084F8342083F311882B462A462946204635
:10162000FFF752FEE3E700BF543400084C340008D3
:101630005034000838B590F834300446152B29D8BA
:10164000DFE803F03E28282828283E28280B2939DF
:1016500028282828282828283E3E90F84B1090F863
:101660004A20C36B42EA01229A4214D9C268128A04
:10167000B3FBF2F502FB15356DB9202383F3118816
:101680002B462A462946FFF71FFE85F311880A23B9
:1016900084F8343038BD142384F83430202383F3A5
:1016A000118800231A4619462046FFF7FBFD002348
:1016B00083F3118838BD036C03B198470023E7E733
:1016C000002101F01DF90021204601F00FF96368A7
:1016D0001B6813B10621204698470623D8E700006F
:1016E00090F83420152A38B5044622D801239340B7
:1016F00040F6416213421DD113F480150FD19B02B5
:1017000017D50B2380F83430202383F311882B4620
:101710002A462946FFF7D8FD85F3118838BDC368EE
:101720009B695B682BB9036C03B19847002384F86D
:10173000343038BD002101F0E3F80021204601F0EB
:10174000D5F863681B6813B1062120469847062325
:10175000EDE70000024B00221B605B609A6070475F
:1017600008260020002303748268054B1B689968D3
:101770009142FBD25A680360426010605860704723
:101780000826002008B5202383F31188037C032B4F
:1017900005D0042B0DD02BB983F3118808BD436904
:1017A00000221A604FF0FF334361FFF7DBFF002395
:1017B000F2E790E80C001A6002685360F2E700005C
:1017C000002303748268054B1B6899689142FBD81B
:1017D0005A68036042601060586070470826002015
:1017E000054B19690874186802681A60536018611B
:1017F00001230374FEF788BD0826002030B54B1C7A
:1018000087B005460A4C10D023690A4A01A800F0A7
:10181000D3F82846FFF7E4FF049B13B101A800F0BA
:1018200007F92369586907B030BDFFF7D9FFF8E71A
:10183000082600208517000838B50C4D41612B693A
:1018400081689A689142044603D8BDE83840FFF7A2
:1018500089BF1846FFF786FF01232C6101462374D8
:101860002046BDE83840FEF74FBD00BF08260020E7
:10187000044B1A681B6990689B68984294BF0020CB
:10188000012070470826002010B5084C2368206905
:101890001A6822605460012223611A74FFF790FFD6
:1018A00001462069BDE81040FEF72EBD0826002045
:1018B0008260022202740022427470478368A3F19E
:1018C0007C0243F80C2C026943F83C2C426943F833
:1018D000382C074A43F81C2CC26843F8102C02220B
:1018E00003F8082C002203F8072CA3F11800704716
:1018F0002103000810B5202383F31188FFF7DEFFD2
:1019000000210446FFF798FF002383F31188204647
:1019100010BD0000024B1B6958610F20FFF760BF2C
:1019200008260020202383F31188FFF7F3BF00006F
:1019300008B50146202383F311880820FFF75EFFD6
:10194000002383F3118808BD49B1064B42681B6927
:1019500018605A60136043600420FFF74FBF4FF0D8
:10196000FF307047082600200368984206D01A68A6
:101970000260506059611846FFF7F4BE70470000DE
:1019800038B504460D462068844200D138BD03684E
:1019900023605C604561FFF7E5FEF4E7054B03F16A
:1019A00014025A619A614FF0FF32DA6100221A6222
:1019B000704700BF08260020F8B503614FF0804350
:1019C000C2605C6A194B1A46022952F8145F38BF8C
:1019D0000221954206461F460AD1586198611C6251
:1019E0000560456081600819BDE8F84001F08AB9DA
:1019F000186AAB68241A0C1902D3E41A2D6804E0A3
:101A00009C4202D2204401F08BF9AB689C42F4D88E
:101A10006B68736035601E606E60B460A9684FF0DB
:101A2000FF33091BA960FB61F8BD00BF0826002039
:101A300010B41B4C234653F8141F814210D0416848
:101A400002680A60026851609A424FF00001C1606A
:101A500003D0936881680B4493605DF8044B704732
:101A60000A68626100209A425360C86003D15DF841
:101A7000044B01F04FB993688868034493604FF0BA
:101A80008042206A526A121A9342E6D9991A0129B1
:101A900098BF931C18445DF8044B01F041B900BF96
:101AA0000826002000207047FEE700007047000075
:101AB0004FF0FF3070470000022906D0032906D0FE
:101AC0000129064818BF0020704705487047032ABF
:101AD0009ABF044800EBC20000207047243500087C
:101AE000D83400080824002070B59AB001AD06462D
:101AF00008462946144600F095F82846FFF73EF9B7
:101B0000C0B2431C5B0086E8180023700323637097
:101B1000002302341946DAB2904204F1020401D8DB
:101B20001AB070BDEA5C04F8022C04F8011C013301
:101B3000F1E7000008B5202383F311880348FFF77D
:101B4000E9FA002383F3118808BD00BF482600206E
:101B500010B50446052916D8DFE801F0161503165E
:101B6000161D202383F311880E4A0121FFF772FB13
:101B700020460D4A0221FFF76DFB0C48FFF790FA53
:101B8000002383F3118810BD202383F311880748B5
:101B9000FFF75CFAF4E7202383F311880348FFF78B
:101BA00073FAEDE7583400087C340008482600201A
:101BB00038B50C4D0C4C0D492A4604F10800FFF7CE
:101BC00093FF05F1CA0204F110000949FFF78CFFE9
:101BD00005F5CA7204F118000649BDE83840FFF760
:101BE00083BF00BF102B002008240020A834000869
:101BF000B2340008BD34000870B5044608460D46EE
:101C0000FFF7BCF8C6B22046013403780BB918467A
:101C100070BD32462946FFF799F80028F3D101201C
:101C200070BD00002DE9F84F05460C46FFF7A6F8F9
:101C30002C49C6B22846FFF7DFFF08B10436F6B2DA
:101C400029492846FFF7D8FF08B11036F6B2632EAF
:101C50000DD8DFF89090DFF890A0DFF89880DFF8DB
:101C600098B0224F2E7846B92670BDE8F88F2946E5
:101C70002046BDE8F84F01F09BBB252E2DD1072251
:101C800049462846FFF762F850B93B6823607B68F5
:101C900063603B892381BB7AA37207350B34E1E78C
:101CA000082251462846FFF751F8B0B9104BA21C44
:101CB00013F8011F09095B4511F8081002F8021C0E
:101CC000197801F00F0102F1020211F8081002F870
:101CD000031CEDD118340835C4E7267001350134F2
:101CE000C0E700BF44350008BD3400084C3500088B
:101CF0000F7AFF1F583500081B7AFF1FBFF34F8F65
:101D0000024AD368DB03FCD4704700BF003C0240AA
:101D100008B5094B1B7873B9FFF7F0FF074B1A6939
:101D2000002ABFBF064A5A6002F188325A601A6818
:101D300022F480621A6008BD6E2D0020003C024033
:101D40002301674508B50B4B1B7893B9FFF7D6FF06
:101D5000094B1A6942F000421A611A6842F4805233
:101D60001A601A6822F480521A601A6842F480627B
:101D70001A6008BD6E2D0020003C02400B2870B593
:101D800013D80B4A0B4C137863B90B4E4FF000611C
:101D900044F8231056F8235001330C2B2944F7D173
:101DA0000123137054F8200070BD002070BD00BFE7
:101DB000A02D0020702D00206C350008014B53F839
:101DC000200070476C3500080C2070470B2810B5B8
:101DD000044601D9002010BDFFF7D0FF064B53F891
:101DE00024301844C21A0BB9012010BD1268013208
:101DF000F0D1043BF6E700BF6C3500080B2810B5A6
:101E0000044621D8FFF77AFFFFF782FF0F4AF3233A
:101E1000D360C300DBB243F4007343F002031361E9
:101E2000136943F480331361FFF768FFFFF7A6FFE0
:101E3000074B53F8241000F0DDF8FFF783FF20462E
:101E4000BDE81040FFF7C2BF002010BD003C0240BB
:101E50006C3500082DE9F84312F00103154640D116
:101E60008218B2F1016F3CD22C4B1B6813F00103B6
:101E700037D02B4CFFF74CFFF323E360FFF73EFF17
:101E800040F20127032D01D9830713D0244C0F46BC
:101E9000401A40F20118EB1B0B44012B00EB070624
:101EA000236924D823F001032361FFF74BFF0120AE
:101EB000BDE8F883236923F44073236123693B431E
:101EC000236151F8046B0660BFF34F8FFFF716FFD5
:101ED00003689E4208D0236923F001032361FFF7C2
:101EE00031FF0020BDE8F883043D0430CAE723F445
:101EF00040732361236943EA08032361B94637F835
:101F0000023B3380BFF34F8FFFF7F8FE3688B9F8F6
:101F10000030B6B2B342BED0DDE700BF00380240A9
:101F2000003C0240084908B50B7828B153B9FFF7C7
:101F3000EFFE01230B7008BD23B1BDE80840087017
:101F4000FFF700BF08BD00BF6E2D002010B5024492
:101F5000064B0439D2B2904200D110BD441C00B2ED
:101F600053F8200041F8040FE0B2F4E75028004095
:101F7000104B30B51C6F240407D41C6F44F400745C
:101F80001C671C6F44F400441C670B4C236843F42B
:101F9000807323600244094B0439D2B2904200D1CD
:101FA00030BD441C00B251F8045F43F82050E0B249
:101FB000F4E700BF003802400070004050280040A5
:101FC00007B5012201A90020FFF7C0FF019803B067
:101FD0005DF804FB13B50446FFF7F2FFA04206D0FC
:101FE00002A9012241F8044D0020FFF7C1FF02B011
:101FF00010BD000070470000034B1B689B0042BFF0
:10200000024B01221A70704774380240A12D002043
:10201000014B1878704700BFA12D002070470000C9
:10202000FEE70000084A094B09498B4204D3094ADC
:102030000021934205D3704752F8040F43F8040B74
:10204000F3E743F8041BF4E71437000818300020C6
:102050001830002018300020836D30B500229D68B4
:10206000446D11464FF0FF3004EB421301329542AC
:10207000C3F80019C3F81019C3F80809C3F8001B06
:10208000C3F8101BC3F8080BEED24FF00113C4F8CD
:102090001C3830BD890141F02001016103699B06B4
:1020A000FCD4122000F0C4BE204B03EB80022DE9CB
:1020B000F047D2F80CE05D6DDEF81420461CD2F833
:1020C00000C005EB063605EB4018516861450BD39F
:1020D000D5F83428012303FA00F022EA0000C5F8FD
:1020E00034081846BDE8F087BEF81040ACEB010399
:1020F000A34228BF2346D8F81849A4B2B3EB840FF3
:1021000010D894681F46A4F1040959F804AFC6F822
:1021100000A0042F01D9043FF7E71C440B4494604E
:102120005360D2E70020BDE8F08700BFA42D002057
:1021300010B5054C2046FFF76DF84FF0A0436365DE
:10214000024BA36510BD00BFA42D0020C0350008C0
:102150000378012B70B5054650D12A4B446D984247
:102160001BD1294B5A6B42F080025A635A6D42F0E0
:1021700080025A655A6D5A6942F080025A615A6962
:1021800022F080025A610E2143205B6900F0D6FBE9
:102190001E4BE3601E4BC4F800380023C4F8003E19
:1021A000C02323606E6D4FF40413A3633369002BC7
:1021B000FCDA012333610C2000F03AFE3369DB07BF
:1021C000FCD4122000F034FE3369002BFCDA002628
:1021D000A6602846FFF740FF6B68C4F81068DB680C
:1021E000C4F81468C4F81C684BB90A4BA3614FF0DB
:1021F000FF336361A36843F00103A36070BD064B26
:10220000F4E700BFA42D0020003802404014004035
:1022100003002002003C30C0083C30C0F8B5446DDB
:10222000054600212046FFF735FFA96D00234FF03A
:1022300001128F68C4F834384FF00066C4F81C28C7
:102240004FF0FF3004EB431201339F42C2F80069A4
:10225000C2F8006BC2F80809C2F8080BF2D20B688A
:102260006A6DEB65636210231361166916F0100640
:10227000FBD1122000F0DCFDD4F8003823F4FE631B
:10228000C4F80038A36943F4402343F01003A3616A
:102290000923C4F81038C4F814380A4BEB604FF027
:1022A000C043C4F8103B084BC4F8003BC4F81069A5
:1022B000C4F80039EB6D03F1100243F48013EA65B2
:1022C000A362F8BD9C35000840800010426D90F874
:1022D0004E10D2F8003823F4FE6343EA0113C2F82B
:1022E000003870472DE9F0410EB200EB86080D462C
:1022F000D8F80C100F6807F00303022B50D0032B03
:1023000050D03D4A3D4F012B18BF1746446D4FEA50
:10231000451E04EB0E030022C3F8102B8A6905F159
:10232000100C002A40D04A8A05F158035B013A4359
:10233000E2500123D4F81C2803FA0CF31343A644FB
:102340004A69C4F81C380023CEF8103905F13F0360
:10235000002A39D00A8A898B9208012988BF4A430A
:10236000C16D04EB8303561841EA0242C665294653
:102370005A602046FFF78EFED8F80C301B8A43EADD
:1023800085531F4305F148035B01E7500123D4F84F
:102390001C2803FA05F51543C4F81C58BDE8F08164
:1023A000174FB3E7174FB1E704EB4613D3F8002BF1
:1023B00022F40042C3F8002BD4F81C28012303FAAE
:1023C0000CF322EA0303BAE704EB83030E4A5A60D4
:1023D00004EB461629462046FFF75CFED6F8003986
:1023E00023F40043C6F80039D4F81C38012202FA5D
:1023F00005F523EA0505CFE70080001000800410F2
:102400000080081000800C1000040002826D126829
:10241000C265FFF721BE00005831436D49015B588A
:1024200013F4004004D013F4001F14BF0120022055
:10243000704700004831436D49015B5813F4004078
:1024400004D013F4001F14BF0120022070470000C5
:1024500000EB8101CB68196A0B6813604B6853600D
:102460007047000000EB810330B5DD68AA6913688E
:10247000D36019B9402B84BF402313606B8A146862
:10248000426D1C44013CB4FBF3F46343033323F07B
:10249000030302EB411043EAC44343F0C043C0F8D6
:1024A000103B2B6803F00303012B09B20ED1D2F8C5
:1024B000083802EB411013F4807FD0F8003B14BFC2
:1024C00043F0805343F00053C0F8003B02EB41124D
:1024D000D2F8003B43F00443C2F8003B30BD00009B
:1024E0002DE9F041244D6E6D06EB40130446D3F800
:1024F000087BC3F8087B38070AD5D6F814381907C3
:1025000006D505EB84032146DB6828465B689847BF
:10251000FA072FD5D6F81438DB072BD505EB840343
:10252000D968CCB98B69488A5E68B6FBF0F200FBCB
:1025300012628AB91868DA6890420DD2121A83E8DA
:102540001400202383F311880B482146FFF78AFFEC
:1025500084F31188BDE8F081012303FA04F26B894A
:1025600023EA02036B81CB6823B121460248BDE810
:10257000F0411847BDE8F081A42D002000EB810355
:1025800070B5DD68436D6C692668E6604A0156BB2C
:102590001A444FF40020C2F810092A6802F003021E
:1025A000012A0AB20ED1D3F8080803EB421410F442
:1025B000807FD4F8000914BF40F0805040F00050F4
:1025C000C4F8000903EB4212D2F8000940F00440BD
:1025D000C2F80009D3F83408012202FA01F10143DC
:1025E000C3F8341870BD19B9402E84BF4020206054
:1025F00020682E8A841940F00050013C1A44B4FB34
:10260000F6F440EAC440C6E7F8B504461E48456DF6
:1026100005EB4413D3F80869C3F80869F10717D527
:10262000D5F81038DA0713D500EB8403D9684B6965
:102630001F68DA68974218D2D21B00271A605F60C1
:10264000202383F311882146FFF798FF87F3118831
:10265000330617D5D5F834280123A340134211D0EF
:102660002046BDE8F840FFF71FBD012303FA04F23E
:10267000038923EA020303818B68002BE8D02146FB
:102680009847E5E7F8BD00BFA42D002096482DE946
:10269000F84F456D6E69AB691E4016F4805F6E6140
:1026A000044605D0FEF722FEBDE8F84F00F054BC0A
:1026B000002E12DAD5F8003E8B489B071EBFD5F8D6
:1026C000003E23F00303C5F8003ED5F8043823F09C
:1026D0000103C5F80438FEF733FE370502D58248FA
:1026E000FEF722FEB0040CD5D5F8083813F0060F1B
:1026F000EB6823F470530CBF43F4105343F4A0531E
:10270000EB60310704D56368DB680BB17648984706
:10271000F2025AD4B3020CD5D4F85480DFF8C8A121
:1027200000274FF00109A36D9B68F9B28B4280F03E
:102730008780F70619D5616D0A6AC2F30A1702F09D
:102740000F0302F4F012B2F5802F00F0A180B2F571
:10275000402F0AD104EB830301F58051DB68186A2E
:1027600000231A469F4240F087803003D5F818486E
:1027700013D5E10302D50020FFF7B2FEA20302D574
:102780000120FFF7ADFE630302D50220FFF7A8FE8C
:10279000270302D50320FFF7A3FE750384D5E007C6
:1027A00002D50020FFF730FFA10702D50120FFF777
:1027B0002BFF620702D50220FFF726FF23077FF5D4
:1027C00073AF0320FFF720FF6EE7D4F85480DFF8E3
:1027D00018A100274FF00109A36D9B685FFA87FBE2
:1027E0005B4597D308EB4B13D3F8002902F4402242
:1027F000B2F5802F22D1D3F80029002A1EDAD3F8AF
:10280000002942F09042C3F80029D3F80029002A99
:10281000FBDB5946606DFFF73DFC228909FA0BF39B
:1028200022EA0303238104EB8B03DB689B6813B16B
:102830005946504698475846FFF736FC0137CBE7D4
:1028400008EB4112D2F8003B03F44023B3F5802F8C
:1028500010D1D2F8003B002B0CDA628909FA01F39F
:1028600022EA0303638104EB8103DB68DB680BB1BD
:1028700050469847013756E79C0708BF0A68072B60
:1028800098BF027003F101039CBF120A013069E78F
:10289000023304EB830201F58051526890690268AB
:1028A000D0F808C04068A2EB000E00221046974204
:1028B0000AD104EB830463689B699A683A449A607E
:1028C0005A6817445F6050E712F0030F08BF0868AA
:1028D000964588BF8CF8000002F1010284BF000A0F
:1028E0000CF1010CE3E700BFA42D0020436D03EBC6
:1028F0004111D1F8003B43F40013C1F8003B70478D
:10290000436D03EB4111D1F8003943F40013C1F8D2
:1029100000397047436D03EB4111D1F8003B23F4BC
:102920000013C1F8003B7047436D03EB4111D1F830
:10293000003923F40013C1F80039704700F16043F7
:1029400000F01F02400903F5614309018000C9B28C
:1029500000F1604083F8001300F5614001239340CB
:10296000C0F880310360704730B5039C01720433B6
:1029700004FB0325C361049B03630021059B0060E6
:102980004060C160426102618561046242628162AD
:10299000C162436330BD00000022416A41610161B0
:1029A000C2608262C2626FF00101FEF7E9BF0000FF
:1029B00003694269934203D1C2680AB1002070479B
:1029C000181D704703691960C2680132C260C2698C
:1029D000134482690361934224BF436A0361002167
:1029E000FEF7C2BF38B504460D46E3683BB16269E5
:1029F000131D1268A3621344E362002038BD237ADA
:102A000033B929462046FEF79FFF0028EDDA38BD8E
:102A10006FF00100FBE70000C368C269013BC360BF
:102A20004369134482694361934224BF436A43610B
:102A300000238362036B03B11847704770B52023EE
:102A4000044683F31188866A3EB9FFF7CBFF05463B
:102A500018B186F31188284670BDA36AE26A13F89C
:102A6000015BA362934202D32046FFF7D5FF002308
:102A700083F31188EFE700002DE9F84F04460E4676
:102A800090469946202787F311880025AA46D4F856
:102A900028B0BBF1000F09D149462046FFF7A2FF3D
:102AA00020B18BF311882846BDE8F88FA16AE36A4C
:102AB000A8EB050B5B1A9B4528BF9B46BBF1400F5B
:102AC0001BD9334601F1400251F8040B43F8040BC3
:102AD0009142F9D1A36A40334036A3624035A26ADD
:102AE000E36A9A4202D32046FFF796FF8AF31188E1
:102AF0004545D8D287F31188C9E730465A46FEF7D4
:102B00001BF9A36A5B445E44A3625D44E7E70000EF
:102B100010B5029C0172043303FB0421C36100233E
:102B20008362C362039B0363049B00604060C460D4
:102B300042610261816104624262436310BD000030
:102B4000026AC260426A4261026100228262C2621B
:102B50006FF00101FEF714BF436902699A4203D185
:102B6000C2680AB100207047184650F8043B0B6059
:102B700070470000C368C2690133C36043691344EE
:102B800082694361934224BF436A43610021FEF797
:102B9000EBBE000038B504460D46E3683BB123693F
:102BA0001A1DA262E2691344E362002038BD237A51
:102BB00033B929462046FEF7C7FE0028EDDA38BDB6
:102BC0006FF00100FBE7000003691960C268013A79
:102BD000C260C269134482690361934224BF436A9D
:102BE000036100238362036B03B118477047000041
:102BF00070B5202304460E4683F31188856A35B9E3
:102C00001146FFF7C7FF10B185F3118870BDA36AA5
:102C10001E70A36AE26A01339342A36204D3E1699E
:102C200020460439FFF7D0FF002080F3118870BDE3
:102C30002DE9F84F04460D4691469A464FF020087C
:102C400088F311880026B346A76A4FB9514620463B
:102C5000FFF7A0FF20B187F311883046BDE8F88F59
:102C6000A06AE76AA9EB06033F1A9F4228BF1F46E6
:102C7000402F1BD905F1400355F8042B40F8042BD5
:102C80009D42F9D1A36A4033A3624036A26AE36A47
:102C90009A4204D3E16920460439FFF795FF8BF38C
:102CA00011884E45D9D288F31188CDE729463A4696
:102CB000FEF742F8A36A3B443D44A3623E44E5E785
:102CC000026943699A4203D1C3681BB91846704729
:102CD0000023FBE7836A002BF8D0043B9B1AF5D056
:102CE0001360C368013BC360C3691A44836902610E
:102CF0009A4224BF436A0361002383620123E5E70C
:102D000000F06CB94FF08043002258631A61022230
:102D1000DA6070474FF080430022DA6070470000AD
:102D20004FF0804358637047FEE7000010B5174C22
:102D3000FEF710FDFEF732FE802215492046FEF711
:102D4000B7FD012344F8180C0374124B124AD968DA
:102D500021F4E0610904090C0A431049DA60CA68E9
:102D600042F08072CA600E490A6842F001020A60AD
:102D70001022DA77202283F82220002383F311889F
:102D800062B60848BDE81040FEF7B4BD302600200A
:102D9000CC35000800ED00E00003FA05F0ED00E09E
:102DA000001000E0D43500082DE9F84F1F4C4FF01B
:102DB0000008656904F11407C1464FF08043266A94
:102DC0005B6AAA689E1B96421DD34FF0200AAA6830
:102DD000236AD5F80CB0134423622B68BB425F60B2
:102DE000A6EB02066361C5F80C8001D1FFF792FFE4
:102DF00089F311882869D8478AF311886569AB6817
:102E00009E42E4D2D9E76269BA420CD0916823624B
:102E10008E1B9660A86802282CBF1818981CBDE865
:102E2000F84FFFF77DBFBDE8F88F00BF08260020F0
:102E3000034B59685A68521A9042FBD8704700BF3A
:102E4000001000E04B6843608B688360CB68C36010
:102E50000B6943614B6903628B6943620B680360D2
:102E60007047000008B5224B22481A6940F2FF1152
:102E70000A431A611A6922F4FF7222F001021A61F0
:102E80001A691A6B0A431A631A6D0A431A651A4AB9
:102E90001B6D1146FFF7D6FF184802F11C01FFF722
:102EA000D1FF174802F13801FFF7CCFF154802F1B6
:102EB0005401FFF7C7FF144802F17001FFF7C2FF8A
:102EC000124802F18C01FFF7BDFF114802F1A80181
:102ED000FFF7B8FF0F4802F1C401FFF7B3FF0E4838
:102EE00002F1E001FFF7AEFFBDE8084000F0E0B8F6
:102EF0000038024000000240F4350008000402409F
:102F000000080240000C0240001002400014024081
:102F100000180240001C02400020024008B500F0EA
:102F200037FAFFF703FFFFF767F8BDE80840FEF741
:102F30003FBE000070470000064A536823F00103BB
:102F40005360EFF30983683383F30988002383F325
:102F50001188704730EF00E010B5202383F311880B
:102F6000104B5B6813F4006318D0F1EE103AEFF3E6
:102F700009844FF0807344F84C3C0B4BDB6844F8F9
:102F8000083CA4F1680383F30988FEF771FC18B1CB
:102F9000064B44F8503C10BD054BFAE783F311880B
:102FA00010BD00BF00ED00E030EF00E0310300088D
:102FB000340300084FF0804310B51A69920708D512
:102FC00000241C61202383F31188FFF7EDFE84F3B6
:102FD0001188BDE81040FFF7BFBF0000104B1A6C0E
:102FE00042F001021A641A6E42F001021A660D4A9A
:102FF0001B6E936843F0010393604FF080435322AC
:103000009A624FF0FF32DA6200229A615A63DA6004
:103010005A6001225A6108211A601C20FFF78EBCF9
:1030200000380240002004E01F4B1A696FEAC252C8
:103030006FEAD2521A611A69C2F308021A614FF09C
:10304000FF301A695A69586100215A6959615A69F1
:103050001A6A62F080521A621A6A02F080521A6288
:103060001A6A5A6A58625A6A59625A6A1A6C42F063
:1030700080521A641A6E42F080521A661A6E0B4A17
:10308000106840F480701060186F00F44070B0F564
:10309000007F1EBF4FF4803018671967536823F410
:1030A0000073536000F054B90038024000700040D3
:1030B000304B4FF080521A642F4A4FF44041116058
:1030C0001A6842F001021A601A689207FCD59A68E1
:1030D00022F003029A60274B19469A6812F00C02FC
:1030E000FBD1186800F0F90018609A601A6842F481
:1030F00080321A600B689B03FCD54B6F43F00103D1
:103100004B671C4B5A6F9007FCD51C4A5A601A68D3
:1031100042F080721A60184A53685904FCD5154B66
:103120001A689201FCD5164A9A60164B1A68164B1B
:103130009A42164B1BD1164A1168164A914216D173
:1031400040F205121A600B4B9A6842F002029A6034
:103150009A6802F00C02082AFAD15A6C42F48042B2
:103160005A645A6E42F480425A665B6E704740F26F
:103170000572E7E70038024000700040085440073D
:1031800000948838002004E011640020003C0240D4
:1031900000ED00E041C20F41084A08B553691168CB
:1031A0000B4003F00103536123B1054A13680BB1CF
:1031B00050689847BDE80840FFF7CEBE003C01408C
:1031C00088250020084A08B5536911680B4003F0B0
:1031D0000203536123B1054A93680BB1D068984745
:1031E000BDE80840FFF7B8BE003C0140882500203C
:1031F000084A08B5536911680B4003F00403536192
:1032000023B1054A13690BB150699847BDE80840DE
:10321000FFF7A2BE003C014088250020084A08B5FF
:10322000536911680B4003F00803536123B1054A49
:1032300093690BB1D0699847BDE80840FFF78CBE91
:10324000003C014088250020084A08B553691168F0
:103250000B4003F01003536123B1054A136A0BB10D
:10326000506A9847BDE80840FFF776BE003C014031
:1032700088250020174B10B55C691A68144004F4C7
:1032800078725A61A30604D5134A936A0BB1D06AC7
:103290009847600604D5104A136B0BB1506B9847E2
:1032A000210604D50C4A936B0BB1D06B9847E2050D
:1032B00004D5094A136C0BB1506C9847A30504D58B
:1032C000054A936C0BB1D06C9847BDE81040FFF7EE
:1032D00043BE00BF003C0140882500201A4B10B5BA
:1032E0005C691A68144004F47C425A61620504D592
:1032F000164A136D0BB1506D9847230504D5134A38
:10330000936D0BB1D06D9847E00404D50F4A136E4E
:103310000BB1506E9847A10404D50C4A936E0BB1C3
:10332000D06E9847620404D5084A136F0BB1506FF2
:103330009847230404D5054A936F0BB1D06F984783
:10334000BDE81040FFF708BE003C01408825002082
:10335000062108B50846FFF7F1FA06210720FFF716
:10336000EDFA06210820FFF7E9FA06210920FFF708
:10337000E5FA06210A20FFF7E1FA06211720FFF7F8
:10338000DDFA06212820BDE80840FFF7D7BA000083
:1033900008B5FFF749FEFDF78BFDFDF739FFFDF797
:1033A0000DFEFFF7C7FDBDE80840FFF7A9BC000010
:1033B000034611F8012B03F8012B002AF9D17047BD
:1033C000121012131211000053544D3332463F3F76
:1033D0003F00000000000000C83300083F0000006C
:1033E00013040000043400083F000000190400002A
:1033F0000E3400083F0000002104000018340008CB
:103400003F00000053544D3332463430780053545B
:103410004D3332463432780053544D3332463434CF
:103420003658580000000000350F0008210F000832
:103430005D0F0008490F0008550F0008410F0008F4
:103440002D0F0008190F0008B90F00080000000038
:103450000100000000000000020000000000000069
:1034600061110008C911000840004000E02A002056
:10347000F02A00200200000000000000030000000D
:10348000000000000D120008000000001000000005
:10349000002B0020000000000100000000000000E0
:1034A000A42D0020010102004172647550696C6F07
:1034B000740025424F415244252D424C002553456E
:1034C0005249414C25000000511B0008B91A000860
:1034D000CD100008351B000843000000E034000850
:1034E00009024300020100C0320904000001020287
:1034F000010005240010010524010001042402023A
:103500000524060001070582030800FF09040100E5
:10351000020A0000000705010240000007058102C1
:1035200040000000120000002C35000812011001BC
:10353000020000400912415700020102030100008D
:103540000403090425424F41524425007370656508
:10355000647962656566340030313233343536372C
:103560003839414243444546000000000040000015
:10357000004000000040000000400000000001008A
:103580000000020000000200000002000000020033
:103590000000020000000200000002000000000025
:1035A0005513000835160008E116000840004000D9
:1035B000042E0020042E002001000000142E002004
:1035C0008000000040010000030000006D61696E92
:1035D00000000000EC350008202E002018300020EC
:1035E00001000000292D00080000000069646C65DE
:1035F000000000000000800200000000AAAAAAAAA1
:1036000000000000FFFF00000000000000A00A0012
:103610000004500000000000AAAAAAAA000050005E
:10362000DFFF0000000000000000000001000000BB
:1036300000000000AAAAAAAA01000000FFFF0000E3
:10364000000000000000000000000000000000007A
:10365000AAAAAAAA00000000FFFF000000000000C4
:10366000000000000000000000000000AAAAAAAAB2
:1036700000000000FFFF000000000000000000004C
:103680000000000000000000AAAAAAAA0000000092
:10369000FFFF00000000000000000000000000002C
:1036A00000000000AAAAAAAA00000000FFFF000074
:1036B000000000000000000000000000000000000A
:1036C0000A000000000000000300000000000000ED
:1036D00000000000000000000000000000000000EA
:1036E00000000000000000000000000000000000DA
:1036F000FF009600000000080400000040350008AC
:1037000000000000000000000000000000000000B9
:103710000000000000000000FFFFFFFFFFFFFFFFB1
:10372000FFFFFFFFFFFFFFFFFFFFFFFFFFFFFFFFA9
:10373000FFFFFFFFFFFFFFFFFFFFFFFFFFFFFFFF99
:10374000FFFFFFFFFFFFFFFFFFFFFFFFFFFFFFFF89
:10375000FFFFFFFFFFFFFFFFFFFFFFFFFFFFFFFF79
:020000040801F1
:10000000000600208912010849820608A581060819
:1000100011820608A5810608DD8106088B120108F9
:100020008B1201088B1201088B120108D562080897
:100030008B1201088B1201088B1201088B12010828
:100040008B1201088B1201088B1201088B12010818
:100050008B1201088B120108F17408081975080841
:10006000417508086975080891750808F51E0808A3
:100070001D1F0808491F0808751F0808A11F080848
:10008000C91F0808F51F0808791E08088B12010807
:100090008B1201088B1201088B120108B975080830
:1000A000DD760808F176080805770808097708085A
:1000B0000D7708088B1201088B12010881250808AA
:1000C000292708088B1201088B1201088B120108DE
:1000D0008B1201088D7608088B120108A17608089A
:1000E0001D7608088B1201088B1201083177080869
:1000F00035770808497708084D770808212008084F
:100100008B1201088B120108217708088B12010855
:10011000B5760808C97608088B1201088B12010809
:100120004D20080875200808A1200808CD200808DF
:10013000F92008088B1201088B1201088B120108A4
:100140008B1201088B1201088B120108016A080842
:10015000212108084D210808792108088B1201087F
:100160008B1201088B1201088B1201088B120108F7
:100170008B1201088B1201088B1201088B120108E7
:100180008B1201088B1201088B1201088B120108D7
:100190008B1201088B1201088B1201088B120108C7
:1001A0008B1201088B1201088B1201088B120108B7
:1001B0008B1201088B1201088B1201088B120108A7
:1001C0008B1201088B1201088B1201088B12010897
:1001D0008B1201088B1201088B1201088B12010887
:1001E000212701080D370108619B0108A5ED0208D0
:1001F000816A0408ED84040889D104084DD90408F3
:1002000085DC0408C53B05084157050845C90508B4
:10021000157B06082D16070881470708659C070807
:10022000BDC207083DCD0708FDFA0708C50008084C
:1002300081F0004102E000BF83F0004330B54FEA97
:1002400041044FEA430594EA050F08BF90EA020F04
:100250001FBF54EA000C55EA020C7FEA645C7FEA97
:10026000655C00F0E2804FEA5454D4EB5555B8BFBA
:100270006D420CDD2C4480EA020281EA030382EA2B
:10028000000083EA010180EA020281EA0303362DBD
:1002900088BF30BD11F0004F4FEA01314FF4801C90
:1002A0004CEA113102D0404261EB410113F0004FA2
:1002B0004FEA03334CEA133302D0524263EB430359
:1002C00094EA050F00F0A780A4F10104D5F1200EF7
:1002D0000DDB02FA0EFC22FA05F2801841F1000152
:1002E00003FA0EF2801843FA05F359410EE0A5F126
:1002F00020050EF1200E012A03FA0EFC28BF4CF057
:10030000020C43FA05F3C01851EBE37101F000450C
:1003100007D54FF0000EDCF1000C7EEB00006EEB19
:100320000101B1F5801F1BD3B1F5001F0CD34908A3
:100330005FEA30004FEA3C0C04F101044FEA4452FA
:1003400012F5800F80F09A80BCF1004F08BF5FEA81
:10035000500C50F1000041EB045141EA050130BD61
:100360005FEA4C0C404141EB0101013C28BFB1F573
:10037000801FE9D291F0000F04BF01460020B1FABE
:1003800081F308BF2033A3F10B03B3F120020CDA91
:100390000C3208DD02F1140CC2F10C0201FA0CF06F
:1003A00021FA02F10CE002F11402D8BFC2F1200CD4
:1003B00001FA02F120FA0CFCDCBF41EA0C0190408A
:1003C000E41AA2BF01EB0451294330BD6FEA0404D3
:1003D0001F3C1CDA0C340EDC04F11404C4F12002BE
:1003E00020FA04F001FA02F340EA030021FA04F3D0
:1003F00045EA030130BDC4F10C04C4F1200220FA27
:1004000002F001FA04F340EA0300294630BD21FA64
:1004100004F0294630BD94F0000F83F4801306BF2A
:1004200081F480110134013D4EE77FEA645C18BF1E
:100430007FEA655C29D094EA050F08BF90EA020FB5
:1004400005D054EA000C04BF1946104630BD91EAAD
:10045000030F1EBF0021002030BD5FEA545C05D1B0
:100460004000494128BF41F0004130BD14F58004EF
:100470003CBF01F5801130BD01F0004545F0FE4163
:1004800041F470014FF0000030BD7FEA645C1ABF98
:10049000194610467FEA655C1CBF0B46024650EACF
:1004A000013406BF52EA033591EA030F41F40021FB
:1004B00030BD00BF90F0000F04BF0021704730B581
:1004C0004FF4806404F132044FF000054FF0000156
:1004D00050E700BF90F0000F04BF0021704730B517
:1004E0004FF4806404F1320410F0004548BF4042EC
:1004F0004FF000013EE700BF42004FEAE2014FEA41
:1005000031014FEA02701FBF12F07F4393F07F4F1B
:1005100081F06051704732F07F4208BF704793F01E
:100520007F4F04BF41F40021704730B54FF4607431
:1005300001F0004521F000411CE700BF50EA010234
:1005400008BF704730B54FF000050AE050EA0102DD
:1005500008BF704730B511F0004502D5404261EB4D
:1005600041014FF4806404F132045FEA915C3FF48E
:10057000D8AE4FF003025FEADC0C18BF03325FEA2B
:10058000DC0C18BF033202EBDC02C2F1200300FADC
:1005900003FC20FA02F001FA03FE40EA0E0021FA01
:1005A00002F11444BDE600BF70B54FF0FF0C4CF4EF
:1005B000E06C1CEA11541DBF1CEA135594EA0C0FA1
:1005C00095EA0C0F00F0DEF82C4481EA030621EADC
:1005D0004C5123EA4C5350EA013518BF52EA033517
:1005E00041F4801143F4801338D0A0FB02CE4FF0C9
:1005F0000005E1FB02E506F00042E0FB03E54FF0F9
:100600000006E1FB03569CF0000F18BF4EF0010EF0
:10061000A4F1FF04B6F5007F64F5407404D25FEAEC
:100620004E0E6D4146EB060642EAC62141EA55519F
:100630004FEAC52040EA5E504FEACE2EB4F1FD0CE1
:1006400088BFBCF5E06F1ED8BEF1004F08BF5FEA5F
:10065000500E50F1000041EB045170BD06F0004611
:1006600046EA010140EA020081EA0301B4EB5C04BE
:10067000C2BFD4EB0C0541EA045170BD41F48011B6
:100680004FF0000E013C00F3AB8014F1360FDEBFDB
:10069000002001F0004170BDC4F10004203C35DAB7
:1006A0000C341BDC04F11404C4F1200500FA05F33A
:1006B00020FA04F001FA05F240EA020001F00042DB
:1006C00021F0004110EBD37021FA04F642EB060151
:1006D0005EEA430E08BF20EAD37070BDC4F10C047B
:1006E000C4F1200500FA04F320FA05F001FA04F23F
:1006F00040EA020001F0004110EBD37041F100012B
:100700005EEA430E08BF20EAD37070BDC4F1200535
:1007100000FA05F24EEA020E20FA04F301FA05F29D
:1007200043EA020321FA04F001F0004121FA04F245
:1007300020EA020000EBD3705EEA430E08BF20EA15
:10074000D37070BD94F0000F0FD101F0004640004F
:1007500041EB010111F4801F08BF013CF7D041EAD1
:10076000060195F0000F18BF704703F000465200D5
:1007700043EB030313F4801F08BF013DF7D043EAA6
:100780000603704794EA0C0F0CEA135518BF95EA5C
:100790000C0F0CD050EA410618BF52EA4306D1D1E3
:1007A00081EA030101F000414FF0000070BD50EA02
:1007B000410606BF1046194652EA430619D094EA8C
:1007C0000C0F02D150EA013613D195EA0C0F05D176
:1007D00052EA03361CBF104619460AD181EA0301CA
:1007E00001F0004141F0FE4141F470014FF0000082
:1007F00070BD41F0FE4141F4780170BD70B54FF01D
:10080000FF0C4CF4E06C1CEA11541DBF1CEA13559C
:1008100094EA0C0F95EA0C0F00F0A7F8A4EB05047E
:1008200081EA030E52EA03354FEA013100F0888075
:100830004FEA03334FF0805545EA131343EA12633E
:100840004FEA022245EA111545EA10654FEA0026F3
:100850000EF000419D4208BF964244F1FD0404F5AC
:10086000407402D25B084FEA3202B61A65EB030508
:100870005B084FEA32024FF480104FF4002CB6EBC5
:10088000020E75EB030E22BFB61A754640EA0C0045
:100890005B084FEA3202B6EB020E75EB030E22BF85
:1008A000B61A754640EA5C005B084FEA3202B6EBC6
:1008B000020E75EB030E22BFB61A754640EA9C0085
:1008C0005B084FEA3202B6EB020E75EB030E22BF55
:1008D000B61A754640EADC0055EA060E18D04FEA13
:1008E000051545EA16754FEA06164FEAC30343EAB3
:1008F00052734FEAC2025FEA1C1CC0D111F4801F80
:100900000BD141EA00014FF000004FF0004CB6E778
:1009100011F4801F04BF01430020B4F1FD0C88BF17
:10092000BCF5E06F3FF6AFAEB5EB030C04BFB6EB22
:10093000020C5FEA500C50F1000041EB045170BD15
:100940000EF0004E4EEA113114EB5C04C2BFD4EB42
:100950000C0541EA045170BD41F480114FF0000EC6
:10096000013C90E645EA060E8DE60CEA135594EA42
:100970000C0F08BF95EA0C0F3FF43BAF94EA0C0F45
:100980000AD150EA01347FF434AF95EA0C0F7FF4BA
:1009900025AF104619462CE795EA0C0F06D152EA0E
:1009A00003353FF4FDAE1046194622E750EA4106F2
:1009B00018BF52EA43067FF4C5AE50EA41047FF403
:1009C0000DAF52EA43057FF4EBAE12E74FF0FF3C68
:1009D00006E000BF4FF0010C02E000BF4FF0010C39
:1009E0004DF804CD4FEA410C7FEA6C5C4FEA430CB2
:1009F00018BF7FEA6C5C1BD001B050EA410C0CBF01
:100A000052EA430C91EA030F02BF90EA020F002062
:100A1000704710F1000F91EA030F58BF994208BFC9
:100A200090422CBFD8176FEAE37040F00100704786
:100A30004FEA410C7FEA6C5C02D150EA013C07D1DD
:100A40004FEA430C7FEA6C5CD6D152EA033CD3D028
:100A50005DF8040B704700BF8446104662468C4622
:100A60001946634600E000BF01B5FFF7B7FF002855
:100A700048BF10F1000F01BD4DF808EDFFF7F4FF7E
:100A80000CBF012000205DF808FB00BF4DF808ED09
:100A9000FFF7EAFF34BF012000205DF808FB00BF2C
:100AA0004DF808EDFFF7E0FF94BF012000205DF84E
:100AB00008FB00BF4DF808EDFFF7CEFF94BF012003
:100AC00000205DF808FB00BF4DF808EDFFF7C4FFFC
:100AD00034BF012000205DF808FB00BF4FEA410C45
:100AE0007FEA6C5C02D150EA013C0AD14FEA430C28
:100AF0007FEA6C5C02D152EA033C02D14FF0000065
:100B000070474FF0010070474FEA410212F50012A2
:100B100015D211D56FF47873B3EB625212D94FEA44
:100B2000C12343F0004343EA505311F0004F23FA2E
:100B300002F018BF404270474FF00000704750EA83
:100B4000013005D111F0004008BF6FF00040704740
:100B50004FF00000704700BF4A0011D212F500129A
:100B600011D20DD56FF47873B3EB62520ED44FEA05
:100B7000C12343F0004343EA505323FA02F0704785
:100B80004FF00000704750EA013002D14FF0FF30C3
:100B900070474FF0000070474FEA4102B2F1E04366
:100BA00024BFB3F5001CDCF1FE5C0DD901F0004C54
:100BB0004FEAC0024CEA5070B2F1004F40EB8300A4
:100BC00008BF20F00100704711F0804F21D113F1D0
:100BD0003872BCBF01F00040704741F480114FEA09
:100BE0005252C2F11802C2F1200C10FA0CF320FA92
:100BF00002F018BF40F001004FEAC1234FEAD323AF
:100C000003FA0CFC40EA0C0023FA02F34FEA430318
:100C1000CCE77FEA625307D150EA01331EBF4FF0A1
:100C2000FE4040F44000704701F0004040F0FE40BC
:100C300040F40000704700BF80F0004002E000BFB9
:100C400081F0004142001FBF5FEA410392EA030FB7
:100C50007FEA226C7FEA236C6AD04FEA1262D2EB01
:100C60001363C1BFD218414048404140B8BF5B4206
:100C7000192B88BF704710F0004F40F4000020F09F
:100C80007F4018BF404211F0004F41F4000121F0B5
:100C90007F4118BF494292EA030F3FD0A2F10102FF
:100CA00041FA03FC10EB0C00C3F1200301FA03F13D
:100CB00000F0004302D5494260EB4000B0F5000F60
:100CC00013D3B0F1807F06D340084FEA310102F11F
:100CD0000102FE2A51D2B1F1004F40EBC25008BFD1
:100CE00020F0010040EA03007047490040EB00009B
:100CF000013A28BFB0F5000FEDD2B0FA80FCACF19C
:100D0000080CB2EB0C0200FA0CF0AABF00EBC250C8
:100D100052421843BCBFD0401843704792F0000FB6
:100D200081F4000106BF80F400000132013BB5E709
:100D30004FEA41037FEA226C18BF7FEA236C21D07F
:100D400092EA030F04D092F0000F08BF08467047E4
:100D500090EA010F1CBF0020704712F07F4F04D1B2
:100D6000400028BF40F00040704712F100723CBFC5
:100D700000F50000704700F0004343F0FE4040F4EF
:100D8000000070477FEA226216BF08467FEA2363AD
:100D90000146420206BF5FEA412390EA010F40F498
:100DA000800070474FF0000304E000BF10F00043E4
:100DB00048BF40425FEA000C08BF704743F09643CB
:100DC00001464FF000001CE050EA010208BF7047E6
:100DD0004FF000030AE000BF50EA010208BF70476D
:100DE00011F0004302D5404261EB41015FEA010C82
:100DF00002BF84460146002043F0B64308BFA3F17A
:100E00008053A3F50003BCFA8CF2083AA3EBC2535B
:100E100010DB01FA02FC634400FA02FCC2F120027A
:100E2000BCF1004F20FA02F243EB020008BF20F0B1
:100E30000100704702F1200201FA02FCC2F1200217
:100E400050EA4C0021FA02F243EB020008BF20EA0C
:100E5000DC7070477BB972B90029BEBF00204FF02B
:100E6000004106E008BF00281CBF6FF000414FF0B2
:100E7000FF3000F007BAADF1080C6DE904CE00298F
:100E800009DB002B1ADB00F095F8DDF804E0DDE962
:100E9000022304B07047404261EB4101002B1BDB91
:100EA00000F088F8DDF804E0DDE9022304B04042F8
:100EB00061EB4101524263EB43037047524263EBE3
:100EC000430300F077F8DDF804E0DDE9022304B025
:100ED000404261EB41017047524263EB430300F033
:100EE00069F8DDF804E0DDE9022304B0524263EB67
:100EF0004303704753B94AB9002908BF00281CBFF3
:100F00004FF0FF314FF0FF3000F0BCB9ADF1080CED
:100F10006DE904CE00F04EF8DDF804E0DDE90223CF
:100F200004B07047430803F05533C01A830803F038
:100F3000333300F03330184400EB101000F00F3062
:100F400000EB002000EB0040000E704707EE900A17
:100F5000F5EEC07AF1EE10FA01D400F00BB8F1EE24
:100F6000677A08B517EE900A00F004F8404261EB8A
:100F7000410108BDD0B5FFF7BFFA0C4B0022064671
:100F80000F46FFF711FBFFF7E7FD0446FFF792FA64
:100F9000074B0022FFF708FB02460B463046394656
:100FA000FFF74AF9FFF7D8FD2146D0BD0000F03D1C
:100FB0000000F0412DE9F047089D04468E46002BC5
:100FC0004DD18A42944669D9B2FA82F252B101FAFD
:100FD00002F3C2F1200120FA01F10CFA02FC41EA0D
:100FE000030E94404FEA1C48210CBEFBF8F61FFA92
:100FF0008CF708FB16E341EA034306FB07F199422D
:101000000AD91CEB030306F1FF3080F01F819942DF
:1010100040F21C81023E63445B1AA4B2B3FBF8F0B9
:1010200008FB103344EA034400FB07F7A7420AD940
:101030001CEB040400F1FF3380F00A81A74240F268
:1010400007816444023840EA0640E41B00261DB1D3
:10105000D4400023C5E900433146BDE8F0878B4208
:1010600009D9002D00F0EF800026C5E900013046C7
:101070003146BDE8F087B3FA83F6002E4AD18B42A1
:1010800002D3824200F2F980841A61EB030301204B
:101090009E46002DE0D0C5E9004EDDE702B9FFDE37
:1010A000B2FA82F2002A40F09280A1EB0C014FEAE2
:1010B0001C471FFA8CFE0126200CB1FBF7F307FB3F
:1010C000131140EA01410EFB03F0884208D91CEBE2
:1010D000010103F1FF3802D2884200F2CB8043467F
:1010E000091AA4B2B1FBF7F007FB101144EA01445E
:1010F0000EFB00FEA64508D91CEB040400F1FF31ED
:1011000002D2A64500F2BB800846A4EB0E0440EADA
:1011100003409CE7C6F12007B34022FA07FC4CEAE3
:10112000030C20FA07F401FA06F31C43F9404FEAD6
:101130001C4900FA06F3B1FBF9F8200C1FFA8CFEEB
:1011400009FB181140EA014108FB0EF0884202FA3F
:1011500006F20BD91CEB010108F1FF3A80F0888000
:10116000884240F28580A8F102086144091AA4B2BD
:10117000B1FBF9F009FB101144EA014100FB0EFE3E
:101180008E4508D91CEB010100F1FF346CD28E456D
:101190006AD90238614440EA0840A0FB0294A1EBFE
:1011A0000E01A142C846A64656D353D05DB1B3EB5B
:1011B000080261EB0E0101FA07F722FA06F3F1408B
:1011C0001F43C5E9007100263146BDE8F087C2F132
:1011D0002003D8400CFA02FC21FA03F391400143AA
:1011E0004FEA1C471FFA8CFEB3FBF7F007FB1036E3
:1011F0000B0C43EA064300FB0EF69E4204FA02F48F
:1012000008D91CEB030300F1FF382FD29E422DD9E1
:10121000023863449B1B89B2B3FBF7F607FB163316
:1012200041EA034106FB0EF38B4208D91CEB010196
:1012300006F1FF3816D28B4214D9023E6144C91A16
:1012400046EA004638E72E46284605E70646E3E626
:101250001846F8E64B45A9D2B9EB020864EB0C0E30
:101260000138A3E74646EAE7204694E74046D1E73F
:10127000D0467BE7023B614432E7304609E76444ED
:10128000023842E7704700BF02E000F000F8FEE7D6
:1012900072B6374880F30888364880F309883648A4
:1012A0003649086040F20000CCF200004EF634717E
:1012B000CEF200010860BFF34F8FBFF36F8F40F293
:1012C0000000C0F2F0004EF68851CEF20001086036
:1012D000BFF34F8FBFF36F8F4FF00000E1EE100AA6
:1012E0004EF63C71CEF200010860062080F31488AF
:1012F000BFF36F8F75F04CF875F096FF4FF05530D7
:101300001F491B4A91423CBF41F8040BFAE71D49B3
:10131000184A91423CBF41F8040BFAE71A491B4AAC
:101320001B4B9A423EBF51F8040B42F8040BF8E7FE
:1013300000201849184A91423CBF41F8040BFAE7D3
:1013400075F02AF875F0C4FF144C154DAC4203DA61
:1013500054F8041B8847F9E701F0D2F9114C124DFB
:10136000AC4203DA54F8041B8847F9E775F012B869
:1013700000060020002200200000010808ED00E027
:101380000000002000060020C0570A0800220020AC
:10139000C8250020C8250020E8190120E001010827
:1013A0003002010830020108300201082DE9F04F37
:1013B0002DED108AC1F80CD0C3689D46BDEC108A93
:1013C000BDE8F08F002383F311882846A047002052
:1013D00073F062FFFEE773F0BFFD00DFFEE7000081
:1013E00001F0FF01102A2BDB10F0070F08D010F8D6
:1013F000013B013A8B422DD010F0070F42B3F6D1DA
:10140000F0B441EA012141EA014122F007047FF0F2
:1014100000070023F0E80256083C85EA010586EA49
:10142000010685FA47F5A3FA87F586FA47F6A5FA85
:1014300087F68EB9EED1F0BC01F0FF0102F0070291
:1014400032B110F8013B013A83EA010313B1F8D13C
:101450000020704701387047002D06BF354603381D
:10146000073815F0010F07D1013015F4807F02BF56
:10147000013015F4C03F0130F0BC0138704700BFA7
:1014800010F8012B11F8013B012A28BF9A42F7D02E
:10149000D01A7047034613F8012B002AFBD1181A03
:1014A0000138704738B50022002304460D46FFF787
:1014B000EDFA28B920462946BDE8384000F00AB8C0
:1014C000204605F1004100F005F8404261EB410182
:1014D00038BD00BFD0B50C4B002206460F46FFF7C3
:1014E00063F8FFF739FB0446FEF7E4FF074B0022E1
:1014F000FFF75AF802460B4630463946FEF79CFE87
:10150000FFF72AFB2146D0BD0000F03D0000F0416E
:1015100000207047704700007047000070470000CF
:10152000002070470020704700207047012070475E
:10153000002070477047000000207047002070476F
:10154000704700007047000000207047002070477F
:1015500070B5154ED6F8380203681B689847042802
:101560001ADC01281DDC002814BF012441240F4B84
:101570001D68E86A0368DB69984701280AD0D6F835
:1015800038220B4B9A4205D0EB6A93F89C300BB192
:1015900044F08004204670BD0A2814BF0124192499
:1015A000E5E71924E3E700BFD0550020CC25002053
:1015B00010580020044BD3F8380203F51072904203
:1015C00014BF042002207047D0550020014B93F82F
:1015D00048017047D04500207047000038B5C578F5
:1015E0000B461C2D044628BF1C251C220021184632
:1015F00078F050FE2A4604F10C01BDE8384078F03E
:10160000FFBD000038B5C5780B46102D044628BF35
:10161000102510220021184678F03CFE2A4604F1DD
:101620000C01BDE8384078F0EBBD000008B53EF095
:10163000EBF930B9034A92F8CC3243F0040382F854
:10164000CC3208BDD055002038B591ED000AF7EE38
:10165000000A0D4618F098FB20B10B4801F0DCFEA3
:10166000002038BDD5ED007A9FED087AF0EEE77ADC
:10167000F4EEC77AF1EE10FA03D5034801F0DEFE6E
:10168000EEE70320EDE700BFD02500200000003486
:1016900010B5044608F072FA204610BD13B58B8BC6
:1016A000B72B0C4607D0B3F5967F21D002B0BDE82A
:1016B000104041F027BE124912481E2201F0E6FEFA
:1016C000D4ED017A94ED007A0D48FCEEE77ABCEE99
:1016D000C77A17EE903A8DED017A9DF804109AB210
:1016E00001F074FB002814BF0020042002B010BDDC
:1016F00004480549022201F0C9FE0020F6E700BFB8
:1017000038580020D02500200C58002000B51F4A72
:10171000DFED1F6AD2EDB17A92EDB07AD2F8B41251
:10172000007CA2F580538BB093F96A310491002BB1
:1017300018BFB0EE677AD2EDAB7A8DED057AFDEE8B
:10174000E77A3E2117EE903AD2EDAC7AF4EEE67AE3
:10175000F1EE10FA58BFF0EE667AFCEEE77A1BB2B3
:10176000ADF82030ADF8223017EE903A0022039207
:1017700006920792ADF82430B7221A23CDE9003241
:1017800003AA3BF0C5FB0BB05DF804FBD05500206D
:1017900000FF7F4770B5154C94F8D2228AB022B969
:1017A0000AB0BDE870403CF07FBE057C56F082FD7B
:1017B000D4E98C61D4F82C32A4F50054CDE905139A
:1017C000B4F86824ADF826200023CDE90733ADF83E
:1017D000243068221C23CDE90306CDE90032212103
:1017E00003AA28463BF094FB0AB070BDD0550020F8
:1017F000F0B53B4CB4F88C31DE078DB0054637D5DB
:10180000D4F84032089302238DF82430D4F85032B3
:10181000D4F84402CDF82530D4F84C32D4F838123C
:10182000D4F83C220590CDF8293062202123D4F849
:101830003062D4F82C720691CDE90030C221192310
:10184000287C079203AA049603973BF061FB287C4F
:101850003BF0F4FA0646287C3CF0F4F900F1210351
:101860009E4205D2287C0DB0BDE8F0403AF062BD42
:10187000B4F88C31990731D5D4F828330893032371
:101880008DF82430D4F83833D4F82423CDF825301B
:10189000D4F83433D4F82C03D4F820130792CDF8BD
:1018A000293062222123D4F81863D4F814730590E8
:1018B000CDE90032287C0691192303AAC22103979F
:1018C00004963BF025FB287C3BF0B8FA0446287CC4
:1018D0003CF0B8F900F121039C42C3D30DB0F0BD38
:1018E000D045002005207047024BD3F8380203682A
:1018F0001B681847D055002030B5CD788BB0272D08
:1019000028BF27250C4627220021684678F0C2FC14
:101910002A4604F10C01684678F072FC1A4BD3F8A1
:10192000381203F5127291422BD1DDED057A9FED4D
:10193000177AF0EEE77AF4EEC77AF1EE10FA20D5D6
:101940009DF8262002F0410141291AD1110618D430
:1019500002F01801182914D00199C3F84C1282F032
:1019600004020299C3F85012C2F380020399C3F82B
:10197000541283F85C220499079AC3F85812C3F8EA
:1019800060220BB030BD00BFD055002000000034F5
:1019900030B5194D95F8D13285B00C464BBBCA789D
:1019A0008DF80C30092A28BF09220C3101A8CDE995
:1019B000013378F025FC9DF808305A1F012A18D908
:1019C00003F0F703122B14D0A5F58053B3F94A2185
:1019D00012B9E279A3F84A21227AE179074800F0A6
:1019E000B1F9227AE179054800F0E4F9012385F89C
:1019F000D13205B030BD00BFD0550020B05000201E
:101A0000F0B51B4BB3F94A3189B005460E46144672
:101A10003BB1D779BB4204D009B0BDE8F0403FF0FC
:101A2000FBBFA27A637A43EA0223E27A43EA0243E3
:101A30001D2B13D0212B08D01BB921462846FFF7B8
:101A4000A7FF224631462846E6E701A92046FFF7D0
:101A5000C5FD084801A901F09FFFF2E701A9204652
:101A6000FFF7D0FD034801A901F0ECFFE9E700BF53
:101A7000D0450020D025002013B5CA78072A4FF0A2
:101A80000003044628BF07220C3168460093CDF8B6
:101A9000033078F0B5FBBDF900304BB901231C21B0
:101AA000204684F80F3302B0BDE8104041F0E2BB9D
:101AB00002B010BD30B5CD7889B01E2D28BF1E25CF
:101AC0000C461E220021684678F0E4FB2A4604F109
:101AD0000C01684678F094FB0248694601F0FEFF6D
:101AE00009B030BDD025002000B589B0084601A955
:101AF000FFF774FD034801A901F04EFF09B05DF83E
:101B000004FB00BFD02500201FB508466946FFF73B
:101B100079FD0348694601F095FF05B05DF804FBC7
:101B2000D02500202DE9F041CC7894B0262C28BF98
:101B3000262488462622002107460AA878F0AAFB18
:101B400002AD224608F10C010AA878F059FB28469C
:101B500007F070FD9DF84A30022B06AC03D0032B32
:101B600044D0002B66D1DFED357ADDED106A9FEDB4
:101B7000346A9DED0F7A66EEA76ADDED0E7A27EEE8
:101B8000067A67EE867A0023FDEEE66ABDEEC77A36
:101B9000FDEEE77A17EE102A17EE901A0093204612
:101BA00016EE903A07F066FD94E80F0085E80F0006
:101BB00097F80F3363BB012698F8083098F8072090
:101BC0008DF8193000238DF818208DF81B309922DC
:101BD0000423CDE90032387C8DF81A6003232246B5
:101BE0002F213BF095F914B0BDE8F081DFED137AB9
:101BF000DDED106A9FED126A9DED0F7A66EEA76A21
:101C0000DDED0E7A27EE067A67EE867A0123BBE7D2
:101C1000BDF8446086B90B483246294601F0D4FB32
:101C20000028C8D0084A062138463DF081FB87F8D5
:101C30000F63C1E70226BFE70026BDE70000C842E8
:101C40008096184BD025002004E5080838B58A7A1C
:101C50004B7A43EA0223CA7A43EA0243272B05461A
:101C60000C460CD81C2B10D91D3B0A2B0DD8DFE8D5
:101C700003F01E0C0C0C1B0C0C0C0C121500452B4D
:101C80000FD0522B01D1FFF737FE21462846BDE881
:101C9000384040F0CFB9FFF7EFFEF6E7FFF742FF1D
:101CA000F3E7FFF707FFF0E7FFF71EFFEDE7FFF7AA
:101CB0002BFFEAE700207047C820704701207047DB
:101CC00000207047002070470120704790F8903046
:101CD0008B4286BF00EB8100D0F894000020704753
:101CE00090F890308B4286BF00EB8100D0F89400D2
:101CF00000207047014B93F846017047D045002003
:101D0000036A43F4E0530362436A43F4E0534362DB
:101D1000836A43F4E05383627047000013B54FF4C5
:101D20004470CDE9002107F021FF044628B1DDE928
:101D3000002140F0E3FE024B2360204602B010BDBC
:101D4000A0E608082DE9F04FDFF8649085B006465C
:101D50000F46904600254FF4837A96F89030ECB207
:101D6000A34222D920463BF069F8834620463BF047
:101D700069FF031D9B4514D399F96B31ADF8083009
:101D800094220623CDE90032422102AA20468DF892
:101D90000A708DF80B80ADF80CA03BF0B9F8013556
:101DA000DBE720463AF0C6FAF9E705B0BDE8F08F68
:101DB000D04500202DE9F04FDFF8649085B006464D
:101DC0000F469046002540F2011A96F89030ECB28A
:101DD000A34222D920463BF031F8834620463BF00F
:101DE00031FF031D9B4514D399F96B31ADF80830D1
:101DF00094220623CDE90032422102AA20468DF822
:101E00000A708DF80B80ADF80CA03BF081F801351D
:101E1000DBE720463AF08EFAF9E705B0BDE8F08F2F
:101E2000D04500201FB500F54053002100F5935028
:101E3000D3F8B4220191D3F8AC32029201A9083050
:101E4000039301F0ABFF03F077FB03F041F905B01A
:101E50005DF804FB70B586B006461322002101A888
:101E600010EE105A10EE904A78F014FAA3238DF871
:101E7000043095238DF8053056F024FA1322CDF85E
:101E80000700CDF80B1006F57C6001A9CDF80F50C6
:101E9000CDF8134037F024FA06B070BD2DE9F041BB
:101EA0008AB00446884617460021232201A8109DC7
:101EB0001E4678F0EFF9A3238DF8043095238DF8B2
:101EC000053001238DF8063056F0FCF92B68CDF86B
:101ED0001B306B68CDF80700CDF80B10CDF81F3024
:101EE0002322AB68CDF80F8001A904F57C60CDF802
:101EF0001370CDF81760CDF8233037F0F1F90AB040
:101F0000BDE8F0819720704710B500F540530446B6
:101F1000D3F8380203681B6898471A22C1B204F547
:101F20007C6037F09DFB04F59070BDE810400FF029
:101F3000CFBF000037B500F505510446012204313A
:101F400035F0AAFF012504F5FF51104A0095002342
:101F50001031DA2033F0BEFD0D4A0095002304F560
:101F60007C61FD2033F0B6FD0A4B1A68D20705D418
:101F7000094A1D6004F58C540C3414600648012194
:101F800003B0BDE8304033F0F7BD00BF14170A08B6
:101F9000389C0908C8250020002200200020704736
:101FA000002070470069C0F3401070470F299DBFA3
:101FB000302303FB010050300020704700207047A1
:101FC0000120704770470000036800221B68184713
:101FD00000207047002070470020704700207047A5
:101FE0000020704700207047002070470020704795
:101FF0000020704700207047704700001020704795
:102000000020704770470000032070470120704790
:1020100070470000012070470020704770470000A3
:1020200000F506501430704700487047D40A09087C
:1020300008B500F54050D0F8380203681B6898478F
:10204000C0B208BD034808600F2111704FF0FF3285
:102050001A6070476422090800207047002070470A
:102060007047000015F030BF37F0A0BA41F032BC25
:102070003FF024BE05F0CCBB06F07EBA00F0D4BE23
:1020800000F0CEBE00F0ECBE01F024BC00F0BABE01
:1020900000F0C0BE00F02ABF70B51F4B036000F512
:1020A00000530446D3F8900C1C4AC3F8E02A08B148
:1020B00007F068FD1A4B236004F5805393F82C2E2B
:1020C00042B9D3F8285E2DB1284614F0E7FD284622
:1020D00007F054FD04F58B50103053F043FC04F529
:1020E0008350183043F0C8FC04F6C44504F6644637
:1020F000B54204D0183D284614F03EFAF8E7094BE3
:10210000C4F8983804F6941039F080F804F510609B
:1021100039F07CF8204670BD9823090844B40908BA
:102120009C950908946C090838B5484B044640F85A
:10213000043B43F019FE04F1100006F043FB04F1E8
:10214000680035F01BF904F590700FF0A3FA04F560
:10215000866005F0CDF904F2545007F015FD04F641
:10216000980015F055FD04F5446043F085FD04F535
:10217000516034F025FE04F57C6036F0F9FF04F57B
:102180008350183043F060FC04F58550143006F09D
:1021900005FC04F58B50103053F0D0FB04F58C5047
:1021A0000C3035F0F7FB04F58F5044F087FF04F551
:1021B00080530025264A83F8045204F5905004F514
:1021C000905304331430136030F09CFF04F59350A7
:1021D0002946083001F0D8FE04F5C55018304CF0FF
:1021E000FBFA04F5E5501C3050F006FC04F5EE5007
:1021F000143052F0FDFC04F5F150183053F032F970
:1022000004F5F450103001F01FFD04F5FF501030BC
:102210004CF006FF04F50150083049F031FE04F59A
:10222000005304F5045083F804510A4D1C3053F058
:10223000D5FE2B6813B1084856F00AF82046074926
:1022400033F0C0FE2C60204638BD00BF9C950908C5
:10225000CC630020485B002064200908D49409085E
:1022600010B59FED225A9FED224A9FED222ADFED05
:10227000221A9FED221A9FED220A86B00446F0EE44
:10228000453AB0EE453AF0EE452AF0EE450AF7EE53
:10229000004A54308DED054A8DED042ACDED031A28
:1022A0008DED021A8DED015A8DED000A4CF034F8D7
:1022B0009DED015A9DED054A9DED042ADDED031AC1
:1022C0009DED021A9DED000AF7EE004AF0EE453A48
:1022D000B0EE453AF0EE452AF0EE450A04F59E7060
:1022E0004CF01AF8204606B010BD00BF00000000F8
:1022F000CDCCCC3D00007A450AD7A33CCDCC4C3D9B
:10230000CDCC4C3EF0B500F50055224BB5F846213A
:102310001A7087B0044643F00DFA42F0C3FF20461E
:1023200001F00CFC04F5805393F8E42412F0010250
:1023300010D102A8019207F07DF904F5935002A98B
:10234000083002F0DBFE28B12368019ADB6C02A999
:1023500020469847104E3368DB6A93F89C7037B17B
:1023600095F806311BB955F0A5FFC5F8080133688B
:1023700085F80671DB6A93F89C20084B5A7135F09A
:102380006FFA34F0C1FF04F50A5007B0BDE8F04021
:102390004CF012B805230020CC250020755A0020EF
:1023A000FFF7B0BF10B50821044601F0ABF918B132
:1023B00017F0EAF815F0F8FA0121204601F0A2F929
:1023C00010B12046FFF72EFD0421204601F09AF9B6
:1023D00018B104F57C6036F041FB1021204601F075
:1023E00091F928B104F57C60BDE8104036F0D0BB0F
:1023F00010BD0000FFF7D6BF102925D8DFE801F097
:10240000090D11191524242424241D2424242424F2
:10241000210000F549500430704700F549502C3038
:10242000704700F549502430704700F54950083096
:10243000704700F549502830704700F548503C304F
:10244000704700F5495070470020704708B54CF0C0
:10245000EBFE044B1B68DB6A93F89C10BDE8084058
:102460004CF0BEBECC250020FFF7F0BF2DE9FF41A8
:102470000446FFF759FE884B236004F5055004F528
:1024800000550430FFF7ECFE002304F50D50C5F8AD
:1024900068332C3041F03CFCDFF860827F4BC5F89C
:1024A0006C3342F2BC3642F2BC67A01941F0BEFD6B
:1024B00044F806803036BE42F7D1A01943F01AF82E
:1024C00004F52B50043039F0E3F804F52B501030AC
:1024D00039F0DEF804F52B570023A5F8DC3A203755
:1024E0006F4BC5F8E03A07F1080055F099F804F58C
:1024F0002C5604F52D580C3608F1300830461436A9
:102500003DF00EFE4645F9D10723C5F8943C002363
:10251000A5F8983C4FF4CB7007F02EFBC5F8900C53
:1025200004F532501C3055F07BF804F53350203060
:1025300055F076F85B4B1A6802B91F605A4BC5F824
:10254000E03A0026594B03930294009604AB04F53D
:10255000335013E90C0040213C3005F0A5FC04F594
:10256000485004F54055283007F064F804F5495305
:10257000C5F838324E4BC5F83C324E4BC5F84032A8
:102580004D4BC5F844324D4BC5F848324FF07E53A1
:10259000C5F84C324A4BC5F8643204F54958494BEA
:1025A000C5F868320027484BC5F86C3208F130088E
:1025B000C5F85872C5F85472C5F8507208F1040095
:1025C00007F038F808F1140007F034F83F4B4048A2
:1025D000C5F89C7204F54B52C5F8A072C5F8A472F8
:1025E0001860103233464FF6FF774FF0140C9EB24E
:1025F0000CFB06010133097C0029F8D1354B364923
:102600001E800B6813B1354855F022FE85F8D13293
:1026100004F54B50012385F8D23214300A6053F090
:102620008BFD2F4BC5F8D4322E4BC5F82843C5E996
:10263000CB342D4B04F54D50C5E9CD342B4BC5F8AB
:102640003C33103006F0F6FF04F54D502C3006F008
:10265000F1FF04F54E50083006F0ECFF04F54C563F
:10266000234BC5F89C33A5F8A07306F1A40006F02F
:10267000E1FF4FF0FF330C36C5F800341D4B1E4907
:102680001E60304633F09EFC2046A5F84873A5F83E
:10269000647304B0BDE8F081982309084820090854
:1026A00044B40908645E002074E708089520010816
:1026B0000C240908F02009085424090840240908BA
:1026C000682409080421090818210908105B002062
:1026D000801A09080C5B0020CC5A002078200908D9
:1026E000B0200908592001085D2001086120010877
:1026F0000000FFFF445A0020C87809089C20090800
:1027000038B5054B1C6823680A461D68034B014613
:102710002046A847002038BDCC250020D025002029
:1027200010B555F0F3F9064C064B18602046FFF73C
:102730009DFE2046044A0549BDE8104075F07CB86E
:10274000D0250020CC25002064B500209920010868
:1027500038B52DED028B0D46F0EE608AB0EE408A62
:10276000144602F0E9FE90ED937AD0ED957A67EE8B
:10277000877A90ED927A67EEA87AE7EE087AC5ED4F
:10278000007AD0ED920AD0ED937A90ED957A67EECB
:10279000A07A67EEA80AE7EE480ABDEC028BC4ED0A
:1027A000000A38BD30B52DED068B83B0F0EE409AAF
:1027B000B0EE60AA0D46044602F0BEFED0ED7F7A70
:1027C000D0F80002B8EEE79A17F0AAFB07EE900ADD
:1027D000F8EEE78A79EEC9AA3AEE688AFDEEEAAA2F
:1027E000B0EE480A17F07EFBBDEEC00A5DB110EEF8
:1027F000103ADFED190A002BCCBF38EE608A38EEB4
:10280000208ABDEEC80AF8EEC00A01AAB8EEEA0AAC
:1028100069462046FFF79CFFDFED107A104B009AC7
:10282000C3F8B82269EEA79A019AC3F8BC2229EE30
:10283000279A2AEE27AA68EEA78AA3F58053C3ED4C
:102840008B9A83ED8C9A83EDC5AAC3EDC68A03B03B
:10285000BDEC068B30BD00BF00A00C470AD7233C5F
:10286000D055002038B52DED028B0D46B0EE408AD4
:10287000F0EE608A144602F05FFED0ED937A9FED91
:10288000147AF0EEE77AF4EEC77AF1EE10FA1DD47E
:10289000D0ED957A90ED927A67EEE87AE8EE077AD5
:1028A000C5ED007A90ED937AD0ED957A90ED926A2D
:1028B000C7EE876A0120C6EE077A67EEA80AE6EE41
:1028C000880AC4ED000ABDEC028B38BD0020FAE78F
:1028D0000000003430B55F4C2DED068BB4F9843127
:1028E000DFED5D8A5B4285B008EE103A054604F6DE
:1028F000C42038F0D1FEB8EEC88A90ED00AAB4F931
:10290000843128EE288AF6EE009A98EE29AA04F679
:10291000C42008EE103A38F0BFFEB8EEC88A90ED39
:10292000009AB4F9883128EE288A04F52D6098EED3
:10293000299A08EE103A38F0AFFEB4F98A31D0ED9A
:10294000009A04F52D600AEE903A38F0A5FEB8EE34
:10295000C88AF8EEEAAAD8EE289A6A4602A990ED4B
:10296000008A8DED00AA9AEEA88A2846F0EE4A0A5F
:10297000B0EE690A8DED038A8DED019ACDED029AD4
:10298000FFF770FF01AA03A9F0EE490AB0EE480A6A
:102990002846FFF767FF02F0CFFDD0F8000217F0DE
:1029A000BFFA04F58053D4ED5F7A93EDAB0A30EEB5
:1029B000270A08EE100A20EE280A17F093FAB8EE5C
:1029C000C88A30EE480A17F08DFADFED247A9DEDC3
:1029D000007AB5EEC00AF1EE10FAACBF70EE676A8D
:1029E000F0EE406AB4EEE67AB4BF70EE277AF0EE0D
:1029F000407AF1EE10FA2ADD9DED016AB4EEE76A45
:102A0000F1EE10FA23D5B5EEC00AF1EE10FA08DDAA
:102A100077EE665A37EEC65AF4EEC55AF1EE10FA62
:102A200013D4B5EEC00AF1EE10FA10D537EE667A7F
:102A300077EEC67AB4EEE77AF1EE10FACCBF012059
:102A4000002005B0BDEC068B30BD0120F9E7002069
:102A5000F7E700BFD04500200000C84200A00C47A7
:102A600070B5314C2DED028BA4F58055D5ED5F7A14
:102A700094EDAB0ADFED2D8A30EE270A84B020EE0C
:102A8000280A064617F02EFAB5F98A31D5ED607A94
:102A900001EE103AB5F98831B0EE408A00EE903A76
:102AA00094EDAD0AB8EEC11A30EE270AF8EEE00A4E
:102AB0000C2017F06BFA20EE280A30468DED010A43
:102AC000FFF708FF9DED010A0146F0EE480A304687
:102AD000FFF768FE9DED010A03AA02A9F0EE480A7D
:102AE0003046FFF735FEB5F98631002B0DDD07EED8
:102AF000903A94EDAC7AF8EEE77AB4EEE77AF1EE3C
:102B000010FA02DA94F870324BB99DED020A0848C7
:102B100000F00CFB9DED030A054800F0E3FB04B058
:102B2000BDEC028B70BD00BFD05500200000C84234
:102B3000D025002038B5484C94F8CC3213F0010170
:102B4000054643D1A4F580529FED447AB2F958214D
:102B500094EDAB0A07EE902AF8EEE77A13F0100F27
:102B600067EE877AF7EE006ABFEE007A08BFB0EE34
:102B7000667AA7EE270AC3F30012DFED397A84EDF7
:102B8000AB0AB5EEC00AF1EE10FA0AD51AB161F33C
:102B9000041384F8CC32B4EEE70AF1EE10FA06DC46
:102BA0000BE0B4EEE70AF1EE10FA06DD2AB994F86C
:102BB000CC3243F0100384F8CC329FED291ADFEDBC
:102BC000290A2C2017F0E2F984EDAB0A94F8CC32F4
:102BD0009807C3F340012ED4234A9FED207AB2F91F
:102BE0005A0107EE900AB2F98801B2F98A21F8EE8B
:102BF000E77A01EE102A00EE900A1A0767EE877A4C
:102C0000F8EEE00A94EDAD7AB8EEC11A18D577EE79
:102C1000677AF4EEE07AF1EE10FAC4EDAD7A03D5FE
:102C200061F3C30384F8CC3294EDAD0A3C2017F075
:102C3000ADF984EDAD0A2846BDE83840FFF710BF76
:102C400077EE877AF4EEC17AF1EE10FAC4EDAD7A40
:102C5000EADD43F00803E5E7D05500200AD7A33C9E
:102C60000000B44300000000D04500200A20704757
:102C700001207047094B93F87012024609B1FFF723
:102C8000EFBE93F8D11229B9A3F5805393F8903190
:102C9000DB0702D51046FFF74DBF7047D055002027
:102CA000042070470120704730B52DED028B8BB0AA
:102CB000044655F0FFFA07AB054606AA05A9201DF4
:102CC00018F082FE274A9FED288A136841F2883166
:102CD000EB1A8B421CD915603FF0F2FEDDED067A4F
:102CE00067EE887A054617EE900AFDF705FCDDEDE4
:102CF000077A67EE887ACDE9020117EE900AFDF7B0
:102D0000FBFB1A4ACDE900010621284639F008F9F3
:102D1000DDED067ADDED070A9FED150A60EE880A03
:102D200027EE888A60EE800A204628EE000A0021FD
:102D3000FFF738FDDDED070A9DED060A09AA08A98F
:102D40002046FFF705FD9DED080A0A4800F0EEF960
:102D50009DED090A074800F0C5FA0BB0BDEC028BE7
:102D600030BD00BFD8590020E02E65421824090864
:102D70000000C842D0250020002070470120704785
:102D8000024B014618680268126810476C5E00200A
:102D900008B50020FFF7F4FFC188472042F036FB5A
:102DA000472042F0FFF90120FFF7EAFFC1884820E1
:102DB00042F02CFBBDE80840482042F0F3B9000087
:102DC0000220704701207047FFF7B4BE08B50B46DC
:102DD000013BDBB2012B114611D85BB9472042F011
:102DE00015FB472042F0DEF942F0D4FB42F0BAF87E
:102DF000012008BD482042F009FB4820F2E70020EE
:102E0000F7E7000008B541F0DDF8BDE8084040F004
:102E1000B9BF000000F593500021083002F012BB4A
:102E200000F2545007F03ABB10B5044607F026FCF8
:102E300090F921308BB190F8403373B194F9783523
:102E40005BB1064B1B68DB6A93F89C302BB904F22C
:102E50005450BDE8104007F039B910BDCC25002012
:102E600070B5044600F590700FF08AFF94F8E433D3
:102E70001C4904EB0312D2F894010A68824210D074
:102E8000B02202FB034294F8285492F8C12145B9BC
:102E9000022A06D9144E08603278012A02D9013A72
:102EA000327070BDFDD104F54055D5F830222AB9F5
:102EB000D5F8342212B905233370F2E7B02202FBB1
:102EC000034303F5E6730FCB05F50A7585E80F009C
:102ED000236804F54851DB6C0022283120469847CE
:102EE0000023E9E7DC5900200C2200207047000095
:102EF00037B5044642F01EFC42F0D4F904F5005503
:102F00004721002042F0D0FA4821012042F0CCFABB
:102F1000B5F8841101EB810101EB8101490089B20F
:102F2000472042F029F9B5F98831B5F98A110F4DDA
:102F3000C91A01EB810101EB8101490089B24820E6
:102F400042F01AF942F026FB42F00CF804F52B503F
:102F500001A90430019538F031FC04F52B5001A98A
:102F60001030019538F02AFC03B030BDCDCCCC3DFB
:102F7000F0B52DED028B00F5005785B0B7F888212C
:102F8000B7F88A3104466425482012FB05F613FB86
:102F900005F542F0E1F804F5405304F50650183009
:102FA000B0EE408ADFED230A93EDAE0A01900021D6
:102FB0004BF06CFB07EE906A38EE000AF8EEE77A09
:102FC0000198B4EEE70AF1EE10FA25D98DED020A68
:102FD00007EE905A9DED027AF8EEE77AF4EEC77AA2
:102FE000F1EE10FA03D8CDED027A4BF043FA482007
:102FF0009DED020A42F09CF897F8DD3A04F52B505B
:10300000103083B10C4B039303AA02A938F0DAFB0A
:1030100005B0BDEC028BF0BD0190CDED027A4BF016
:1030200029FA0198D4E702A938F038FB012387F880
:10303000DD3AEDE70AD7A33C0AD7A33C00F540539D
:1030400000F50050D0ED5C7A90ED5E6A93EDAE7ABB
:1030500067EE867AF0EEC76AF4EEE76AF1EE10FAF0
:1030600004D59FED180A482042F062B8DFED167AC9
:10307000B5EEC07AF1EE10FA20EE270A10DDB0F8B6
:103080008831642213FB02F307EE903AF8EEE77AF8
:10309000F4EEC07AF1EE10FA02D59FED0C0AE2E7E9
:1030A000B0F88A31642213FB02F307EE903AF8EE8F
:1030B000E77AF4EEC07AF1EE10FA02DD9FED040A31
:1030C000D1E77047000000000000C84200A00CC615
:1030D00000A00C4610B5044600F5405304F500541A
:1030E00000F50650DFED100A93EDAE0A002118300E
:1030F0004BF0CCFAB4F98A01B4F988313221C21A02
:103100001B1A4A434B4301EE102A00EE903A8020EE
:10311000B8EEC11AF8EEE00A16F038FFBDE810402C
:10312000482042F005B800BF0AD7A33C00F5005381
:1031300093F96831012B03D0022B03D0FFF718BF9E
:10314000FFF77CBFFFF7C6BFF0B52DED028B00F592
:1031500000563223B6F88451DFED310A15FB03F532
:1031600000F50A5700F5405393EDAF0A83B00021F4
:10317000044638464BF08AFA9FED2A1ADFED2A0AF8
:10318000BF2016F003FF4720B0EE408A41F0E4FF75
:103190009FED241ADFED240A30EE080AC02016F055
:1031A000F5FE6B4207EE903AF8EEE77AB4EEE70AE6
:1031B000F1EE10FA26D98DED000A07EE905A9DED3A
:1031C000007AF8EEE77AF4EEC77AF1EE10FA04D856
:1031D0003846CDED007A4BF04DF947209DED000AC1
:1031E00041F0A6FF96F8DC3A04F52B5004307BB191
:1031F0000E4B019301AA694638F0E4FA03B0BDEC26
:10320000028BF0BD3846CDED007A4BF033F9D4E7B0
:10321000694638F043FA012386F8DC3AEEE700BF4E
:103220000AD7A33C00A08C4600A08CC60AD7A33CBA
:1032300000F540539FED117AD3EDAF7A00F50050C1
:1032400067EE877A90ED5D6A90ED5B7A27EE067AFD
:10325000F0EEE76AF4EEC76AF1EE10FA04D59FEDDE
:10326000080A472041F064BFF5EEC07AF1EE10FA8B
:10327000CCBF9FED040A9FED040AF2E70AD7233C76
:103280000000000000A08C4600A08CC610B50446CB
:1032900000F5405304F50054DFED110A93EDAF0A39
:1032A000002100F50A504BF0F1F9B4F984314FF6E2
:1032B000CE71322213FB02F213FB01F301EE102A4E
:1032C00000EE903AF120B8EEC11AF8EEE00AB1EE45
:1032D000400A16F05BFEBDE81040472041F028BFD1
:1032E0000AD7A33C00F5005393F96931012B03D0B1
:1032F000022B03D0FFF728BFFFF79ABFFFF7C6BF27
:10330000FEF702BE70B500F5005088B090F991014B
:103310000C46D8B105210E4842F0CAFA09210646EA
:103320000B4842F0C5FA01210390094842F0C0FA67
:1033300004AD00210346039A00912846314606F069
:1033400099F995E80F0084E80F00012008B070BDDE
:10335000E059002037B50C460022054611460F48BB
:1033600042F0B2FA62680D48012142F0C5FAA26843
:103370000A48052142F0C0FAE2680848092142F0F3
:10338000BBFA05F5065001240DF1070111308DF847
:10339000074033F00FFC204603B030BDE059002059
:1033A00037B503680191DD6C04460FF027FD90F8F6
:1033B000C412019AB02303FB0101AC3120462B4615
:1033C00003B0BDE8304018477FB5044604F5935676
:1033D000684608360D4606F02DF96946304601F07C
:1033E000B1FE48B929462046FFF7B4FF064650B95A
:1033F0000026304604B070BD2946304601F06CFD11
:103400000028EFD1F4E795E80F0004F5485428347C
:1034100084E80F00EDE7000010B5074B1B68044679
:10342000D86A036801211B68984704F57C60012174
:10343000BDE8104035F03CBFCC25002010B5074B4F
:103440001B680446D86A036800211B68984704F586
:103450007C600021BDE8104035F02ABFCC2500205B
:1034600010B5044654F026FF04F500540021C4F8BA
:103470006803472041F0E8FF0021482041F0E4FFC5
:1034800042F088F8BDE8104041F06CBD70B50446CC
:1034900004F5005304F5405583F80421D5F838327B
:1034A0008B420846164627D0C5F838120B685B6871
:1034B000984710B32046FFF7AFFFD5F838020368EE
:1034C0001B6898473246C1B204F57C6036F0C8F8F4
:1034D00004F52B500021203004F580543FF0EAFE23
:1034E00004F58D63D3ED007A9FED067AF8EEE77A66
:1034F00067EE877AC5EDAB7A70BD2046FFF79EFF79
:10350000DBE700BF0AD7233CF7B5044600F590502F
:1035100014302FF081FF5F4B04F5335001223C3013
:103520009A71DA7104F5866704F06AFD04F52B558B
:103530000823C4F844343846203504F0DFFB28461D
:103540003CF038FE284640F0C5F907F097F82023F4
:10355000036307F093F808F009F904F59356022382
:10356000C4F8743104F5907008360EF00FF9304647
:1035700000F078FE04F58053002283F87125B4F939
:10358000A43004F698001BB9B4F8A230A4F8A43013
:10359000B4F8A41016F06AF8304600F05DFF384623
:1035A000012104F045FA3C4B00933C4B019302ABE4
:1035B00013E9060004F57C6035F06EFE40F002FD74
:1035C0009922292141F00EFC40F0FCFC40F0A2FCC5
:1035D00004F500562046FFF78BFC96ED577ADFED99
:1035E000307AF0EEC76AF4EEE76AF1EE10FA04F50D
:1035F000405747D8D6ED587ADFED2A6AB0EEE76A31
:10360000B4EEE66AF1EE10FA3CD8DFED276A27EE59
:10361000267A67EEA67ABDEEC77AFDEEE77A87EDE9
:103620008C7AC7ED8D7AD7F8303243B9D7F8343277
:103630002BB904F5485128312046FFF763FE1B4B98
:103640001B68986A03684FF47A715B68984796F92B
:103650008E112046FEF7D0FE014610B904F54951FF
:1036600004311F222046FFF711FFD6ED597AF5EEFF
:10367000C07AF1EE10FA0BDD204603B0BDE8F04051
:10368000FFF7EEBE0A4A0521284638F049FCCAE792
:1036900003B0F0BD755A0020D02500200133010889
:1036A0000000B442000034438096184BCC25002023
:1036B0007424090808B50A2922D8DFE801F00D1999
:1036C00011151D2121212121060000F548513C3111
:1036D000FFF7DCFE012008BD00F549510431F7E792
:1036E00000F549512431F3E700F549512831EFE75E
:1036F00000F549512C31EBE700F549510831E7E776
:103700000020E8E700F57C6036F052BC0148032158
:1037100042F030B8E059002070B505462DED028B1F
:1037200005F5405454F0BAFDD4F89432DFED1D7A1B
:10373000C31A08EE103AB8EE488A28EE278AF1EE4E
:10374000047AB4EEE78AF1EE10FA29D504F51D7378
:103750000FCB04F5217686E80F00D4EDA80A94ED8E
:10376000A70A05F54A5068EE200A28EE000A043040
:1037700006F0F0F9DFED0C7A94EDA97A27EE277ABE
:10378000D4EDA27AF8EEE77A0123E7EE087AFDEEAF
:10379000E77AC4EDA27A84F87032BDEC028B70BD7A
:1037A0000023F8E7BD3786350000C84230B585B044
:1037B0006D460446284605F03DFF04F59350294622
:1037C000083001F09BFC50B104F54054002384F80C
:1037D000D23295E80F0004F50A7484E80F0005B0B2
:1037E00030BD0000F8B52DED028B00F540540546C4
:1037F00094F87032002B5ED0D4F8382200F549538B
:10380000243300F5485600F54A579A4206F1280637
:1038100007F1040717D094F8CC32DA0713D43946ED
:10382000304606F085F89FED277AF6EE007AE0EE56
:10383000077A9FED257AFDEEE77AF8EEE77A67EEF4
:10384000877AC4EDAB7A3946304606F013F905F5B0
:10385000005584EDAC0A95F96A31DFED1C6AD4F8A5
:103860003802012B05BFD4F88832D4F82C22D4EDCD
:10387000AA7A9B1A08BF07EE903AF8EEE77A87EE2D
:10388000A67A84EDB17A03681B689847022812D0A3
:1038900094F8CC329B070ED495F96A31D4EDAC0A7A
:1038A0009FED0B8A53B994EDB00A74F00DFB20EE36
:1038B000080A84EDAD0ABDEC028BF8BD94EDB10AA7
:1038C000F3E700BFA00CB3450AD7233C0000C84271
:1038D000E02E654273B50446FFF71EFF2046FFF752
:1038E00065FF04F500552046FFF77CFFD5ED597ABA
:1038F000F5EEC07AF1EE10FA09DC244B1E68F06A8E
:103900000368DB699847012816D102B070BD54F0F6
:10391000D1FCD5F8683395ED597ADFED1D6AC01AF0
:1039200007EE900A27EE267AF8EE677AF4EEC77A69
:10393000F1EE10FAE1D5E8E7F36A93F89C10E9B9E3
:1039400095F98F31012B10D19FED120A472041F0DC
:10395000EFFB9FED100A482041F0EAFB41F01AFE10
:1039600002B0BDE8704041F0FDBA4720019141F03E
:103970004DFD0199482041F049FDEFE704F5405421
:10398000D4F8380203689B689847E7E7CC25002005
:1039900000007A440000000037B54B68054613B9B3
:1039A0008A68002A49D005F540540A20C4F87C32C0
:1039B0008B68C4F88032CA6892FBF0F2C4F87822AF
:1039C0000B6993FBF0F3C4F8A832B1F91630DFEDC0
:1039D0001C7A07EE103AB1F91830B8EEC77A87EEC4
:1039E000276A07EE103AB1F9143084EDA86AB8EEF0
:1039F000C77AC7EE276A07EE103AB8EEC77AC4ED69
:103A0000A96AC7EE275AC4EDA75A54F047FCC4F878
:103A1000940254F04FFC0221C4F898022846FFF7A4
:103A200071FE50B105F54A531C330093D4E99F123F
:103A3000D4F878322846FEF731FA03B030BD00BF23
:103A40000000C84210B52DED028B044691ED018AAD
:103A5000DFED207A94F8413428EE278A00F586605D
:103A6000242202FB0303F0EE480A93ED090A03F057
:103A700087FCB4EE400AF1EE10FAF0EE400A1FD6D1
:103A80009FED157AF0EEC07AF4EE477AF1EE10FA77
:103A900016DC04F54053D3EDB27A93F8CC2277EEDE
:103AA000807A5107C3EDB07A0AD5F1EE407A002151
:103AB0006FF38202C3EDB27AC3F8C01283F8CC224E
:103AC000B0EE480ABDEC028B2046BDE81040FEF780
:103AD000C1B900BF0000C842FFFF7F7FB1F90030CD
:103AE00007EE903AF8EEE77A00F5405010B5C0EDD9
:103AF000AB7AB1F9023007EE903AF8EEE77A00239C
:103B0000C0F8B032C0EDAD7AB1F9002090F8CC32F7
:103B100047F6FF74121B18BF012262F3000380F8FE
:103B2000CC32B1F9023090F8CC221B1B18BF012314
:103B300063F3410280F8CC2210BD000010B500F5FF
:103B40004054D4F8980250B154F0B4FBD4F89832F1
:103B5000C01A41F2873398428CBF00200120014BEC
:103B6000187110BD755A002070B52DED028B00F54F
:103B700000541646B4F98A2194ED600A01EE102A29
:103B8000B4F9882100F54053D3EDAD7AD3EDAB8A7B
:103B900000EE902ADA20B8EEC11AF8EEE00A30EE14
:103BA000270A0D4616F0F2F9B4F98821B4F98A31E2
:103BB00007EE902AF8EEE77A9B1A30EE670A07EED6
:103BC000903A30EE000AF8EEE77AB7EE008A80EE1F
:103BD000277A37EE487A86ED007A94ED5F0A38EE60
:103BE000800A16F03FF9B4F9843107EE103A30EE4E
:103BF000000AB8EEC77A0120C0EE077A77EEC87ADD
:103C0000BDEC028BC5ED007A70BD0000704700006E
:103C10000020704770470000002070470020704768
:103C200000207047002070479FED010A704700BFD9
:103C3000000000009FED010A704700BF0000000077
:103C4000002070477047000010B50446143000F0A3
:103C500019F804F12C0000F015F804F1740054F088
:103C600035FB04F1F40054F031FB4FF0FF33C4F89E
:103C70005031204610BD0000014B1868704700BF4E
:103C8000E459002070470000F0B52DED048B91B091
:103C900004466D46284605F0CDFC94F8BC33002B55
:103CA00072D004F57A730FCB85E80F0094F8F833DF
:103CB000D4EDEC8A94EDED8A94EDEE9A002B63D06E
:103CC00094F8D033002B5FD02D22002104A8D4F823
:103CD000C073D4F8C463D4F8C853D4F8CC4376F096
:103CE000D9FAA3238DF8103095238DF8113046238F
:103CF0008DF8123054F0E6FA9FED250A9FED257AF3
:103D0000CDF8171068EE807ACDF8130067EE877A49
:103D1000FDEEE77A17EE903A68EE007A29EE000A97
:103D200067EE877AADF81B30FDEEE77A20EE070AE2
:103D300017EE903AADF81D3016F0BEF8DDED017AC1
:103D40009FED157ACDF82D70BCEEC00AF8EEE77A3B
:103D500010EE103A67EE877AADF81F3017EE903A02
:103D6000CDF82130029BCDF82530039BCDF82930CA
:103D7000CDF83160CDF83550CDF8394036F04EF9F8
:103D80002D2204A935F0ACFA11B0BDEC048BF0BDC6
:103D9000E02E65420000C8420AD7233C30B52DED25
:103DA000028B8BB0044624220D4601A8002176F038
:103DB00071FAA3238DF8043095238DF8053048233C
:103DC0009FED1F8A8DF8063054F07CFAD4ED817A8D
:103DD0002B68CDF80F3067EE887A95ED020ACDF8A2
:103DE0000B1017EE903AD4ED827ACDF8133067EECF
:103DF000887A6B68CDF8173017EE903ACDF8070047
:103E0000CDF81B3016F02EF810EE103A94ED830A20
:103E1000CDF81F3020EE080A16F024F810EE103A04
:103E2000CDF8233094F80C338DF8273036F0F6F8BF
:103E3000242201A935F054FA0BB0BDEC028B30BD41
:103E4000E02E654230B587B014460D461822002199
:103E5000684676F01FFAA3238DF8003095238DF87D
:103E6000013049238DF8023054F02CFAA3680393F3
:103E7000E36804936368CDF807100593CDF8030059
:103E80008DF80B5036F0CAF81822694635F028FA3A
:103E900007B030BD10B58EB0044602A805F0CAFBCD
:103EA00002A9204601F02AF9002845D001F044FB80
:103EB000694600F0BBFF1F22002106A876F0EAF950
:103EC000A3238DF8183095238DF819304A238DF8E7
:103ED0001A3054F0F7F9DDED037A9FED1B7A049B5D
:103EE000CDF82330F8EEE77A059BCDF8273067EE62
:103EF000877ACDF81B0017EE903ADDED007ACDF809
:103F00002B30F1EE677A17EE903ACDF81F1020466D
:103F100001A9CDF82F3000F0FDFB78B1DDED017A7D
:103F2000F1EE677A17EE903ACDF8333036F076F846
:103F30001F2206A935F0D4F90EB010BD36F06EF888
:103F4000DFED027AEEE700BF0AD7233C5241C07F83
:103F50000023036043608360C36003614361836146
:103F6000C36103627047000090F8C432B02202FBC4
:103F7000030390F8082393F8A13012B1012B28BF56
:103F800001231846704700002DE9F04F04468BB01E
:103F90004FF0000A0D461BF0F1FF84F814A204F55F
:103FA00006704FF07E5753F03BFB4FF47A73A4F842
:103FB000623284F86852C4F84872C4F84C72C4F88B
:103FC000507204F51B70002505F034FB04F52B79C5
:103FD0000323C4F8803204F53476C4F89452C4F84C
:103FE0009852C4F89C52C4F8A052C4F8A452C4F821
:103FF000A8524846FFF7ACFF04F5487B3046FFF770
:10400000A7FFC4F81453C4F81853C4F81C535846F7
:10401000FFF79EFFC4F84453C4F84853C4F84C5308
:10402000C4F85053C4F85453C4F85853C4F85C53FC
:10403000C4F86053C4F86453C4F86853C4F86C53AC
:10404000C4F87053C4F88C53C4F89053C4F8945314
:10405000C4F8A853C4F8A453C4F8A053C4F8B05388
:10406000C4F8B453C4F8B853C4F8CC53C4F8C85314
:10407000C4F8C453C4F89C73C4F8C07304F57570D5
:1040800005F0D8FA04F57A7005F0D4FA04F58063E7
:10409000C4F8FC531D6004F5816304F583601D6062
:1040A0005D609D6005F0C6FA04F22C4304F264489A
:1040B0001D605D609D60684BC4F83C3404F50D7371
:1040C000C4F8403404F50E73C4F8443404F50F7397
:1040D000C4F8483404F51073C4F84C3404F2452392
:1040E000C4F8503404F51173C4F8543404F58B63E8
:1040F00040461D605D609D60FFF72AFF04F59160FA
:10410000FFF726FF04F5976304F23C421D605D60F3
:104110009D6004F2C44304F2A4501D605D609D6084
:1041200004F59A631D605D609D6004F2DC431D60D0
:104130005D609D6004F2EC431D605D609D6004F273
:10414000FC431D605D609D6004F5A463C2F8D470FB
:10415000C2F8D8701D605D609D6004F22C531D6034
:104160005D609D6004F5A9631F605D6004F26C539F
:104170001D605D609D6004F5AF631D605D609D60C6
:1041800004F5B2631D605D609D6005F053FA04F2B2
:10419000B45324221D605D6004F2BC5351461D607F
:1041A0005D6004F2C45340461D605D6076F072F8B5
:1041B00004F2E450C8F82070C8F81070C8F8007015
:1041C000FFF7C6FE04F5C16304F5C7601D605D60BE
:1041D0009D6004F214631D605D609D6004F5C4631E
:1041E0001D605D609D6004F22C631D605D609D60DC
:1041F00005F020FA194B1A491C60204631F0E2FE06
:1042000051462422584676F045F8C4F84073C4F865
:104210003073C4F8207304F5257207CA04F52873B7
:1042200083E80700484694EDAA1AD4EDA90A94ED54
:10423000A80A16F06FFA3546494668466E4616F0EB
:104240008BF90FCE0FC50FCE0FC533682B602046FC
:104250000BB0BDE8F08F00BFB4260908E859002074
:104260006425090810B5044688B001F0EFF994F907
:104270003232012B02D1274804F072FB022B0AD103
:10428000032384F8323204A9012304F111008DF8CC
:10429000103032F051FC94F8323284F8903204F24B
:1042A0003C4001F089F994F93132642B30D1652317
:1042B00004A904F231208DF8103032F07BFC04A9FF
:1042C000204631F055F918B304238DF81830002337
:1042D000CDE9013303930F230593694604A831F018
:1042E00019FB059B28B108AA02EB8302009942F84A
:1042F000581C0133112B0593EFD951F001FF9DEDAF
:10430000031ADDED020A9DED010A652151F0B6FEAA
:1043100008B010BDC424090870B500F5257600F575
:1043200028758CB004463146284617F0DFFDE0B909
:1043300096E8070085E8070004F52B7194EDAA1AAA
:10434000D4EDA90A94EDA80A0191084616F0E2F905
:1043500002AD019902A816F0FFF80FCD04F53474F0
:104360000FC40FCD0FC42B6823600CB070BD0000CC
:1043700013B540F2411200F50671044601A812F08F
:1043800047FA04F23C4001F0FFFA20461BF0D4FF4C
:1043900001A812F05FFA02B010BD0000F8B50B687A
:1043A000C0F804324B68C0F808328B68C0F80C3291
:1043B00001F10C0607460C4600F548750FCE0FC5F7
:1043C0000FCE0FC533682B6004F1300207CA07F522
:1043D000457383E8070004F13C0207CA07F55173EF
:1043E00083E8070004F1480207CA07F5547383E81D
:1043F0000700543494E8070007F5577383E8070073
:10440000384601F037FA3846BDE8F84001F01ABAEC
:1044100013B5044600F23C40019002F0ABFE04F5F7
:10442000BB610198009102F003FA0099204602B0A6
:10443000BDE81040FFF7B2BF4A78064BC2F3401206
:104440001A754A78C2F380125A750A78C2F30012BC
:104450009A757047755A002013B540F2F52204464C
:1044600000F5067101A812F0D3F9002104F23C40D6
:1044700001F0FCFC94F8603223B120461CF008F9EE
:1044800084F8600201A812F0E5F902B010BD000046
:1044900038B590F80C3305460C462BB1032B0BD0E6
:1044A00095F86832DB070CD405F5C7630FCB84E8B9
:1044B0000F0095F8480603E01BF094FF0028EFD0AA
:1044C00038BD0020FCE7000000F23C4090ED350ACA
:1044D0007047000000F23C4090ED360A7047000043
:1044E00010B490F80C230C462AB1032A0AD00020FD
:1044F0005DF8044B704700F5B26007C884E8070018
:104500000120F5E75DF8044B1BF054BF90F88403DD
:10451000431E58425841704738B590F80C330D4649
:104520008BB900F23C4001F0A1FA044610B9002416
:10453000204638BD01F0EEF9D5ED007A27EE800A6D
:1045400085ED000AF4E7D0EDE07AC1ED007A90F84D
:104550007C43002CEBD090EDDE7ADFED086AB4EE00
:10456000E67AF1EE10FAF7EE006AB8BFB0EE667ABE
:1045700067EE877AC1ED007ADAE700BF0000003409
:1045800090F80C33032B01D11BF094BE0020704730
:1045900090F80C23032A01D11BF0AEBF00F23C407F
:1045A00001F0C6BE30B590F80C3385B004460D4618
:1045B0008BB1032B18D004F5257017F0D1FC2846D9
:1045C00001A98DED010ACDED020A8DED031A17F058
:1045D00021FB012006E000F23C4001F0F1F9002847
:1045E000E9D1002005B030BD90F86032002BF8D042
:1045F0001BF06AFFDFE700007FB590F80C2332B1B3
:10460000032A4FF0000309D0039304930CE000F257
:104610003C4007B05DF804EB01F0ACBA03A903938A
:10462000049305931BF03CFE9DED030ADDED040AA7
:1046300007B05DF804FB000007B590F80C3333B108
:1046400000F57F7003B05DF804EB17F0EFBB00F2EC
:104650003C4001F08FFA68468DED000ACDED010A6D
:1046600017F0E4FB03B05DF804FB000090F80C03C6
:10467000003818BF0120704708B590F80C23032AB2
:1046800005D0BDE8084000F23C4001F05DBA1BF0E7
:1046900007FE012008BD000010B590F80C230C4661
:1046A0001AB1032A07D0002010BDBDE8104000F267
:1046B0003C4001F0EDB91BF009FE012084ED000A39
:1046C000F2E7000030B590F80C3385B005460C4693
:1046D00023B1032B09D0002005B030BD00F23C40CF
:1046E00005B0BDE8304002F0D3B8002302A9029320
:1046F00003931BF0BDFD0028EDD001A928461BF057
:10470000C3FD0028E7D0029B2360039B6360019BED
:10471000A360E1E790F80C231AB1032A05D000202A
:10472000704700F23C4002F0D9B81BF0ADBD00006C
:1047300090F932323BB990F8683213F0010F14BF90
:10474000032000207047032070470000F7B504469F
:10475000FFF7EEFF0546002862D0032839D194F810
:1047600060326BB394F86832D8072BD501A9204684
:104770001CF0B8F8BDF80430002B18BF002594F8E1
:10478000146206F0FD06012E4AD10023032D019389
:1047900007D101A920461CF0B1F820461BF0B8FE55
:1047A000064604F23C4002F025F908B994F80903E2
:1047B0009DF80430D90703D55A0701D59F0632D496
:1047C00000252DE020461BF02DFD002808BF002508
:1047D000D5E70025D3E713F0020F2EE094F9443219
:1047E00023B99DF80430DB092FD0E9E7002EF8D07B
:1047F0000EF004FBFFF7B8FB022807D99DF805303F
:104800009806DDD59DF80430D906D9D5FB6A93F812
:104810009C30002BE5D118E0DA0601D41B0718D52F
:10482000284603B0F0BD0028FAD094F80923B4F963
:104830004C36002ACFD013F0010FF1D1154B1F6871
:10484000FB6A93F89C30002BC8D19DF804309C077C
:10485000E2D405F013FF05F00FFE0028B0D10EF0F2
:10486000CDFAFFF781FB0228AAD90EF0C7FA90F81B
:10487000C432B02202FB030090ED2F7AF0EE007AF2
:10488000B4EEE77AF1EE10FA9AD59DF80530DB091F
:10489000C6D195E7CC2500202DE9F04790F860328D
:1048A00092B00446002B00F0948020461CF026F9BC
:1048B0002046FFF74BFF03287BD104F548780027FB
:1048C000414620460097019702971BF0F3FD694689
:1048D00020461BF0E5FD009BC4F80432019BC4F8A0
:1048E0000832029BC4F80C32204600F0C3FF204679
:1048F00000F0A8FF14F048FE054620461BF0AAFC75
:104900000028A8BFC6B203AA4FF0FF312046BCBFA3
:1049100095F8129395F813630397A8BFB1460497CF
:1049200005971BF0E1FC03A817F01AFB4FF00C0AE7
:104930000AFB095084EDD10AC4EDD20A84EDD31AE2
:1049400004F5517100F5117017F01AFB04F5577753
:104950000AFB065584EDC50AC4EDC60A84EDC71AE4
:104960003A464FF0FF31204605F5C4751BF0D0FCE8
:1049700095E8070006AE86E807003946304617F08E
:1049800065FB04F52B72414609A815F075FD31460B
:1049900009A815F0F3FC09A9204684EDD40AC4ED5A
:1049A000D50A84EDD61A1BF0A9FF09A92046FFF706
:1049B00043FD94F84E36002B3AD109A804F03AFE94
:1049C00009A920461BF01AFD90B3012384F84E3646
:1049D0002EE0D0F864321BB953F06CFCC4F86402CA
:1049E000154B1B68D86A03685B68984788B153F019
:1049F00061FCD4F86432C01AB4F86232984204D927
:104A000020461BF045FE84F8600294F860327BB1CA
:104A10004BE753F04FFCD4F86432C01A41F28733AD
:104A20009842E4D835F0FAFA35F0DEFA0028DED103
:104A300012B0BDE8F08700BFCC25002090F80C3301
:104A400023B1032B4FF0000007D0704790F93222BA
:104A5000032A04D10A70012070470870FBE718464A
:104A60007047000073B50D460DF107010446FFF7CE
:104A7000E5FF064628B19DF807302BB1032B09D07E
:104A80000026304602B070BD04F5C7630FCB85E841
:104A90000F00F6E7294620461BF0A4FC94F860625C
:104AA000EFE700007FB50E460DF103010446FFF766
:104AB000C5FF054618B90025284604B070BD9DF80D
:104AC000033083B1032B16D004F5257017F048FA94
:104AD00001A930468DED010ACDED020A8DED031AD4
:104AE00017F098F8E8E7314604F23C4000F068FF20
:104AF0000028E9D1DFE794F86032002BDBD03146A3
:104B000020461BF0E1FCDFE737B50D460DF107014C
:104B10000446FFF793FF28B19DF8073023B1032B1C
:104B20000FD0002003B030BD04F5BB631B682B60C1
:104B300004F2DC5304F5BC641B686B602368AB6053
:104B4000F0E7204629461BF0ABFC94F86002E9E749
:104B500010B50446FFF7ECFD18B1032807D000207C
:104B600010BD04F23C40BDE8104000F053BF94F883
:104B70006032002BF3D020461BF054FB0028EED00F
:104B800094F8143203F0FD03012BE9D194F80C03DF
:104B9000C31E58425841E3E710B50446FFF7C8FD6D
:104BA00080B1032810D194F8600250B153F082FB19
:104BB000D4F86432C01A44F62063984294BF0020AF
:104BC000012010BD0120FCE70020FAE708B50246ED
:104BD000FFF7AEFD032804D110461BF08FFE012025
:104BE00008BD0020FCE7000030B585B00446019107
:104BF000FFF742F80199054610B9002005B030BD15
:104C00000191FFF70BF801990028F6D02846FFF72D
:104C100009F80028F1D0B4F84C365907EED494F8CE
:104C20000933002BEAD00B4A1268D26A92F89C50E2
:104C30006DB103A92046FFF7C9FF30B19DF80E30D2
:104C40009A07DBD5C3F38000D8E72846D6E7184695
:104C5000D4E700BFCC2500202DE9F04190F80C33BB
:104C60008CB00027032B06460C461546009701978B
:104C7000029719D11BF0EEFA6A4680464FF0FF31D9
:104C800030461BF045FBB8F1FF3FA7606760276027
:104C90000DD114F079FC2B4690F81313224613F033
:104CA00001FD0CB0BDE8F0814FF0FF38EBE714F0E8
:104CB0006BFC2B4622465FFA88F113F0F3FC95ED6E
:104CC000000A684617F088F903A920468DED051AF9
:104CD0008DED030ACDED040A17F0B8F906F52B7235
:104CE00006F5487103A815F0C7FB214603A815F087
:104CF00045FB84ED021A84ED000AC4ED010A95ED2E
:104D0000007ADFED037AA7EE271A84ED021AC8E7CE
:104D10000AE81C4137B5054600F5067140F6033236
:104D200001A811F075FD2846FFF702FD044640B1C9
:104D300003280AD0002401A811F08CFD204603B0FE
:104D400030BD28461BF012FBF5E728461BF00EFB92
:104D50000446F0E708B50246FFF7EAFC10B1032865
:104D600006D008BDBDE8084002F23C4000F01CBE81
:104D7000BDE8084010461BF0CDBD00000B4610B446
:104D800011462BB1032B09D000205DF8044B70476E
:104D90005DF8044B00F23C4000F01CBE5DF8044B93
:104DA0001BF02CBB13B50446FFF7C2FC0A460146B4
:104DB00020460192FFF7E2FF70B9084B019A1B6889
:104DC000DB6A93F89C0038B194F80C13204602B0CB
:104DD000BDE81040FFF7D2BF02B010BDCC250020C7
:104DE00037B504460D4640F2B25200F5067101A8EF
:104DF00011F00EFD294620461BF01EFB94F80C33E3
:104E0000032B054610D148B104F583612046FFF716
:104E1000C9FF84F82804204600F05CFD01A811F0C9
:104E200019FD284603B030BD0025F7E770B590F8AE
:104E30007C32DB0786B004460D460CD402F044FFFA
:104E4000437C242202FB0300D0ED0B7AF1EE677A5B
:104E5000C5ED007A3BE002A804F0ECFB01A9204676
:104E6000FFF758FCE8B90DF0C9FF94F94432022B62
:104E70000646E3D1FFF778F80228DFD996F8C40296
:104E80009FED147AB02303FB0066D4F87032D6F895
:104E9000B0209B1A07EE903AF8EEE77A67EE877A31
:104EA000D6E702A92046FFF77DFF0028DBD0D4F823
:104EB0007022039BDFED076A9DED017A9B1A07EED6
:104EC000903AF8EEE77AA7EEE67A85ED007A06B03A
:104ED00070BD00BF0AD7233CF0B50C4687B000F583
:104EE0000671064640F6863201A811F091FCA368CF
:104EF00053B9E36843B9636833B9002701A811F0D7
:104F0000A9FC384607B0F0BD204604F069FC002833
:104F1000F3D094E80F0002AD85E80F000021284689
:104F200004F020FC07460028E7D096F87C32DB0727
:104F300004D435F073F8192134F0ACFF95E80F0074
:104F400006F51B7C8CE80F0096F87C3243F00103D9
:104F500086F87C32304600F0BDFC3DF0B1FD4621C4
:104F60003EF0A8F93DF0ACFD45213EF0A3F9054B1C
:104F7000A2681B68DB6A1A61E2685A6162689A611A
:104F8000BCE700BFCC25002038B5144B1B68DD6A98
:104F90002B6804465B6828469847F0B12B690BB92B
:104FA0006A69D2B1C4F874326B69C4F87832A969FD
:104FB000002204F51B7004F043FB94F87C3223F0CC
:104FC000030343F0030384F87C323DF079FDBDE830
:104FD0003840034A062136F0A3BF38BDCC25002057
:104FE000EC24090810B588B004460593FFF7A0FB30
:104FF0000328059B4FF000000AD10690079006A8F1
:1050000002900B9801900A98009020461BF066FAD7
:1050100008B010BD38B50446FEF72EFE0546D0B1E7
:1050200094F80C33032B03D095F84E41204638BD3D
:1050300020461BF0CBF9FF280446F5D00146284650
:10504000FEF7F0FD0028EFD021462846FEF7E6FDEA
:105050000028E9D0EAE70446E8E7000008B590F840
:105060000C33032B05D014F08FFA90F91203C0B261
:1050700008BD1BF0EFF8431CF9D1F4E708B590F830
:105080000C3383B1032B03D1BDE808401BF0DAB821
:1050900033F098FB40F6ED424FF4801133F04AFBB9
:1050A0004FF0FF3008BD1846FCE7000090F80C33C5
:1050B000032B01D11BF06EBE7047000090F80C333B
:1050C000032B01D11BF00CB8704700001BF092B805
:1050D00010B504461DF0A0FE2046FEF7D5FD204683
:1050E000BDE81040FEF7D6BE90F80C330BB1032B91
:1050F00001D11BF0CBBE00207047000030B500F599
:10510000757304460D460FCB85E80F0094F8E40351
:1051100030BD0000D0F880330B6090F87C037047FE
:10512000D0F888330B6090F88503704730B500F5F0
:10513000677304460D460FCB85E80F0094F8AC0367
:1051400030BD000030B500F5836304460D460FCB3B
:1051500085E80F0094F8280430BD000010B500F277
:105160002C4203460C4607CA84E8070093F838042B
:1051700010BD00002DE9F0432DED028B8BB00546EC
:105180000E461746FFF746FF014680462846FFF7C2
:105190002BFD0446002848D0FEF76EFD4146FEF781
:1051A00043FD86ED000A95F93032002B3ADD0DF013
:1051B00025FEFEF7D9FE012834D90DF01FFE90F828
:1051C000C432D5EDDE7ADFED5D8A96ED000AB022BD
:1051D00002FB030095F93032D0ED2F0A07EE103AAA
:1051E000F4EEE87AB8EEC77AF1EE10FAB7EE008A7C
:1051F000B8BFF0EE487A37EE201A20EE270A70EE9C
:10520000C70A40F2B63014F0C1FED5EDDE7AF4EEF6
:10521000E87AF1EE10FAB8BFF0EE487A80EE277A1D
:1052200086ED007A01233B7003E095F8083333B92B
:10523000387020460BB0BDEC028BBDE8F08395F8CA
:105240000C334FF00009CDF80490CDF80890CDF85C
:105250000C9043B1032B10D0CDF81090CDF81490E2
:10526000CDF818907CB902233B703246414605F2D6
:105270003C4001F083FB0446DBE701A928461BF014
:1052800099F80446E8E795F80C33002BEBD004A915
:105290002846FFF763FF04460028E4D001A904A8CC
:1052A00016F084FE07A8CDED080A8DED091A8DEDE4
:1052B000070A17F08FFA04A8B0EE408A17F08AFAAE
:1052C00095F93032002B30DD07EE903AF8EEE77AB0
:1052D0004FF47F7070EE670A37EE801AF5EEC00A61
:1052E000F1EE10FA48BFDFED160AF4EE410AF1EED6
:1052F00010FAB0EE480AC8BFB0EE601A14F046FECD
:10530000B0EE408AD5EDDE7A9FED0C7AF4EEC77AE6
:10531000F1EE10FAB7EE007AB8BFF0EE477A88EEF9
:10532000277A032386ED007A7DE7B5EEC08AF1EE99
:1053300010FA48BF9FED028AE4E700BF0000003486
:105340000000000010B50446FFF788FE84F80D0346
:105350002046FFF783FE84F80E032046FFF77EFE0B
:1053600084F80F032046FFF789FE04F55A7184F88C
:1053700010032046FFF7B4F884F8740300F0CAFA6B
:1053800004F5617284EDDE0A04F560712046FFF7D2
:10539000F1FE04F5627184F87C032046FFF7BCF847
:1053A00004F5637184F885032046FFF7E9F804F5F6
:1053B000677184F898032046FFF7F4F804F56C71E0
:1053C00084F8AC032046FFF79FFB04F5707184F866
:1053D000BC032046FFF766FB04F5757184F8D00323
:1053E0002046FFF755F804F57A7184F8E403204667
:1053F000FFF738FB84F8F8032046FFF7FDF804F5C3
:10540000806384EDFF0A2046C3ED000AFFF714F91C
:1054100004F2044383ED000A04F2144204F58161AE
:105420002046FFF719FC04F583612046FFF7BAFC1C
:1054300004F22C4184F828042046FFF71DF984F873
:10544000380410BD37B50D46044600F0FFF81DB90D
:1054500014F09AF813F056F84FF4BE7204F5067182
:1054600001A811F0D5F994F869322BB92046FFF75D
:105470008BFD012384F86932224B1D68A86A0368FA
:105480009B6998472046FEF747FF2046FEF7C0FF7E
:10549000204600F051FA2046FFF7FEF9286B30B1A4
:1054A0000368D4EDD20ADB6894EDD10A9847D4F8AA
:1054B000100208B153F06CFE204600F07DF8204643
:1054C000FFF744F994F8903284F80C0383420ED02D
:1054D00084F8900298B10C4D0C4B032808BF1D4670
:1054E0003DF0EEFA0A4A2B46062136F019FD204619
:1054F000FFF728FF01A811F0ADF903B030BD054D4D
:10550000EEE700BFCC2500202FF80808E3240908A7
:1055100004250908E8240908D0EDDE7A9FED057A14
:10552000F4EEC77AF1EE10FAB7EE000AA8BFB0EEBB
:10553000670A704700000034014B1868704700BFCD
:10554000E85900204FF0FF307047000001207047FD
:10555000704700000020704700207047704700002F
:1055600070470000002070470020704700207047FF
:1055700000207047002070470020704700207047CF
:10558000012070470368D3F8943018470020704713
:1055900000207047002070470020704700207047AF
:1055A000002070470020704700207047002070479F
:1055B00000207047704700007047000008B513F0E6
:1055C000E3FF90F8130308BD08B513F0DDFF90F872
:1055D000120308BD30B52DED028B9FED1A1ADFEDD9
:1055E0001A0A91ED000A87B005462D200C468DED74
:1055F000011ACDED000A14F0C9FC9DED011ADDED94
:10560000000AF0EE408A2E2094ED010A14F0BEFC50
:105610009DED011ADDED000AB0EE408A2F2094EDD9
:10562000020A14F0B3FC03A905F52570CDED038A39
:105630008DED048A8DED050A31F0A0FB07B0BDECBD
:10564000028B30BDC2B8323EC2B832BE10B504467D
:1056500052F030FED4F8F4321BB1C21AB2F57A7FA0
:1056600012D30A4A1268D26A92F89C2002B15BB93E
:10567000C4F8F40294F8314213F086FF80F80D4329
:1056800004F0FCFF80F8254010BD00BFCC250020B1
:105690002DE9F0432DED028B91ED007AD1ED037AE7
:1056A00087B08DED047AB0EEC77AB5EEC07AF1EE30
:1056B00010FADDE91087DDF84C90CDED057A0C4647
:1056C00015461E4606DCF0EEE77AF5EEC07AF1EEFE
:1056D00010FA02DD04A816F0FBFB6B20B7EE001AEF
:1056E000FFEE000A9DED050A14F050FC6C2089EDD8
:1056F000000AB7EE001AFFEE000A9DED040A14F04E
:1057000045FC04A888ED000A16F06AFBB7EE008A93
:10571000002852D00023C9F8003088ED008AD4ED6B
:10572000067A67EEA77AF4EEC87AF1EE10FA4ADB51
:105730000023336085ED008ADFED3F0A96ED000A15
:105740007C20B7EE001A14F021FC86ED000A95EDDE
:10575000000A7D20B7EE001AFFEE000A14F016FCD6
:1057600085ED000AD4ED067A129BDFED346AF1EE86
:10577000677AC3ED007A96ED007AF0EEC77AF4EE20
:10578000E67AF1EE10FA2BD503AB02AA01A9204666
:1057900015F020F89DED018AB0EE480A72F072F91A
:1057A00085ED000AB0EE480A72F0C2FA87ED000AF1
:1057B00007B0BDEC028BBDE8F08304A816F0FCFA3C
:1057C0000028A7D1ABE738EE670A14F011FB86ED8D
:1057D000000A94ED087AC7EE007AC5ED007AABE7CF
:1057E00094ED076AC6EE077AC7ED007A96ED007A67
:1057F000B0EEC77AB4EEE67AF1EE10FAC4D495EDC5
:10580000007ADFED0F6AB0EEC76AB4EE666AF1EEB9
:1058100010FAB9DCB4EE477AF1EE10FAB4D6B0EE75
:10582000E77AB4EE667AF1EE10FAADDCF4EE677A60
:10583000F1EE10FABCD7A7E700000000000000342A
:10584000FFFF7F7F1FB500F51773039300F51673F5
:10585000029300F51573019300F51473009300F59E
:10586000127200F5137300F54871FFF711FF05B0D0
:105870005DF804FB9FED156A90ED817ADFED146A07
:10588000D0ED837A27EE067A67EE867A27EE267ABF
:1058900067EEA67ABDEEC77AFDEEE77A80ED7E7AF6
:1058A00090ED827A27EE067A17EE903A27EE267A66
:1058B000002BB8BF03F50C43BDEEC77AB8BFA033C9
:1058C00080ED7F7AC0F80032704700BFE02E65425D
:1058D0000000C8421FB50E4B1B680446B3B16846B2
:1058E00003F0A8FE69462046FFF72CFC20B16A466B
:1058F00000212046FEF7A6FA94F87C32DB0705D596
:1059000004F51B7201212046FEF79CFA04B010BD7D
:10591000945C002008B502F0D7F9BDE8084001F01A
:105920006FBD000010B580F8F812044652F0C2FCBA
:10593000C4F8FC0210BD000010B590F8F83204461F
:1059400053B152F0B7FCD4F8FC32C01AB0F57A7FEC
:1059500084BF002384F8F83294F8003353B152F036
:10596000A9FCD4F80433C01AB0F57A7F84BF0023B1
:1059700084F8003310BD000000F5AA700B4607C87C
:1059800083E80700012070470023C0F89C30C0F86E
:105990009830C0F89430C0F8A830C0F8A430C0F8EF
:1059A000A030C0F8AC30704770470000024B0B606D
:1059B0004FF07C531360704700004842704700006E
:1059C00008B50B4600F12801184615F06DFD0120C1
:1059D00008BD000010B500F5B4700C460FC884E88F
:1059E0000F00204603F016FE30B1FFF7A5FD00F5CD
:1059F0001B700FC884E80F00204603F00BFE80F0F8
:105A00000100C0B210BD000010B5044604F0B6F8A5
:105A1000204610BD10B5D0F8603104465BB152F09D
:105A200049FCD4F86031C01A41F28833984294BFDF
:105A30000020012010BD0120FCE7000013B50093F9
:105A400003680192D3F890309847DDE900210446BD
:105A500028B90448044B0068C06A11F0B9F8204620
:105A600002B010BDCC2500202426090813B5044639
:105A70000191FEF701F92368019A1B6D014608B1F7
:105A800090F84E11204602B0BDE8104018470000C3
:105A900030B585B0002301930293039303680D464C
:105AA000DB6D01A99847044620B1039B2B6020467B
:105AB00005B030BD02F008F9417C01F0DDFD04467F
:105AC0000028F4D002F000F901F03CFDB1EE400AEC
:105AD00085ED000AEBE7000090ED007ADFED0F7A2C
:105AE000B0EEC77AB4EEE77AF1EE10FA14D590ED85
:105AF000017AB0EEC77AB4EEE77AF1EE10FA0BD580
:105B000090ED027AB0EEC77AB4EEE77AF1EE10FAD1
:105B10004CBF012000207047002070470000003477
:105B200010B5FEF7A9F8044658B190F84E11FEF7EB
:105B300075F830B194F84E112046BDE81040FEF7DC
:105B400071B8002010BD000038B50D460DF056F9B3
:105B50000446FEF709FA022881BF94F8C402B02374
:105B600003FB0040D43089BF07C8002085E8070048
:105B7000012038BD2DE9F0432DED028B8FB0036875
:105B80000025DB6C0395049505950695029502A901
:105B900004469847064638B1FFF7BCFEDDED027AB1
:105BA00027EE800A8DED020A0DF028F9FEF7DCF9E8
:105BB0000746002E50D0DDED027AD4ED646A94EDF4
:105BC000657A23680B9527EE877A67EEA67A8DEDC6
:105BD000097ACDED0A7A0C950D959B6C0BA92046A0
:105BE00009AD98470BA9284616F070F8012F8DEDE6
:105BF000030ACDED040A40F2B3800DF0FFF890F8EF
:105C0000C432DFED5B7AB02505FB030090ED308AEE
:105C100028EE278AB0EE480A71F034FFF0EE408A91
:105C2000B0EE480A72F084F8CDED0B8A8DED0C0AC7
:105C30000DF0E4F890F8C43205FB030090ED2F0A54
:105C40000BA816F063F809AD8DED050ACDED060A37
:105C500005A896BB03C885E00128CED89DED020AB1
:105C6000B5EEC00AF1EE10FA7FDD07AED4F894214C
:105C7000D4F8903107923046089316F065F82368FF
:105C80000B950C950D959B6C0BA920469847DDED67
:105C9000077A9DED0B7A77EE877A9DED0C7ACDED44
:105CA000077ADDED087A77EE877A09ABCDED087AD1
:105CB00096E8030083E8030049E0236993ED000AB6
:105CC000B7EE008A38EE408A16F020F804F5BC7969
:105CD0008DED090A4846B0EE480ACDED0A0A16F0E5
:105CE00015F80BA92846CDED0C0A8DED0B0A15F021
:105CF000EDFF04F5C47603AFC4ED5F0A314684EDD1
:105D00005E0A384615F0F2FF04F5C0788DED090AF9
:105D10004046B0EE480ACDED0A0A15F0F7FF0BA990
:105D200028468DED0B0ACDED0C0A15F0CFFF97E854
:105D3000030084ED600AC4ED610A86E80300494669
:105D4000404615F0C3FF8DED090ACDED0A0A9DED21
:105D5000090ADDED0A0A0FB0BDEC028BBDE8F08345
:105D6000DDE9030185E80300F1E709950A95EEE70F
:105D700035FA8E3C10B590F84213044604F098F8BA
:105D80007C23C0B203FB0044D4F8A00010BD000087
:105D9000044B026F1B68DB6A5A60426F9A60826F25
:105DA000DA607047CC250020F0B58FB0044613F0C0
:105DB000EBFB002302930393049390F8121301ABBF
:105DC00002AA054612F014FC04F19407D8B39DED25
:105DD000010AB5EEC00AF1EE10FA34DD02A816F0A1
:105DE0000BF904F1B00684ED2C0AC4ED2D0A84ED04
:105DF0002E1A3946304616F00FF904F17C01304670
:105E000016F0BEF804F1880105A88DED050ACDED68
:105E1000060A8DED071A16F0B3F808A88DED080AEA
:105E20009DED010ACDED090A8DED0A1A16F0D4F8A0
:105E30000BA904F128008DED0B0ACDED0C0A8DEDB8
:105E40000D1A14F073FD95F812030C2303FB005098
:105E5000394600F5117016F093F884ED2C0AC4ED64
:105E60002D0A84ED2E1A0FB0F0BD00002DE9F04789
:105E7000824B00251F682DED028BC0F89C50C0F8A6
:105E80009850C0F89450C0F88450C0F88050C5674E
:105E9000C0F89050C0F88C50C0F88850C0F8B85086
:105EA000C0F8B450C0F8B0500446F86A03688AB02D
:105EB0005B680E46984704F12809002854D052F038
:105EC000F9F942F20F7398424ED8FB6A9FED6C8A43
:105ED00093ED010A84ED1C0AD3ED020AC4ED1D0AFC
:105EE00093ED031A484684ED1E1A14F013FC3CF09F
:105EF000E7FDD4ED1E7A67EE887A054617EE900A24
:105F0000FAF7FAFAD4ED1D7A67EE887ACDE9040142
:105F100017EE900AFAF7F0FAD4ED1C7A67EE887A59
:105F2000CDE9020117EE900AFAF7E6FA554ACDE9F3
:105F300000010621284635F0F3FF94ED1E8AB0EEED
:105F4000480A71F09FFD84ED650AB0EE480A71F0D1
:105F5000EFFE84ED640A52F0ADF9C4F864010AB0B2
:105F6000BDEC028BBDE8F087A6B194ED1C0AB4EE3F
:105F7000400AF1EE10FA0DD6D4ED1D0AF4EE600AD7
:105F8000F1EE10FA06D694ED1E1AB4EE411AF1EEB7
:105F900010FA52D713F0F8FA90F813334FF00C0AB6
:105FA0000AFB030303F5C473074693E8070007AE33
:105FB00086E807004FF01508B2EE028AF2EE068A74
:105FC000304616F007FCB4EEC80AF1EE10FA38D5E8
:105FD00008F1FF3818F0FF083CD1304616F0FAFB04
:105FE000F1EE047AB4EEE70AF1EE10FA43DD9DED2E
:105FF000090ADDED087A9DED078A20EE000AA7EE7A
:10600000A70A72F0ABF8F0EE400AB0EE480A71F061
:106010005BFFDDED090A84ED1D0A9DED080AF1EE36
:10602000600AB1EE400A71F04FFF84ED1C0A9FED4B
:10603000161AD4ED1D0A94ED1C0A484614F06AFBAA
:106040007BE7304616F0C6FBB4EEE80AF1EE10FA34
:10605000BEDCC2E7384612F08DF9384612F052FA2B
:1060600097F813330AFB037303F5C47393E807002F
:1060700086E80700A4E725676567D8E7CC250020F8
:10608000E02E654230260908000000000021FFF7DD
:10609000EDBE000037B5044608461546019116F0DE
:1060A00099FBB7EE007AC7EE007AB4F8D0300198C9
:1060B0000133A4F8D03094ED337A37EE277A84EDAB
:1060C000337AB0EE007AF4EEC77AF1EE10FA06D524
:1060D000B6EE007AF4EEC77AF1EE10FA0DDC9FED21
:1060E0000E7AF4EEC77AF1EE10FA13D59FED0B7A23
:1060F000F4EEC77AF1EE10FA0CDDB0EE670A15F097
:106100006BFF012085ED000AC5ED010A85ED021A3D
:1061100003B030BD0020FBE700247449BD3786354D
:1061200070B52DED028B00F1280600F134058AB020
:1061300029460446304615F0CBFFB6EE008A20EE25
:10614000088A2846B0EE480A15F046FF07A93046EF
:10615000CDED080A8DED091A8DED070A15F026FF21
:1061600030468DED010AB0EE480ACDED020A8DED04
:10617000031A15F031FF07A928468DED070ACDED6A
:10618000080A8DED091A15F011FF04A901A88DED7B
:10619000040ACDED050A8DED061A15F0ADFF324665
:1061A00001A920468DED070ACDED080A8DED091AEB
:1061B000FFF770FF58B952F07DF80121C4F8600173
:1061C0002046FFF753FE0AB0BDEC028B70BD2A4695
:1061D00004A92046FFF75EFF0028ECD004F140023E
:1061E00007A92046FFF756FF0028E4D0EBE70000A0
:1061F00030B52DED028B0D4683B091F84213044665
:10620000284603F055FEC1B27C2000FB01519031BD
:1062100004F1280014F00EF968468DED000ACDED6A
:10622000010A15F003FEDFED1C7AB4EEE70AF1EE89
:1062300010FA05D59FED190A03B0BDEC028B30BDF5
:10624000684615F045FE684615F0CAFD0028F1D1F4
:10625000284694ED428A03F09FFFF0EE400AB0EE2C
:10626000480A13F091FD80B9284603F095FF84EDAC
:10627000420AB0EE408A71F005FC84ED430AB0EEAC
:10628000480A71F055FD84ED440A04F586716846AC
:1062900015F084FDD0E700BF0000003400000000CE
:1062A0009FED0C7AB4EEC70AF1EE10FA0BD4DFEDD5
:1062B0000A7AB4EEE70AF1EE10FA07DCC0EE077ACC
:1062C000B0EE670A7047F7EE007AF9E7F2EE047A6B
:1062D000F6E700BFF3665F3F58A00B4108B51C30DE
:1062E00015F0A4FDF1EE007AB4EEE70AF1EE10FA33
:1062F0009DBFF1EE027A37EEC00ADFED047A9FED22
:10630000040A98BF20EE270A08BD00BFCDCC4C3E42
:10631000CDCCCC3D08B5836993F9000038B10CF0C1
:106320006DFDFDF721FE012894BF0020012008BD6E
:10633000F8B52DED028B054604F0A0F904F09CF8A9
:106340000446B8B3FFF7F8F890F8093393B328463A
:10635000FFF7E0FF064668B30CF050FD90F8C4323A
:10636000B02707FB030090ED2F7AF0EE087AB4EE29
:10637000E77AF1EE10FA1DD495ED1E8A0CF03EFD81
:1063800090F8C432DFED1E7A07FB030090ED300A6F
:1063900098EE270A13F07CFDDFED1A7AB0EEC00A02
:1063A000B4EEE70AF1EE10FA08DC51F083FF344650
:1063B000C5F85001BDEC028B2046F8BD05F5AA706A
:1063C00016F008FAB0EE408A0CF018FD90F8C432CE
:1063D0009FED0D7A07FB0303D3ED2F7A67EE877AE3
:1063E000B4EEE78AF1EE10FADFD551F063FFD5F88D
:1063F0005041001BB0F5FA6F8CBF00240124D9E78F
:10640000E02E654200003442CDCC4C3F10B50A4B23
:106410001B68DB6A93F89C3004465BB951F04AFF75
:10642000D4F86431C01A44F61F6398428CBF002030
:10643000012010BD0020FCE7CC250020F8B52DED93
:10644000068B04460CF0DAFC054604F017F9064604
:1064500006F000FE002840F0AA802046FFF768FF03
:10646000002800F0A7803046FFF784FCD4F8DC3029
:10647000984200F018813046FFF77CFCD4F8DC30FD
:10648000DFED8E7AC31A08EE903AF8EE688A30464D
:1064900068EEA78AFFF76EFC94F8BC30C4F8DC0005
:1064A000F3B9304603F0FAFFD0B104F1280796F8AB
:1064B00042233946304603F073FED4ED1D0AB0EE98
:1064C000401A384694ED1C0A14F024F90023C4F84D
:1064D0009030C4F88C30C4F88830012384F8BC3084
:1064E00020463146FFF784FE95F8C40205EB0015FF
:1064F000B0EE408A2B6FC4F8E03004F1B000D4ED68
:10650000129A16F067F96368DFED6D7A93ED007A01
:10651000B4EEE77AF1EE10FA68EE299AB0EE40AAEE
:1065200001D5C3ED007A2046B0EE4A0AFFF7B8FE67
:10653000636820EE299A93ED000A29EE009AFFF78E
:10654000CDFE29EE009A204684ED249AFFF75EFFE7
:1065500038B1D4ED247AB2EE007A67EE877AC4EDD2
:10656000247AF0EE007AF4EEE78AF1EE10FA10D514
:10657000DFED547AB4EEE7AAF1EE10FA09D5DFEDBB
:10658000527A69EEA79AD4ED2A7AE9EEA87AC4ED98
:106590002A7A9FED4E0A94ED367ADFED4D7AB0EE11
:1065A000C88A28EE008AA7EE278A84ED368ABDECD9
:1065B000068BF8BDFEF7C0FF90F80933002B72D0B0
:1065C0002046FFF7A7FE00286DD095F8C42205EB02
:1065D0000213196FD4F8E0308B4264D0B02606FB6A
:1065E000025292ED2F7AF0EE087AB4EEE77AF1EEED
:1065F00010FA58DBCB1AC4F8E01008EE903A95F880
:10660000C4329FED341A94ED1E0ADFED337A06FB97
:106610000353D3ED309A69EE819AF8EE688A39EE29
:10662000C00A68EEA78A13F09DFCB0EE409A71F0A4
:106630007FFB94F8BC30B0EE408AF3B1F3EE047AFD
:10664000F4EEE78AF1EE10FA17DC95F8C40206FBC7
:10665000005595ED2F7AF2EE027AB4EEE77AF1EE7C
:1066600010FAFFF64AAFDFED1D7AB0EEC99AB4EE2C
:10667000E79AF1EE10FAFFF640AF9FED198AD4EDDC
:106680001D0A94ED1C0AB0EE691A04F1280014F0FA
:1066900041F8012384ED248A84ED238A84ED228A43
:1066A00084F8BC3029E7BDEC068B04F188009FED2F
:1066B0000D0ABDE8F84015F0E3BC00BFBD378635D4
:1066C000CDCC4C3DC2B8B23E0AD7233CCDCC4C3EDB
:1066D000CDCC4C3F35FA8E3C6F12833A1904863F7D
:1066E00000000000EC51783F30B50C2303FB0101A2
:1066F00001F1C003144693E807008BB004AD85E8B0
:10670000070094E8070083E807002846FFF7E4F94C
:1067100007AB58B194E8070083E807009DED070A2E
:10672000DDED080A9DED091A0BB030BD95E80700B4
:10673000F2E70000F0B52DED028BD0F818318B6038
:10674000D0F81C31CB6085B004460D4601F0BCFA90
:1067500006460CF053FBA36993F90030022B074661
:106760004BD1FDF701FC022847D997F8C432B0227B
:1067700002FB0373D3F8B0100022284602F060FF3A
:10678000D4ED4A0A94ED490A284603F0E3F994F857
:106790002C3163B351F08EFD9FED228A97F8C4121D
:1067A0008DED018A01AA064638460BF0ABFBD4F802
:1067B00020019FED1D0A361A07EE906AF8EE677AFF
:1067C0004FF4876027EE800AB6EE001AF0EE480A12
:1067D00013F0DCFBDDED017A30EE270A04F1F00066
:1067E0008DED010A15F092FA284603F0B3F994F8FA
:1067F0002C0105B0BDEC028BF0BD707C242303FBA3
:10680000006696ED0B8AFEF797FED0ED9C7A9FED21
:10681000077AF8EEE77AE8EE077AFDEEE77A17EE08
:10682000901AA9E7000000006F12833A0000C842E6
:10683000F8B5036F0B60436F4B60836F8B6000F1A3
:106840004C050E46074601F10C040FCD0FC40FCDC9
:106850000FC42B68236007F1B00207CA06F13003AA
:1068600083E8070007F1940207CA06F13C0383E8B6
:10687000070007F11C0207CA06F1480383E8070076
:1068800006F160013846FFF755FF86F87000F8BD45
:1068900030B589B0044668460D4602F0CBFE694625
:1068A0002046FFF797F818B90024204609B030BDFC
:1068B00004A802F0BFFE204604A9FFF73BFF0446F0
:1068C0000028F1D004A9684603F09CF885ED000A81
:1068D000C5ED010A85ED021AE7E700001FB50023A8
:1068E0000C4601A9019302930393FFF7D1FF08B16E
:1068F000039B236004B010BD30B585B001AD00230B
:106900000C462946019302930393FFF7C1FF034608
:1069100018B195E8030084E80300184605B030BDBF
:10692000F8B506460F461546FDF7A6F9044690B1A0
:106930003946FDF773F970B120463946FDF772F913
:10694000044640B1FDF798F93946FDF76DF985ED3C
:10695000000A2046F8BDFEF7EFFD90F8083343B17A
:106960003046FFF7D7FC044618B1D6F84C312B60FF
:10697000EFE7D6F84C312B600024EAE770B52DED37
:10698000048B1646FFF7CCFF054670B3FEF7D4FD27
:1069900090F930424CB30CF031FAFDF7E5FA0128DA
:1069A00023D9E4B207EE904AB8EE678A0CF026FAD3
:1069B00090F8C43296ED009AB02202FB0300D0EDAD
:1069C0002F8AFEF7A7FF38EE281A78EEC80A40F2A1
:1069D000614029EE000A13F0D9FAB0EE408AFEF7C2
:1069E00099FFC8EE007AC6ED007ABDEC048B28460C
:1069F00070BD000008B503F041FEBDE8084003F09B
:106A00003BBD000010B5044615F092FB50B904F1EF
:106A10000C0015F08DFB28B904F11800BDE81040FA
:106A200015F086BB012010BD38B500F128050446DD
:106A30002846FFF7E7FF28B120460121BDE838408E
:106A4000FFF714BAD4ED107AB7EE007AF4EEC77AF5
:106A5000F1EE10FA06D5BFEE007AF4EEC77AF1EE49
:106A600010FA12DC2046FFF75BFB2846FFF7CAFF4F
:106A70000028E1D1D4ED107AB2EE047AF0EEE77A94
:106A8000F4EEC77AF1EE10FAD6DC38BD10B5044644
:106A900015F0A0FE2046BDE8104015F005BB000033
:106AA0002DE9F04F2DED048B9FEDC48A95B004467F
:106AB000F0EE408A8DED028A8DED038A8DED048A19
:106AC000FFF7BCFC12F060FD0023054695F8792124
:106AD000012AA8BF012293423FD20021284611F08B
:106AE000B5FB01230028F1D008AB0BAA00212846F2
:106AF0008DED0B8A8DED0C8A8DED0D8A11F0D2FD96
:106B00009DED080AB5EEC00AF1EE10FA23DD0BA8E0
:106B100015F072FA11A904F128008DED110ACDEDDE
:106B2000120A8DED131A13F029FC0EA88DED0E0A32
:106B3000B0EE680ACDED0F0A8DED101A15F04CFA83
:106B400011A904F1E4008DED110ACDED120A8DEDCD
:106B5000131A15F061FA0123B8E795F813130C2303
:106B600003FB015104F1280B01F5C471584613F0E1
:106B700005FC84ED070A94ED3F0AC4ED080A70EEA7
:106B8000288A84ED091AC4ED3F8A0CF037F90646CD
:106B9000FEF7D2FC90F8093300932046FFF7BAFBCA
:106BA00080B13046FDF7E0F902280BD996F8C422EF
:106BB0006169B02303FB026391F9001093F8D200DE
:106BC00088425FDA94ED3F7ADFED7D7AB4EEE77AC2
:106BD000F1EE10FA5DD4D4ED538AFEF7A1FF38B17F
:106BE000FDF74AF890F84E11FDF71EF8F0EE408AD6
:106BF000236C626BA16A1393B0EE680A11A812921B
:106C0000119115F0E9F904F5AA7102A88DED020AB7
:106C1000CDED030A8DED041A15F0FEF951F04AFB93
:106C20000023074684F814312046FFF773FB002841
:106C300065D096F8C422B02302FB03323244526876
:106C4000C4F8182196F8C42202FB033333449B682E
:106C5000C4F81C3151F02EFB0123C4F8200184ED4F
:106C6000498A84ED4A8A84F82C31D4F80031002B0B
:106C700058D102AB93E80700C4F80071F03484E8FF
:106C8000070006E006EB0212176FD4F80021BA42A3
:106C900004D115B0BDEC048BBDE8F08FD43393E87C
:106CA000070094F814310DF1080C8CE807001BB9AB
:106CB00004F1F00383E807000123604684F81431EF
:106CC00004F5AA7115F072F911A904F14C008DEDCB
:106CD000110ACDED120A8DED131A13F07DFBB5EEFE
:106CE000C00AF1EE10FA8DED110AD8BF9FED330AFC
:106CF000CDED120A8DED131A84ED530A94E794ED4D
:106D00003F7AD4ED497ADDED026AE6EE877ADDED71
:106D1000036AC4ED497AD4ED4A7AE7EE267AC4EDE7
:106D20004A7AA2E7D4ED3F7A224B8DED058AF5EE43
:106D3000C07AF1EE10FA8DED068A0793A9D99FED7E
:106D40001E7A94F8143167EE877AB7EE007AC7EEB0
:106D5000279A1BB9009B002B00F0AA80E36804F17E
:106D6000F00102A8D3ED008A15F020F969EEA88A97
:106D70008DED110A11A8B0EE680ACDED120A8DED65
:106D8000131A15F029F90EA905A88DED0E0ACDEDFF
:106D90000F0A8DED101A15F03FF905A8FFF776FEE2
:106DA00005A815F0DFF9D8B151F084FAC4F86001F4
:106DB0006FE700BF000080BF0AE81C410000000030
:106DC000CDCC4C3ECDCC4C3FCDCC4C3D920A06BFF9
:106DD000920A063FC2B8B23E728A0E3C5B821839F4
:106DE000012301930023CDE90833CDE90A33CDE92E
:106DF0000C335FED0E8A4FF0FF3A04F1E40895F88A
:106E00007921012A1046A8BF0120834257D20123CD
:106E1000002AFAD095F835130029F6D0B0EE690AA9
:106E2000404615F02DF9019B0DF12C09002B41D0A6
:106E3000424600212046FFF757FC8DED0B0ACDEDB1
:106E40000C0A8DED0D1A4846FEF746FE70BB48460B
:106E5000FFF71CFE484615F085F938BB05A94846E2
:106E600015F04AF9484605A98DED080ACDED090A45
:106E70008DED0A1A15F02CF908A8B0EE409A15F01D
:106E8000A9FCBAF1000F06D1F4EEC08AF1EE10FAB7
:106E9000D8BFB0EE680AB5EEC09AF1EE10FAF7EE80
:106EA000008A58BFF0EE408A4FF0000A0123A6E79F
:106EB000009B96E798E8070089E80700C3E7BAF166
:106EC000000F7FF471AF002384F804312046FFF7F0
:106ED0002FFA38B12046FFF71DFA002840F025812F
:106EE0008DED0A8A95F8123395F878219A4240F28E
:106EF00033812B4493F83433002B00F02D8195F827
:106F0000133395F879219A4240F226812B4493F865
:106F10003533002B00F0208108A9584613F05CFAA5
:106F20008DED080ACDED090A8DED0A1A08A815F0B5
:106F3000FFF8002840F0178108A815F013F9002881
:106F400040F011815FED627A94ED357A68EEA78AA0
:106F50005FED647AE7EE278A04F1B000C4ED358A6C
:106F600015F038FCA3685FED687A93ED007AB4EE13
:106F7000E77AF1EE10FAF0EE408A00F1F880204650
:106F8000B0EE680AFFF78CF908A815F025F8A36899
:106F90008DED110ACDED120A8DED131A93ED000A55
:106FA00011A815F019F8204684ED1F0AC4ED200A37
:106FB00084ED211AFFF72AFA28B1B2EE000A04F193
:106FC0007C0015F05DF8009BB3B33046FCF7CCFFB6
:106FD000012831D996F8C402B02303FB006696ED70
:106FE0002F7AF0EE087AB4EEE77AF1EE10FA23D5B4
:106FF00095F813030C2303FB005595ED627AF1EE2F
:107000000C7AB4EEE77AF1EE10FA15DBD4ED1D7AC6
:107010001FED927AF4EEC77AF1EE10FA0CDD1FED57
:10702000947AF4EEC77AF1EE10FA05D5B6EE000ABE
:1070300004F17C0015F024F85FED9A7AF4EEE78A0B
:10704000F1EE10FA22D51FED9C0A08A814F0C4FF37
:107050000EA88DED0E0A94ED3F0ACDED0F0A8DEDD1
:10706000101A14F0B9FF11A904F1A0008DED110A56
:10707000CDED120A8DED131A14F0CEFFD4ED2B7A5C
:1070800094ED3F7A77EE877AC4ED2B7A94ED2B7AE4
:10709000F1EE047AB4EEE77AF1EE10FA3BDB12F08F
:1070A00073FA5FEDB27A94ED2B1A94ED280A21EE73
:1070B000271A40F2C530F1EE410A8DED011ACDEDEF
:1070C000000A12F063FF9DED011ADDED000A84ED68
:1070D000280A40F2C63094ED290A12F057FF9DEDC0
:1070E000011ADDED000A84ED290A40F2C73094ED63
:1070F0002A0A12F04BFF04F1A00184ED2A0A04F1E0
:10710000940014F089FF84ED2A8A84ED298A84EDA5
:10711000288A84ED2B8A0023C4F8E430C4F8E830D0
:10712000C4F8EC3084ED3F8AA3E5E368F7EE000A8B
:1071300093ED000A12F028FE00283FF4D1AE94ED42
:107140001C0AB0EEC00A70F0F3FDDDED0A7A27EEFE
:10715000800A8DED0A0AC5E68DED0A8A8DED098A51
:107160008DED088AE2E62046FFF75EFC1CE6C3EDE3
:10717000007A04E72DE9F04D2DED048B9EB0044616
:1071800012F002FAD0EDC87A90ED618AF4EE487AF6
:10719000F1EE10FA48BFB0EE678ADFED5C7AB4EE2C
:1071A000E78AF1EE10FA0EDD0023C4F8E430C4F8EB
:1071B000E830C4F8EC300023C4F8FC301EB0BDEC5D
:1071C000048BBDE8F08D2046FEF7EEFD2046FEF76D
:1071D000A7FFB0EE480A2046FFF762FC2046FFF703
:1071E00023FCFEF7A9F914AD00F5347204F128016F
:1071F00014A813F041F90FCD04F14C060FC60FCDC2
:107200000FC62B68336004F1740204F1780304F1B3
:10721000700104F14C0013F0DDFA94ED1E8AB0EE1B
:10722000480A70F02FFC84ED650AB0EE480A70F051
:107230007FFD204684ED640AFEF7AAFDFEF77CF987
:1072400004F5B471FDF77EFF51F034F8D4F89831AD
:10725000C31A632BB2D9C4F8980132F0DFFE9FED58
:107260002C9A054651F02EF8D4ED1C7A67EE897AF7
:10727000074617EE900A0E46F9F73EF9D4ED1D7A4F
:1072800067EE897A824617EE900A8B46F9F734F951
:1072900094ED1E0A20EE090A41EC180B12F0E2FDF3
:1072A000D4F85C0110EE108AF9F726F9CDE9120145
:1072B000D4F85801F9F720F9CDE91001D4F85401B8
:1072C000F9F71AF9CDE90E01D4F8D800F9F714F955
:1072D000CDE90C01D4F8D400F9F70EF9CDE90A0193
:1072E0004046F9F709F90B4B01930B4B0093CDE99D
:1072F00008018DED068BCDE904ABCDE90276074B95
:10730000074A0849284632F015FC57E7CDCC4C3ED9
:10731000E02E6542952609089F2609085C26090883
:1073200066260908E824090808B52DED048BB0EE9F
:10733000609AF0EE408A00F011F9B0EE408A89EED2
:10734000280A70F02BFEDFED0B7A20EE270A70F092
:10735000BDFDDFED097A38EE278ADFED087A28EEE9
:10736000278AF7EE007A37EEC00A28EE000ABDEC55
:10737000048B08BD41D3423E33938843A1D81943BF
:10738000FFF7D2BF08B52DED048B9FED189AF0EEF4
:10739000E07AF4EEC97AF1EE10FAF0EE408AB0EE3F
:1073A000608A1ED400F0DAF8DFED117A9FED117AD1
:1073B00070EE277A9FED100AE8EEC77A9FED0F7AFC
:1073C00027EE800AC8EE007A87EE270AB4EEC90AD3
:1073D000F1EE10FA05DBBDEC048BBDE8084070F05F
:1073E000BDBEBDEC048BB7EE000A08BD0000003442
:1073F00033938843F4FDD43B48A18F43CDCC9C3FCD
:10740000427CD0ED257A242101FB020292ED0B0A89
:10741000D2ED090A30EE270AFFF7B4BF38B52DEDDB
:10742000088BDFED21AA9FED21AA9FED21BA054629
:10743000B0EE409AF0EE609AB0EE408A1524013C1E
:10744000A4B25CB3F0EE490A2846B0EE480AFFF752
:107450006BFFF0EE490A70EE698A284638EE2A0A78
:10746000FFF762FFB0EEE87A70EE697AB4EECA7A9E
:10747000F1EE10FA77EEE87A10D468EEAA8A40F2BC
:10748000631088EEA70AB0EE4B1A38EE400AF0EE11
:107490004A0A12F07BFDB0EE408AD0E7B0EE480A0F
:1074A000BDEC088B38BD00BFCDCCCC3D0AD7233C0A
:1074B00000247449002343608360C3600361436117
:1074C0008361C361002380F82030704790F820204A
:1074D000531CDBB2062B80F8203000EB820288BF01
:1074E000002382ED010A88BF80F820307047000039
:1074F0004FF0FF3310B543610E4BC0F8A8300023A6
:10750000044680F8C830A830FFF7D4FF0A4BC4F80F
:10751000A83004F5867050F083F8084B08491C60C9
:1075200020462EF04FFDD4F89030C4F89430204619
:1075300010BD00BFC8280908D8280908EC59002048
:107540007029090808B5A83033F098FDDFED027AFC
:1075500020EE270A08BD00BF00007A4490ED3C0AE7
:10756000DFED057AB0EEC07AB4EEE77AF1EE10FA0C
:1075700048BF90ED3D0A70470000003473B5D0F865
:10758000A43004460E4663B150F094FED4F8A43003
:10759000C01A42F20F73984203D894ED280A02B041
:1075A00070BD114B1D687DB195F84E112846FCF752
:1075B00039FB48B195F84E1101AA2846FCF728FB83
:1075C00010B19DED010AEAE7242101FB064494ED88
:1075D0000A0ADFED067AB4EEE70AF1EE10FA58BFB8
:1075E000B0EE670ADBE700BFE459002000000C4260
:1075F00008B561B10378022B02D9064850F028FE85
:107600005A1C027000EB83004160012008BD08464F
:10761000FCE700BF842709082DE9F84305460E461C
:107620009146002400F13C082B78A34211DD002391
:107630004A46314601200EF05FFF2423634307468C
:10764000002158F803000EF067FF874204D0013490
:10765000EAE70020BDE8F8830120FBE7054B1B6843
:107660002BB141694A1C02D0184632F0A1BC00205F
:10767000704700BF945C002002290BD8242303FB31
:10768000010191F8390030B191F83A0018B191F840
:107690003B007047002070472DE9F047044650F04A
:1076A00009FED4F8F86042F21073861B9E4288BF30
:1076B000C4F8F80000274FF0240942F2107A237C26
:1076C000FDB2AB421CD929462046FFF7D5FF70B169
:1076D00009FB054898ED0D0AD8ED097AD4ED250A85
:1076E00030EE270A2046FFF799FE88ED0C0A564532
:1076F00004D909FB054030302EF03CFE0137DEE7AF
:10770000617C2046FFF73AFF84ED3D0ABDE8F08733
:1077100070B5044686B050F0CDFDD4F89830C31A49
:10772000B3F57A7F05464FD3344B94ED257A1B6829
:10773000DFED336ADB6AD4ED247A93F89C60B0EE17
:10774000C76AB4EEE66AF1EE10FA32D5B0EEE76A37
:10775000B4EEE66AF1EE10FA2BD502A801F06AFF4A
:1077600096BBFDF7E9FE02A9FDF7ECFC60B3DDED89
:10777000037A9FED247AF8EEE77A67EE877AC4ED14
:10778000257AC4F89850FDF7D7FEFDF7C3FA2046D6
:10779000FFF782FF3BF094F90546D4F89400F8F720
:1077A000ABFE194ACDE900010621284634F0B8FBAA
:1077B0000AE037EE676AF7EE005AB0EEC66AB4EE3A
:1077C000E56AF1EE10FA01DC06B070BDB0EEE76AD2
:1077D000B4EEE66AF1EE10FAF6D4002ECFD02046D1
:1077E000903080ED007A2EF0C5FD3BF069F9074A34
:1077F000012106B0BDE8704034F092BBCC250020DA
:10780000000000340AD7233CC5270908A02709082F
:10781000F0B52DED048B85B004464FF4537200F59E
:10782000867103A80EF0F4FFD4ED227AD4ED236A1A
:107830009FED796A637C37EEE67A2422B0EEC77A50
:10784000B4EEC67AF1EE10FAC1BF9FED747A67EE1E
:10785000877A9FED737AE6EE877A02FB0343002571
:10786000C4ED237A93F839602378E9B28B4206D9C4
:1078700004EB81030135586852F090F8F4E7DFED2E
:10788000698A9FED698A9FED699A0027237CFDB282
:10789000AB4264D9242303FB054393F83920002A23
:1078A0005BD0D3ED0C7AF4EEE87AF1EE10FA0BDB54
:1078B000F4EE677AF1EE10FA06D6F0EEE77AF4EE1F
:1078C000487AF1EE10FA04DD242303FB05435A6ADB
:1078D0001A63242303FB0543D3ED090AD3ED0D7A84
:1078E00093F8382070EEA70AA2B993ED0C0A20464F
:1078F000FFF746FDD4ED257A30EE670AB4EE400A74
:10790000F1EE10FA16D7242303FB0545002385F872
:107910003A3022E0012A09BFD3ED0C7A93ED0B0A2D
:1079200077EEE00AD4ED3B7A04BF80EE897A87EEE9
:10793000270AE3E7F0EEC07AF4EE487A2423F1EE6A
:1079400010FA03FB0545E1DC012385F83A30D4ED5C
:10795000237A37EE800A85ED0B0A013796E7627CC1
:1079600020461146FFF788FE48B1242101FB024260
:1079700092ED0B0AD16904F1A80033F05FFB94F992
:107980009C10277C002907DBB94205DACAB21146F0
:107990002046FFF771FE68B900226274D5B2AF428B
:1079A00009D929462046FFF767FE01320028F5D0A5
:1079B000657400E062742046FFF7AAFE2046FFF7D8
:1079C0004DFE10B1204652F0EFF8637C242505FBF4
:1079D000034393F83930B34216D032F01FFB4FF611
:1079E000FF7132F0E5FA78B1607C05FB004494F851
:1079F0003930002B14BF00220422019232F00EFB1A
:107A0000019A122132F066FA03A80EF023FF05B0A6
:107A1000BDEC048BF0BD00BF0AD7233C0AD7A33CC2
:107A200048E17A3F00000034FFFF7F7F00201946C5
:107A30002DE9F04F0446007C0F4687B004F13A036D
:107A400000220121D5B2A84203F1240305D903F88D
:107A5000231C03F8241C0132F4E7744B1E68F06AFF
:107A600003685B68984740B13BF02AF8704A0621EA
:107A700007B0BDE8F04F34F053BA23781BB1237C34
:107A80000BB163681BB93BF01BF86A4AEFE73BF0A8
:107A900017F8694A062134F043FA002303A904F1D8
:107AA000880003932FF01CF80A2550F003FC804651
:107AB0002046FFF7ADFE50F0FDFBA0EB0800B0F54F
:107AC000FA7F02D95D4800F04BFFB06A03680A21D3
:107AD0005B689847617C2046FFF7CEFD0028E7D021
:107AE000B06A036864215B68013D984715F0FF05A3
:107AF000DBD1534B05951B888DF80650CDE9035516
:107B0000ADF80430052550F0D5FB80462046FFF740
:107B10007FFE50F0CFFBA0EB0800B0F5FA7FD1D884
:107B2000617C2046FFF7A8FD0028EFD094F810B044
:107B30000DF10C08A14601AA4FF0000A5FFA8AF184
:107B40008B4516D92046FFF797FD50B1D8ED007A46
:107B500099ED097A137877EE877A0133C8ED007AC8
:107B600013700AF1010A08F1040809F1240901322D
:107B7000E4E7B06A036864215B68013D984715F04B
:107B8000FF05C0D1A9464FF02408237C5FFA89F68F
:107B9000B34226D906AB334413F8143C33B908FB7F
:107BA000064686F83B3009F10109EEE7002FFAD0CE
:107BB00007EE903A06AA02EB8602F8EEE77A12ED9B
:107BC000030AD4ED250A204680EE270AFFF726FC9B
:107BD00008FB064002A930308DED020A2EF080FF2E
:107BE000E1E7617CDFF860902046FFF7C7FC0026E4
:107BF00084ED3D0A4FF02408237CF7B2BB420FD935
:107C000008FB074393F83B3043B13AF059FF7B1C24
:107C10004A46062134F084F90135EDB20136EBE72E
:107C20000DB908484FE707B0BDE8F08FCC2500201C
:107C3000E02709080B280908382809084E280908F0
:107C400098E308088A2809086828090808B5037C09
:107C5000022B02D9034850F0FBFA5A1C0274184652
:107C600008BD00BFAC28090838B5057C02460024D1
:107C7000E1B28D4206D91046FFF7FEFC0134002820
:107C8000F6D138BD281E18BF0120FAE770B50D46A1
:107C900009780729044606D8027E437E22B90122CC
:107CA0008A401343437670BD002BFCD00026227817
:107CB000F3B29A42F7D904EB830329465868036864
:107CC000DB6898470136F2E7014B1868704700BF40
:107CD000EC59002010B50446006810B103685B68D9
:107CE0009847204610BD000010B50446006810B14A
:107CF00003685B689847204610BD000070B5D0ED62
:107D0000247A9FED5F7AF0EEE77AF4EEC77A0123EA
:107D1000F1EE10FA8AB00446037609D490300023BD
:107D200009A9059009932EF0DBFE05982EF022FBA1
:107D30000026E6632666C4F8846077223146204632
:107D4000FFF76AFC0546002833D0CDE90666079A9E
:107D50000992002309A92046CDE9073351F082FD9D
:107D600001462046FFF744FC09A8FFF7B3FF08A827
:107D7000FFF7B0FF07A8FFF7B7FF15B106A8FFF799
:107D8000B3FF2378032B4DD0237C032B4AD094F9E7
:107D90009D1000291CDAD4F80031DA0454D40025EF
:107DA000637EEB40DB07EAB254D40135082DF7D1EE
:107DB00038E0344B1B68596804220B68CDE9010296
:107DC000314A00921E680246772307A8B047BEE7F3
:107DD0007722C9B22046FFF71FFC054620B30023D7
:107DE000CDE90633079B0993002209A92046CDE976
:107DF000072252F00DFC01462046FFF7F9FB09A8C7
:107E0000FFF768FF08A8FFF765FF07A8FFF76CFFFB
:107E100015B106A8FFF768FF2378032B02D0237C57
:107E2000032BB8D10AB070BD164B1B6859680422E9
:107E30000B68CDE90102144A00921E6894F89D2057
:107E4000772307A8B047CDE7637E002BA7D1012396
:107E50006376A4E73820059201F088FE064618B143
:107E6000059A214652F072FC31462046FFF7C0FBCE
:107E70002378032BD6D0237C032B96D1D2E700BFE7
:107E800000000034CC250020801A060090F8183538
:107E9000934207D902F59E7250F8220010B1036890
:107EA0009B6A1847002070472DE9F34105466E464E
:107EB00086E80C00134B45F8043B04460F4600F5DA
:107EC000C87828462C3500F073FCA845F9D196E80F
:107ED000030004F21C53C4F8147583E80300089BE4
:107EE000C4F82435084920462EF06CF8074B1A6870
:107EF00012B1074850F0ACF920461C6002B0BDE852
:107F0000F08100BF902C0908582B0908F059002077
:107F10009C2A09082DE9F041A2B00C4607A92DF0D2
:107F200027FB002855D000210D220CA80591ADF8A3
:107F300018100B9172F0AEF92B4B611C1F68C9B27F
:107F40000BAD0129F86A0A9546D1284B062205A9EE
:107F50000EF03EFE264B019305AB00930024112248
:107F60002946244BF86A8DF819400EF031FE04AA18
:107F70000DF10F0128468DF83C4004942EF08EFC44
:107F800038B31D49DFF86C80482210A872F038F928
:107F9000062610AC2268531E049AC2F3513202EB3B
:107FA000831223798DF82430A368019305AB0093E5
:107FB0000892434611222946F86A0EF009FE002174
:107FC000B7EE000A07A82DF0D5FC013E04F10C0421
:107FD000E0D122B0BDE8F0810091084B062205A94E
:107FE0000EF0F6FDB6E700BFCC250020211A0908E7
:107FF000CD2A0908C72A09089CE30808C02A0908ED
:108000002DE9F74F90F818650446002E40D17F23E4
:1080100080F8283500F5C87500F59E68071D5FFAE1
:1080200086F91822FF21284672F034F985F8579016
:1080300097F924A0BAF1090F4AD02CDCAAF1030366
:10804000DBB2012B37D9D8F8000050B1E96DC5F883
:1080500058A031B1244B43F826102EF0C1F92EF070
:10806000B7F958F8040B09F1010A5FFA8AFA40B12E
:1080700003689B68984784F818A549462046FFF78F
:1080800049FF0136092E05F1600507F12C07C6D11D
:1080900003B0BDE8F08FBAF10A0FD4D1302001F05F
:1080A00065FD834688B1CDF800903B462A462146BF
:1080B00053F0D2F909E0442001F058FD834620B185
:1080C0003B462A46214652F0CDFBC8F800B0BAE73D
:1080D000382001F04BFD83460028F6D03B462A4667
:1080E000214653F017F8F0E7F459002090F81835BE
:1080F0008B4283BF602303FB010090F8D501002071
:108100007047000090F818358B4283BF602303FB53
:10811000010090ED6A0A9FED010A7047000000001F
:1081200090F818358B4206D901F59E7150F8210060
:1081300008B152F02BBD9FED010A7047000000000E
:1081400010B490F818458C420A4614D901F59E7473
:1081500050F824407CB1E468246A640603D55DF8D5
:10816000044BFFF7DDBF602101FB020393ED6A0AB8
:108170005DF8044B70479FED010AF9E7000000002D
:1081800090F818358B420BD901F59E7150F82100FB
:1081900038B1C3681B6A1A4214BF0120002070471F
:1081A0000020704770B590F81835934204460E468B
:1081B000154601D8002070BD02F59E7350F82300CB
:1081C0000028F7D003689B6998470028F2D0602206
:1081D00002FB0544D4F8AC313360ECE770B590F89D
:1081E0001835934204460E46154601D8002070BD4E
:1081F00002F59E7350F823000028F7D003689B69AE
:1082000098470028F2D0602202FB0544D4ED6C7A36
:10821000F4EE677AF1EE10FAE8D6C6ED007AE6E7FA
:1082200070B590F81835934204460E46154601D8AD
:10823000002070BD02F59E7350F823000028F7D08F
:1082400003685B6998470028F2D0602202FB05446E
:10825000D4F8B4313360ECE790F8183593420ED976
:1082600002F59E7350F823305BB1602303FB0202DA
:1082700092F8E40130B1D2F8E0310B607047002091
:10828000704718467047000008299DBF2C2303FB48
:1082900001004068002070472DE9F04F4B4B2DED59
:1082A000028B1B68DB6A93F89C3089B00446002B74
:1082B00000F08680DFF82CB19FED458A4FF0000971
:1082C00094F818355FFA89F5AB4279D905F59E73B4
:1082D00054F8230000285DD003685B6B9847602347
:1082E00003FB0543074693F8D431834252D2032857
:1082F00061D8DFE800F04F025259364E4FF00008C7
:108300003AF0DEFB94F81825AA4284BF602202FBF3
:1083100005424FF0600105F1010301FB05458CBFEB
:10832000D2F8A82118EE102A8246D5F8B001CDE97E
:108330000632F8F7E1F8079ACDE904011046F8F79C
:10834000DBF8069B0096CDE902015A46042150460F
:1083500033F0E6FD0123204A84F8293585F8D471ED
:10836000D372D4F824354BB3002255B25957481C68
:1083700003D0414502F10102F7D194F92835AB420F
:1083800008DBD4F82035D4F81C054246314698471E
:1083900084F8285509F1010992E72C2303FB0543D2
:1083A0000E4E93F92B80ABE72C2303FB05430C4EB9
:1083B00093F92C80A4E70026B046A1E71D46DCE730
:1083C00009B0BDEC028BBDE8F08F00BFCC250020CA
:1083D00000000000E12A0908755A0020062D0A084D
:1083E000D82A0908F02A090890F818358B4207D9CD
:1083F00001F59E7150F8210010B10368DB69184740
:108400000020704708299CBF602303FB010000F592
:10841000C870704790F81835934207D902F59E72DC
:1084200050F8220010B103685B6A184700207047BB
:108430002DE9F04F002493B005460E46174621461D
:108440002F2206A8059405F59E6971F023FF05F11A
:10845000280A4FF02C0B05F5F4730BFB04F259F8C6
:10846000040B1AF90210E5B230B951B90134092CE4
:10847000F3D14FF0010813E0602262439A58914211
:1084800012D01548154B006801930135EDB20095E7
:10849000134BC06A324639460EF09AFB4FF0000883
:1084A000404613B0BDE8F08F05A93322039352F084
:1084B0004FFC039B804605A90028D7D106480191AF
:1084C0000135EDB200680095054BC06A3246394669
:1084D0000EF07EFBE4E700BFCC250020262B090828
:1084E000182B09082DE9F04FDFF88090DFF880A005
:1084F000DFF880B08DB00646002796F81835FCB23C
:10850000A3422ED9602505FB046595F8DC3133B311
:1085100095F8DD1119BB4FF001082022444404A84E
:1085200089F8198071F0B6FE07EE904A4AF21043BE
:10853000F8EEE77A03AA4C21ADF828305046242300
:10854000CDED037A35F0ECFB3AF0BAFA9BF8003047
:10855000054A0094042133F0E3FC85F8DD810137FE
:10856000CBE70DB0BDE8F08F302B0908755A00201D
:10857000215D0020052300202DE9F04F2F4B1E68C0
:1085800085B0044646B1D0F81415304631F010FDE0
:1085900010B1304630F06EFC4FF08CFE4FF000080A
:1085A00001904FF02C0A4FF0600B94F818355FFAE9
:1085B00088F5AB4239D904EB8507D7F8F00488B3C6
:1085C0000AFB05430BFB054993F92820D9F8E8116C
:1085D0008A4227D132B30268D2689047D7F8F004B4
:1085E0000268126B904799F8D52112B1019BC9F826
:1085F000D831BEB1D4F81415304631F0D9FC88B169
:108600004FF060FECDE9021002460B46D7F8F004A9
:10861000294652F093FDDDE90232D7F8F0042946ED
:1086200052F00AFE08F10108BFE72046FFF734FECA
:10863000204605B0BDE8F04FFFF754BF945C002022
:108640002DE9F0474FF000082DED028B04468946D6
:10865000B0EE408A474601264FF0600A94F818357C
:108660005FFA88F5AB421AD929FA05F3DB070AD578
:1086700005F59E7354F8230078B10368B0EE480AFC
:108680009B6B984706400AFB054508F1010895F8E1
:10869000D4319F4238BF1F46E0E70646F3E727B9CB
:1086A0007F23A4F82835034BDF72BDEC028B3046E4
:1086B000BDE8F087755A002090F818358B4207D92D
:1086C00001F59E7150F8210010B10368DB6B18476B
:1086D000002070470B46114690F818259A4207D99A
:1086E00003F59E7350F8230010B103681B6C184704
:1086F0007047000070B504460E46002594F8183502
:10870000E9B28B4205D932462046FFF7E3FF013537
:10871000F4E770BD2DE9F84390F81855024600249F
:1087200000F128062C2700F5F4784FF06009E1B23B
:108730008D420FD907FB04F309FB04F0F35658F8F8
:108740000000834209D11BB11046FFF7CFFC10B1E6
:108750000134ECE70120BDE8F8830020FBE70000CE
:1087600010B590F818258A42044617D9602202FBFA
:10877000010393F8D431022B03D004D9032B18BF83
:108780000023184610BDFFF797FF48B92046FFF7B2
:10879000C1FF00280CBF06230123F2E70023F0E706
:1087A0000623EEE7014B1868704700BFF059002020
:1087B00010B5034904462DF005FC204610BD00BF4E
:1087C000082D090810B50446203043F01FFA044B69
:1087D00004491C6020462DF0F5FB204610BD00BF6B
:1087E000185A00207C2E0908F7B5B7EE000A0022BF
:1087F000022104462DF0D6F9204652F077FE43F0D0
:10880000E9FA144B1D680646E86A03685B6A9847F4
:108810000B46022102460091304643F00DFAB4F9AE
:108820004A60002E14DDEF6A3B6838465B68B4B2DC
:10883000984728B197F84D3013B1C92EA8BFC82466
:10884000A86A03685B68214603B0BDE8F04018479A
:1088500003B0F0BDCC25002010B5044652F014FE44
:108860002046BDE8104052F03FBE00002DE9804890
:10887000284BDFF8A490DFF8A4A0DFF8A4B01446DA
:10888000012293B005460E461A704FF000084FF0D3
:1088900011FDD9F800300393A0EB080241F28733B1
:1088A0009A4207461FD9CDE9005603985346342211
:1088B00005A9C06A0EF08CF9214605A804944EF073
:1088C0002DFFCDE9005603985B46342205A9C06A06
:1088D0000EF07EF904943AF0F3F8049B05AA022105
:1088E00033F004FBB8463AF0EBF839F0E7F93AF028
:1088F000E7F83AF0EFFF0A2105A80DF06FFF039BA0
:10890000986A036805215B68984705A80DF072FF17
:10891000BDE700BF1C5A0020CC250020F82D090817
:1089200021410A080FB400B595B016AA002152F8EB
:10893000043B039205A83C220193049171F0AAFC28
:10894000054A019B402104A84EF090FE039A03487B
:1089500004A9FFF78BFF00BF002E0908162E090897
:108960000FB407B504AA034852F8041B0192FFF79D
:108970007DFF00BF282E09080146D0E9070300B19A
:108980001847002BFCD17047B0F9023002889A4397
:1089900014BFC3F3C00000207047000038B50723A0
:1089A0000380022200230525C0E90532C0E90D330A
:1089B000C0E91033C0E92C330C490362C0F89C5065
:1089C00004462DF0FFFA0A4B196811B109484FF01F
:1089D0003FFC94F910001C602A4611F015FB637CE3
:1089E000207403F010036361204638BDCC2F0908C2
:1089F000205A00200C2F0908012343610423C3647B
:108A000070470000002343610423C36470470000E3
:108A10000123C364704700000223C3647047000051
:108A20000323C3647047000010B5C36993B190F984
:108A3000514090F950309C4207DA074B07480068D4
:108A4000C06A0EF0C5F8002010BD036A012B01D8E2
:108A5000034BF3E70120F7E7282F0908CC25002076
:108A6000342F0908F8B504463BF0ACFA3BF096FA0F
:108A70003CF054F907463BF0A5FA3BF099FA3CF07C
:108A80004DF906463BF09EFA3BF074FA3CF046F98D
:108A900005463BF097FA3BF077FA3CF03FF9024687
:108AA000606C50B101285FD1012E5DD1012A5BD1EC
:108AB000012D14BF00200820F8BD012F28D176B960
:108AC000012A61D1012D63D1627CD70705D494F9C5
:108AD000511094F95020914210DA0220ECE7022E56
:108AE00016D1012A50D1012D52D1627CD60741D432
:108AF00094F9511094F9502091423BDB6269216C4A
:108B00008A421AD0002A33D0012A08BF0A20D3E7AC
:108B1000002D3BD0012E0BD1012A09D1022DEDD120
:108B20002046FFF731FF002814BF04200320C3E7CD
:108B3000E2B1022AE2D10620BEE7E26CA16B8A42D2
:108B4000BAD0012A1DD1617C0D0715D4617C49077B
:108B500010D4022A12D1617C0B070DD4627C12F072
:108B6000040F18BF0220A7E70020A5E70520A3E710
:108B70000920A1E701209FE710469DE7042A9BD129
:108B8000ECE7032AE5D1E1E7002DD1D1072093E7F7
:108B9000002DB3D1FAE700004B6A022B4FF000031F
:108BA00003D080F84830436470478A68032A05D0B0
:108BB000042A05D0002380F8483070474364F9E761
:108BC0000B680A7B5B78012A03F00F0305D0022AA9
:108BD000F0D1002BEED00262ECE7002BEAD00523A7
:108BE0000362E7E7FFF7D8BF037C033B022B94BF88
:108BF0000120032070470000037C033B022B94BF3D
:108C00000120042070470000C06910B103681B6A8E
:108C10001847704770B50446C069036800215B6C53
:108C20009847E069036801219B6C9847E0690368F5
:108C30000021DB6B9847E5692B682846D3E90D6373
:108C4000984740F4407081B22846B0470A23E06953
:108C50001A464FF4E1310DF087FEE0690368BDE884
:108C600070401B6A18470000033904299ABF024B61
:108C700058560020704700BFC42F0908F7B5C369D4
:108C800004466BB3E2B9012915BF00230123032772
:108C90000427CC208DF804008DF805100BB18DF859
:108CA0000620002630467D1EF3B2AB4206F10106D7
:108CB00009DA02AA134413F8041C11F069FAF3E765
:108CC00001230427E5E702AB1D443A4605F8040CEE
:108CD000E069036801A9DB689847E0690DF0A0FE30
:108CE00003B0F0BD10B5C4693CB18469012C06D154
:108CF000C262CAB22146FFF7C1FF204610BD002064
:108D0000FCE70000042910B5044604DC02290DDC50
:108D100001290ED010BD0A29FCD1FFF765FFE268DA
:108D200001462046FFF7DEFF032306E0437C9B0756
:108D3000F0D5FF23A4F8523004232362EAE70000B1
:108D400010B590F8513080F85030044643F094F953
:108D500020B100F58050002380F884346369012B32
:108D60000DD163885B060AD52046FFF73DFFE26818
:108D700001462046FFF7B6FF0323236210BD0223FE
:108D8000FBE70000013938B50446062969D8DFE859
:108D900001F0042031688B8BB60090F95030002B25
:108DA0005FDC013380F85030C2680221FFF79AFF80
:108DB00094F95030002B0ADD43F05EF920B100F544
:108DC0008050012380F884340523236249E0042382
:108DD000FBE790F95030002B08DD013BC26880F8BA
:108DE00050300221FFF77EFF0623EEE7BDE8384052
:108DF000FFF7A6BF90F9503090F95210012B20DDFB
:108E000090F91000484D421EC2EBC202AB18AA5C9A
:108E10002AB353FA81F394F853205B78013B9A42CA
:108E20001DD105281BD0A26800212046FFF75AFF5C
:108E3000002384F8533094F85030013B84F85030CC
:108E40000FE00CD190F910203748531EC3EBC30339
:108E5000C35C23B1013B994201D1052A02D100290B
:108E60000BDA38BDE26800212046FFF73BFF94F89B
:108E70005030013B84F85030B6E794F910302A4A5C
:108E8000013BC3EBC30313440B445B78002BE8D0D6
:108E9000A26800212046FFF725FF94F950300133E6
:108EA000022BA8BF0223C9E701218268FFF71AFF3E
:108EB00094F950301C49012B94F9103011DD013B1D
:108EC00094F8520094F85320C3EBC3030B440344BB
:108ED00001325B78B2FBF3F103FB112284F85320DB
:108EE000BFE7013BC3EBC30394F95220CB5C0132D3
:108EF00092FBF3F103FB112284F85220B1E790F9C1
:108F00005030002B09DD013B80F850300023C2684F
:108F100080F853300221FFF7E5FE94F95030002B22
:108F20009FD194F85130A5E70D22002010B5436978
:108F3000012B044610D143885B060ED5437CD9062D
:108F400007D4FFF751FEE268014652002046FFF7C2
:108F5000C9FE0323236210BD0BB10223FAE7438845
:108F60005A06FAD5437CDB06F7D5FFF745FEE268E3
:108F7000014652002046FFF7B5FEEEE7042910B582
:108F8000044604DC02290DDC01290ED010BD09299C
:108F9000FCD1FFF731FEE26801462046FFF7A2FE52
:108FA00002230EE0437C9B07F0D52046FFF724FE0A
:108FB000E26801462046FFF795FEFF23A4F85230F1
:108FC00004232362E2E7000010B504464FF072F973
:108FD000A36AE26AC31A934207D3226AA0620023FB
:108FE000022AE36202D0032A10D010BD6269012A6E
:108FF0000AD1638813F0400F0CBF00210A212046DC
:10900000BDE81040FFF77EBE1946F8E7616949B92F
:10901000638813F0400F18BF09212046BDE81040B7
:10902000FFF7ACBF1946F8E773B50B685B7883614F
:1090300043885B045EBF0B685B884380B0F90230F5
:10904000002B04461ADD0123036239F039FD054681
:109050002046B4F90260FFF797FC68B92388B34350
:109060000CBF022300230093094A334606212846F9
:1090700032F056FF02B070BD0523F4E739F020FD51
:10908000044A042102B0BDE8704032F049BF00BF7D
:10909000482F0908792F0908FFF7C6BF70B50446A5
:1090A000D0F8B8000E46E8B1D4F8A83023B1D4F80F
:1090B000A420CB1A934221D3B4F8AC509DB12046E2
:1090C000FFF7A8FDD4E9260194F8A020FFF7D6FD0C
:1090D000B4F8AC30C4F8A8600020013B84F8A100CB
:1090E000A4F8AC3070BD042304F19400C4F8B83087
:1090F000FFF742FCC4F8B8502846F3E70120F1E737
:1091000038B50024054620466B7BA34205DD2B685D
:10911000195D11F03DF80134F6E738BD2DE9F04155
:10912000C3690446002B43D04FF0C4F801462046E3
:10913000FFF7B4FF00283BD0E06903685B699847FC
:10914000402828BF40200025064604F19407A84681
:10915000AE422DD04FF0AEF801462046FFF79EFFFD
:1091600030B3E06903689B69984794F8A130C0B2B6
:109170000BB9CC281AD1D4F89420D05494F8A1304B
:1091800094F8A2200133DBB29A4284F8A1300DD1C9
:109190003846FFF7B5FF00280CBF02230323C4F8AD
:1091A000B8303846FFF7E8FBC4F8B8800135CFE7A0
:1091B000BDE8F081074A002352F83300884203D10A
:1091C00002EBC303187970470133042BF4D100205C
:1091D000704700BF3022002038B50373002343736B
:1091E000049B03611546BDF81430856001F15402FB
:1091F0000446C0E90021038300F11C03DDE90601F8
:1092000083E80300012363624FF054F8294660614C
:109210002046FFF7CFFFA073204638BD2DE9F0436D
:109220008FB016AC064634F8049B0F4690461D4698
:10923000FFF7EAFC94E8030002AB83E803003A4638
:10924000CDE900594346314604A804ACFFF7C4FFFA
:109250000FCC06F194050FC50FCC0FC594E80300A1
:10926000424685E80300394630460FB0BDE8F0437A
:10927000FFF704BD10B586B0094B0593049006AA0C
:1092800012E9030001AB83E8030000224FF6FF73ED
:10929000009311464FF47A63FFF7C0FF06B010BD8C
:1092A0009990010813B51A4B0446186820B10022A2
:1092B0001A212EF04FFCE061E36953B101230DF157
:1092C000070104F110008DF807302DF045FC2DF05A
:1092D0007FF894F9103013B9E36102B010BDE26970
:1092E000002AFAD0022B01D0052B03D14FF6FF73D1
:1092F000A4F850302046FFF78DFC4EF0DBFF63688A
:10930000A0622046E36202B0BDE81040FFF7B2BFA2
:10931000445B002030B587B004AB83E80600054607
:1093200093E8030001AC022384E8050004210093C4
:1093300001224FF4C8732846FFF770FF07B030BD15
:1093400030B587B004AB83E80600054693E8030018
:1093500001AC84E80500022200924FF4C873042196
:109360002846FFF75BFF07B030BD000010B586B0A0
:1093700006AC04E90C0061B10124446401AC84E84A
:109380000C000224CAB200944FF4C8732146FFF7C0
:1093900045FF06B010BD000070B586B004AB83E891
:1093A000060002254564044693E8030001AE86E802
:1093B00005004FF4C8730095002203212046FFF7F3
:1093C0002DFF06B070BD000010B5012380F84830B5
:1093D0004B1E88B00446C262072B31D8DFE803F089
:1093E000040E181818181825164B00901A46014636
:1093F000019308B0BDE81040FFF78CBF114B0290FD
:109400001A460146039308B0BDE81040FFF798BF25
:10941000FFF72AFC0B4B0494014622462046059395
:1094200008B0BDE81040FFF7A1BF064B07930690B8
:1094300008AB13E9060008B0BDE81040FFF7ACBF69
:1094400008B010BDE58B01084B1E10B50446092B72
:1094500020D8DFE803F00C233636363636053636AC
:10946000642208212046BDE81040FFF7ADBF90F907
:10947000503083B942F000FE20B100F58050012346
:1094800080F88434642201212046FFF79DFF0123E8
:1094900084F8503010BD64220321E3E790F9503086
:1094A000002BF7DD42F0E8FD20B100F580500023ED
:1094B00080F88434642202212046FFF785FF0023D0
:1094C000E6E76422CEE7000013B504460191FFF7FA
:1094D0005BFA019928B1204602B0BDE81040FFF7C1
:1094E000B3BF2388B4F90220934305D1204602B0CC
:1094F000BDE81040FFF746BC02B010BD70B5044691
:109500004EF0D8FE94F8482022B9A36AE16AC31A43
:109510008B4202D20023236370BDC4E90A022046B5
:10952000FFF7A0FA236B626983420146236AE06C6D
:109530000ED1656BAB420BD1A56B854208D194F976
:109540003C6094F95050AE4202D1256C9542E3D074
:10955000C4E90C13A063013B94F8500084F83C006C
:109560002264052BD8D8DFE803F003080D12131886
:109570002046BDE87040FFF7D9BC2046BDE87040EA
:10958000FFF7C0BB2046BDE87040FFF7F7BC0121E4
:109590002046BDE87040FFF797BF0221F8E70000C2
:1095A00010B50D4B1B68DB6A93F89C30044623B161
:1095B0002046BDE81040FFF707BD42F05DFD28B131
:1095C00000F5805393F86434032BF1D82046BDE8AE
:1095D0001040FFF793BF00BFCC25002038B5C3690A
:1095E00004467BB190F9103063B1FFF797FD4EF060
:1095F00061FE636AC31A642B054603D92046FFF750
:10960000CFFF656238BD0000014B1868704700BF8E
:10961000205A002008B50449102270F0E1FDB0FA8C
:1096200080F0400908BD00BF245A0020102200210C
:1096300070F030BE10B50446FFF7F8FF204610BDAD
:109640000378416023F00D03022A037008D0032A37
:109650000AD0012A03D1DBB243F001030370704743
:10966000037843F00803F9E7037823F0050343F098
:109670000503F3E773B504460E4615460193FFF75D
:10968000D5FF2046C4E90265069A0199FFF7D8FF85
:1096900002B070BD0078420704D4030704D400F080
:1096A000010070470320704702207047F0B585B075
:1096B00005461646FFF7EEFF88420F4605D16B6858
:1096C00033600124204605B0F0BD032801D10024F9
:1096D000F8E70329FBD001280BD0022816D018BBCD
:1096E0006D68012F22D0022F2ED0002FEFD13560D0
:1096F000E7E7FBF721FF90F87C32DB07E7D56D68E1
:10970000FBF71AFFD0F870321D44EAE76846FFF70E
:109710008DFFFBF711FF6946FBF714FD0446002897
:10972000D0D06D68019BEFE70025DAE7FBF704FF77
:1097300090F87C4214F00104C9D0FBF7FDFED0F88C
:109740007032ED1A3560BDE76846FFF76FFFFBF733
:10975000F3FE6946FBF7F6FC04460028B2D0019BF5
:10976000EFE7000073B501AA05460E46FFF79EFF1E
:10977000044620B1019932462846FFF761FF204692
:1097800002B070BD13B5144601AAFFF78FFF48B1B0
:10979000DDED017A9FED047AF8EEE77A67EE877ADD
:1097A000C4ED007A02B010BD0AD7233C07EE900A40
:1097B0009FED090AF8EEE77A08B527EE800A6EF009
:1097C00061F9DFED067AB4EEE70AF1EE10FAD8BFE0
:1097D000B0EE670A08BD00BF50E0EF300AD7233C67
:1097E00010B50446806810F07BFD20B1E068BDE84C
:1097F000104010F089BD10BD0D4B83424FF00003A7
:109800008B4106DA00F1255000F5311000F5E050EB
:109810007047084B98424FF0FF3371EB0303BEBF14
:1098200000F1564000F5130000F52440704700BFDA
:1098300000D2496B002EB69490EA010F01D4401A71
:109840007047C317401A63EBE1710D4B83424FF031
:1098500000038B4106DA00F1255000F5311000F5C8
:10986000E0507047074B98424FF0FF3371EB030312
:10987000BEBF00F1564000F5130000F524407047CC
:1098800000D2496B002EB69470B52DED028B84B0DA
:10989000044668460D46FFF7C9FEFBF74DFE6946D4
:1098A000FBF750FC064608B3A368029ADFED128A64
:1098B00003999B1A07EE903AF8EEE77A67EEA87ADA
:1098C000C5ED007AE068FFF7B7FF08EE100AA06860
:1098D000024402EBD272B8EEC88A5010FFF766FF5E
:1098E00028EE288A28EE000A85ED010A304604B0E9
:1098F000BDEC028B70BD00BFF67C8E3F37B50023F8
:109900000C4601AA022105460193FFF7CFFE10B9CC
:10991000002003B030BD21462846FFF7B5FF0028E0
:10992000F6D0DDED017AF8EEE77AC4ED027AF0E7E1
:1099300038B52DED028B0C460246C168E068FFF792
:109940007BFF9568A46808EE100A601900EBD070E0
:109950004010641BFFF72AFF07EE904AF8EEE77A03
:10996000F8EEC80A87EE807ABDEEC70A10EE103A0C
:109970005B4200EE103AB8EEC00A6EF0A5FADFEDD9
:10998000087A30EE270ABDEC028BB5EEC00AF1EE84
:1099900010FA44BFDFED037A30EE270A38BD00BF6E
:1099A000DB0FC93FDB0FC94030B52DED028B0B46F5
:1099B00085B08C68D0E90251D868FFF73DFF08EE0A
:1099C000100A601900EBD0704010FFF7EFFE641B27
:1099D00007EE904AF0EE400AB8EEC88A9FED060AFC
:1099E000F8EEE77A28EE008A27EE800A68EE200A71
:1099F00005B0BDEC028B30BD8262363C82B002B055
:109A0000FFF7D2BFF0B52DED028B0D4689B08C6803
:109A10000646D0E90271E868FFF70EFF08EE100A6B
:109A2000E01900EBD0704010FFF7C0FE73686A6861
:109A30009FED0E1A9B1A07EE903AE41BB8EEE77AF8
:109A4000F0EE400A07EE904A9FED090AB8EEC88A88
:109A5000F8EEE77A28EE008A27EE011A27EE800A50
:109A600068EE200A09B0BDEC028BF0BD0AD7233C9A
:109A70008262363C10B52DED028B84688A680B46F5
:109A8000111B08EE901AC168D868FFF7D5FE224472
:109A900002EBD27208EE100A5010FFF787FEB8EE04
:109AA000C88AF8EEE88A28EE000A20EE000AA8EE3E
:109AB000A80A6EF053FBBDEC028BDFED027A20EEBC
:109AC000270A10BD8262363C094B984206DDC0F180
:109AD000D64000F5930000F5A4407047054B98422E
:109AE000BEBFC0F1144000F5360000F53850704795
:109AF00000E9A43500175BCAF8B52DED028BDFED48
:109B0000148A076820EE280A0646FDEEC07A0D4644
:109B100017EE904A04EBD47007EB6000B0EE608A59
:109B2000FFF744FE28EE288A3819C8EE007AFFF7BE
:109B3000CBFF306017EE900AF7F708FA2B68C018D1
:109B400041EBE371FFF758FEBDEC028B2860F8BDD6
:109B500002AAB34200F10C010830FFF7CDBF0000AC
:109B60000148FFF763BD00BF245A0020012188424D
:109B700038BF08466CF0B0B8FFF7F8BF08B16CF01A
:109B8000AFB87047FFF7FABF00214FF0FF3310B5B1
:109B900000220363044601600171C0F805104172A0
:109BA00080F8251000F13C0300F50B70D9709A6025
:109BB000DA601A615A619A61DA611A625A629A62CB
:109BC000DA631A645A649A64DA641A655A659A65A3
:109BD000DA65DA661A675A677C339842E6D121461D
:109BE00004F5167007F0AAFA044B1A6822B9044962
:109BF0001C6020462CF0E6F9204610BD345A0020A7
:109C00000432090873B5D0F83C32019199420446F8
:109C100013D0D0F84032994218D0D0F844328B4259
:109C200016D102200AE0D4F8343253B3D4F83832D3
:109C30004BB34FF0030002B070BD002094F8223007
:109C40008342F8D8431C84F82230F4E70120F5E77A
:109C5000D0F83062002EE6D194F841233546B600A4
:109C60009AB1A319C3F83012A319019AC3F83C2280
:109C700094F82230AB429CBF6B1C84F822302846FB
:109C8000D9E70126E8E70226E6E704F50C7001A90A
:109C900030442DF033F8E7E738B504460D462CF094
:109CA000A3FF291D201D2CF09FFF05F1080104F1E1
:109CB00008002DF073F805F1140104F114002DF0E3
:109CC0006DF805F1200104F120002DF067F805F191
:109CD0002C0104F12C002CF01BFF05F1300104F1E4
:109CE00030002DF023F805F13C0104F13C002DF08B
:109CF00055F8AB6BA3636B6B636338BD2DE9F04321
:109D0000A1B00023002500F13C0706468DF807505E
:109D100003930493059306930793089309930A9377
:109D20000B9310931193129313931493159316930B
:109D3000179318931C931D931E9300F50F78B94643
:109D400058F8043BF3B1F26E934223D0D6F8E820E2
:109D5000934221D0D6F86421934213D10221EBB271
:109D600099420FD0C1EB411109EB8104214601A8B2
:109D7000FFF792FF39462046FFF78EFF01A93846CC
:109D8000FFF78AFF0135032D07F17C07D8D121B0F9
:109D9000BDE8F0830021E2E70121E0E72DE9F0478B
:109DA00006460F461546804604464FF0000A3946DF
:109DB0003046FFF727FF626FBA425FFA8AF90ED189
:109DC000C3B2022B0BD87C2202FB0A66012086F864
:109DD0003E0086F83F3085F80090BDE8F0870AF134
:109DE000010ABAF1030F04F17C04E0D100243946E2
:109DF0003046FFF707FFD8F86C205FFA84F912B9F4
:109E0000C3B2022B22D90134032C08F17C08EED115
:109E100000244FF07C0906F13E0A39463046FFF730
:109E2000F1FE034609FB04F05FFA84F81AF80020FB
:109E300012B9DBB2022B12D90134032CEDD196F802
:109E40002300042814D919484EF002FA7C2000FBA4
:109E50000464012084F83E0084F83F30BBE70644E8
:109E6000012086F83E0086F83F3085F80080B4E790
:109E700006F54371002251F8043BBB42D4B208D12D
:109E8000A04202D8631C86F8233003342C700020D3
:109E9000A3E73BB9421C06EB800086F82320C0F8FC
:109EA0000C73F2E70132052AE5D1F0E73C300908EE
:109EB000C9B200EB8101D1F83C3253B1026F934239
:109EC0000AD0D0F8EC20934208D0D0F86821934211
:109ED00006D04FF003007047002070470120704704
:109EE0000220704759B190F82030032B07D05A1C3C
:109EF00080F8202000EB83004161012070470020A2
:109F0000704700002DE9F8430F469146044600F5DE
:109F1000BA7894F83E5035B97C344445F9D10025DF
:109F20002846BDE8F88300234A46394601200CF054
:109F3000E3FA00210646E06E0CF0EEFA8642EBD121
:109F4000EEE700002DE9F043DFF87C8085B00446A1
:109F500000F50F7600257C27B14656F80C3CD9F861
:109F600000209342E9B206F1040619D1C3B120469C
:109F7000FFF79EFFC0B207FB004090F83E307BB970
:109F800003A9A9F10C0003932CF0B8FE38F098FD5A
:109F900056F8043C009342462B46012131F0C0FFA5
:109FA0000135032DD8D104F16C0504F5F07429684E
:109FB00021B9AB6813B128462BF0F6FA7C35A542DF
:109FC000F5D105B0BDE8F0835830090838B504462E
:109FD0001546FFF76DFFC0B2022808D87C2303FBAB
:109FE000004029465030BDE838402CF0C7BE38BD8F
:109FF00038B504461546FFF75BFFC0B2022808D803
:10A000007C2303FB004029465C30BDE838402CF03F
:10A01000B5BE38BD37B50D4604468DED010AFFF7D4
:10A0200047FF022D07D8C0B27C2303FB004001A9E3
:10A0300068302CF055FD03B030BD000038B5054642
:10A04000FFF736FFC4B2022C13D8C4EB4414A400AB
:10A050003C3504F10800284400212BF0A5FA04F156
:10A06000340104F1300029442844BDE838402CF084
:10A0700045BE38BD70B505460E461446FFF718FFBD
:10A08000C3B2022B0DD87C2000FB035394E80700D9
:10A09000443383E8070031462846BDE87040FFF7A7
:10A0A000CDBF70BD37B504461546FFF701FFC0B2FE
:10A0B000022809D87C2303FB00400DF10701403042
:10A0C0008DF807502CF090FD03B030BD10B5002185
:10A0D0000446FFF7B3FF20460121FFF7AFFF2046FC
:10A0E0000221BDE81040FFF7A9BF00001FB590F99D
:10A0F0002C30044623B390F921300BB36846FFF7A8
:10A1000099FAFBF719FA6946FAF7F8FFC0B1DDEDE5
:10A11000037A9FED0C0AF8EEE70ADDED027AF8EE1D
:10A12000E77A0123C0EE800A84F83D3387EE800A87
:10A1300007F046FADFED047A20EE270A84ED0A0ADA
:10A1400004B010BD8096184B35FA8E3C024690F94B
:10A15000210058B192F8400340B1114491F92C020A
:10A1600020B192F92400033818BF01207047000085
:10A1700038B590F8223005465BB100242346E1B2A1
:10A180002846FFF7E3FF08B10133DBB20134032CAB
:10A19000F5D1184638BD000090ED0A0A704700005E
:10A1A00038B50C46D1ED066A11460546FFF780FE2C
:10A1B000C3B27C2000FB0353D4ED087AD3ED260A0A
:10A1C00094ED076AD3ED255A93ED245A26EE600AE2
:10A1D00067EEA00AA5EEA70AF0EE607AE5EE867AB1
:10A1E000B7EE007AA6EEE67A67EEE60AB1EE400A2E
:10A1F000E5EE070A6DF068FE9FED071ADFED070A2E
:10A2000040F61C000FF0C2FED5ED0A7ABDE83840DA
:10A2100030EE270A0FF0A6BEDB0F4940DB0F49C026
:10A220002DE9F04190F822308B4204460D4602D2CF
:10A230000020BDE8F081FFF73BFEC0B204F13C0610
:10A24000C0EB401006EB8000083012F0C3FADFEDDF
:10A25000157AB0EEC00AB4EEE70AF1EE10FAE7D4D0
:10A2600029462046FFF724FEC5B27C2000FB0547A7
:10A270003B6F002BDCD0032DDAD000FB05603030C3
:10A28000D7F86C802BF074FFD7E91B32934201D1D1
:10A29000984505D07C2000FB0544C4F86C80C7E7D6
:10A2A0000120C6E7000000342DE9F74F04460E46B2
:10A2B000174600F50F7A4FF0000B5AF8049B5FFA2F
:10A2C0008BF8B9F1000F26D041462046FFF73EFF3C
:10A2D00008B341462046FFF7EBFD7C23C0B203FBE9
:10A2E000004090F83E505DB908F101031B4ADBB213
:10A2F000394630464DF0BAF9284603B0BDE8F08F34
:10A300005AF8102C914506D0154A394630464DF082
:10A31000ADF90025F0E70BF1010BBBF1030FCCD138
:10A320004FF0000894F822305FFA88F18B420DD983
:10A3300020460191FFF774FF054620B90199204698
:10A34000FFF704FF20B908F10108EBE70125D3E787
:10A35000044A394630464DF089F9CDE78030090886
:10A3600095300908BA3009082DE9F0412DED048B2C
:10A3700090F842139FED348ADFED348A9FED349AD2
:10A3800082B00646FFF794FD06F13C07C5B27C207B
:10A3900000FB057554354FF0000896F822205FFA4F
:10A3A00088F39A424ED919463046FFF7CFFE10B9CE
:10A3B00008F10108F1E719463046FFF779FDC4B20C
:10A3C0007C2000FB0474D4ED157AF0EEE77AF4EE0D
:10A3D000C87AF1EE10FA04F154040ED5D4ED017AE6
:10A3E000F0EEE77AF4EEC87AF1EE10FA05D5002027
:10A3F00002B0BDEC048BBDE8F0812946204612F086
:10A4000001FAB4EEE80AF1EE10FAF0DC2946204633
:10A4100011F020FDB4EEC90AF1EE10FAE7DC214696
:10A42000284611F063FC68468DED000ACDED010A67
:10A4300011F0FCFCDFED077AB4EEE70AF1EE10FA5A
:10A44000B6DDD4E70120D3E700000034DB0FC93FBD
:10A45000920A863F00004843022910B5044608D8F6
:10A46000FFF726FD7C23C0B203FB004494F83D00B7
:10A4700010BD0020FCE7000013B590F842130191D5
:10A480000446FFF7E9FF30B10199204602B0BDE86C
:10A490001040FFF75BBE02B010BD0000F7B590F9A9
:10A4A00021500446002D73D090F84053002D6FD0FA
:10A4B00090F84213FFF7D0FF94F83D33064613B9E6
:10A4C0002046FFF713FE002594F82020EBB29A42B5
:10A4D00007D904EB83030135586903689B689847E3
:10A4E000F2E74DF0E7FE0027224604F5BA7140F28C
:10A4F000F315D2F89C30C31AAB428CBF0023012362
:10A5000082F83D307C32914247EA0307F1D194F959
:10A510002430032B07D194F83C33002B3BD0D4F8E4
:10A520003803002849D167B1236B013309D02FF0DC
:10A5300075FD216B2FF03CFD18B12FF06FFD2EF053
:10A54000ADFD94F92C32002B3AD194F92D32CBBBCE
:10A5500094F92E3213B1022384F8423394F8421353
:10A560002046FFF779FF8642054611D02FF056FDB1
:10A570004FF6FF712FF01CFD50B1002D14BF0022CB
:10A58000042201922FF04AFD019A03212FF0A2FC30
:10A59000284603B0F0BD012384F83C330420FFF7C4
:10A5A000E5FA054610B1214606F05EFE94F9243026
:10A5B000C4F83853032BB2D0B5E706F063FEB2E718
:10A5C0000023C9E70123C7E738B590F921300446D5
:10A5D000D3B190F84053BDB1FFF76AFCC0B2022876
:10A5E00012D87C2303FB0044D4ED1A7A9FED087A3D
:10A5F000F4EEC77AF1EE10FA06D4B7EE087AF4EE6C
:10A60000C77AF1EE10FA00DD0025284638BD00BFFC
:10A61000ABAA2A3F70B5D0F8085315F400350446AC
:10A620000E460DD190F840335BB90A78072A07D857
:10A63000012303FA02F290F83F33134380F83F33CB
:10A6400070BD94F82020EBB29A42F9D904EB830351
:10A65000314658690368DB6898470135F1E7000027
:10A6600038B505466C242B591BB1002128192AF056
:10A670009BFF7C34B4F5F07FF5D138BD014B1868F1
:10A68000704700BF345A00202DE9F04FAA4BD3F891
:10A6900000800446D8F8040003688DB09B68984792
:10A6A000002507464FF0010909FA05F33B4240F047
:10A6B00082820135202DF7D1D8F804000368DB68C9
:10A6C0009847002507464FF0010909FA05F33B4278
:10A6D00040F0B3820135202DF7D1D8F8040003688B
:10A6E0009B689847002507464FF0010909FA05F3D2
:10A6F0003B4240F0E1820135202DF7D1D8F804002B
:10A70000DFF840B203689B68984700250490049ADC
:10A710000123AB40134240F00B830135202DF6D1CD
:10A72000D8F80400DFF81CB20368DB6898470025FE
:10A730000490049A0123AB40134240F0C9830135D1
:10A74000202DF6D1D8F804000368DB68984700256F
:10A7500007464FF0010909FA05F33B4240F08384B4
:10A760000135202DF7D1D8F804000368DB6898473D
:10A77000002507464FF0010909FA05F33B4240F076
:10A78000B1840135202DF7D1D8F8040003689B6807
:10A790009847002507464FF0010909FA05F33B42A7
:10A7A00040F0DF840135202DF7D1D8F8040003688C
:10A7B0009B689847002507464FF0010909FA05F301
:10A7C0003B4240F00E850135202DF7D1D8F804002A
:10A7D00003689B689847002507464FF0010909FA6E
:10A7E00005F33B4240F03D850135202DF7D1D8F8E7
:10A7F00004000368DB689847002507464FF001090D
:10A8000009FA05F33B4240F068850135202DF7D168
:10A810004A4B089308AF0425D8F8040003689B68E6
:10A820009847002683460123B34013EA0B0F40F0FC
:10A830008F850136202EF6D1D8F804000368DB6836
:10A840009847002683460123B34013EA0B0F40F0DC
:10A85000C4850136202EF6D1013D15F0FF0507F124
:10A860000107D9D1D8F8040003689B6898474FF0D6
:10A870000109074609FA05F33B4240F0F28501352C
:10A88000202DF7D1D8F804000368DB68984700252D
:10A8900007464FF0010909FA05F33B4240F01D86D7
:10A8A0000135202DF7D1D8F8040003689B6898473C
:10A8B000002507464FF0010909FA05F33B4240F035
:10A8C00048860135202DF7D1D8F804000368DB68ED
:10A8D0009847002507464FF0010909FA05F33B4266
:10A8E00040F073860135202DF7D1154B0793D8F82A
:10A8F000040003689B689847002583460123AB400A
:10A9000013EA0B0F42D000275FFA85F9D4F8083319
:10A9100013F4803A32D107AB4946DB5D04931A4603
:10A920002046FFF7EFFA049B0646002800F08986D0
:10A93000CDE908AA08E000BFCC2500200C0D0E0FC1
:10A9400020212223801A0600099B0B93002201215B
:10A950000BA8CDE9092204F003FE01462046FFF7CB
:10A96000C1FA0BA8FDF7B6F90AA8FDF7B3F909A8D3
:10A97000FDF7BAF916B108A8FDF7B6F994F8233037
:10A98000052B00F048810137042FBFD10135202D60
:10A99000B4D1D8F804000368DB68984700258346E3
:10A9A0000123AB4013EA0B0F38D000275FFA85F97B
:10A9B000D4F8083313F4803A28D107AB4946DB5D5D
:10A9C00004931A462046FFF79DFA049B064600288A
:10A9D00000F04686CDE908AA0022099B0B93114698
:10A9E0000BA8CDE9092204F0BBFD01462046FFF784
:10A9F00079FA0BA8FDF76EF90AA8FDF76BF909A81B
:10AA0000FDF772F916B108A8FDF76EF994F8233036
:10AA1000052B00F000810137042FC9D10135202D0D
:10AA2000BED1D8F8040003689B6898470026824688
:10AA30000123B34013EA0A0F31D010255FFA86F9DB
:10AA4000D4F8083313F0080B20D12A464946204693
:10AA5000FFF758FA0746002800F01186CDE909BB38
:10AA60000A9B002201210BA8CDE90A2301F00AFC70
:10AA700001462046FFF736FA0BA8FDF735F90AA87C
:10AA8000FDF732F917B109A8FDF72EF994F8233034
:10AA9000052B00F0C0800135EDB2142DD0D1013668
:10AAA000202EC5D1D8F8040003689B68984700267B
:10AAB00082460123B34013EA0A0F34D014255FFA0B
:10AAC00086F9D4F8083313F4001B24D12A464946EA
:10AAD0002046FFF717FA0746002800F0E385CDE986
:10AAE00008BB099B0B93002201210BA8CDE9092289
:10AAF00001F0DAFF01462046FFF7F4F90BA8FDF755
:10AB0000E9F80AA8FDF7E6F809A8FDF7EDF817B18E
:10AB100008A8FDF7E9F894F82330052B7BD0013520
:10AB2000EDB2182DCDD10136202EC2D1D8F80400B7
:10AB30000368DB689847002682460123B34013EA86
:10AB40000A0F34D014255FFA86F9D4F8083313F4C9
:10AB5000001B24D12A4649462046FFF7D3F9074671
:10AB6000002800F0AF85CDE908BB0022099B0B93BC
:10AB700011460BA8CDE9092201F096FF01462046B7
:10AB8000FFF7B0F90BA8FDF7A5F80AA8FDF7A2F8A2
:10AB900009A8FDF7A9F817B108A8FDF7A5F894F8DA
:10ABA0002330052B37D00135EDB2182DCDD101362C
:10ABB000202EC2D12FE0D4F8083313F0010A25D19A
:10ABC0005FFA85FB1E2259462046FFF79BF9064691
:10ABD00020B3CDE908AA099A0B920023082201218B
:10ABE0000BA8CDE9093303F089FA01462046FFF7A7
:10ABF00079F90BA8FDF76EF80AA8FDF76BF809A81C
:10AC0000FDF772F816B108A8FDF76EF894F8233036
:10AC1000052B7FF44EAD0DB0BDE8F08FD8F80410D1
:10AC200004220B68CDE90102A84A0092D3F800A0E3
:10AC30005A461E2309A8D047CDE7D4F8083313F0AD
:10AC4000010A24D15FFA85FB1E2259462046FFF7F0
:10AC500059F9064608B3CDE908AA099B0B930622C9
:10AC600000210BA8CDE9091103F048FA014620465E
:10AC7000FFF738F90BA8FDF72DF80AA8FDF72AF819
:10AC800009A8FDF731F816B108A8FDF72DF894F8DA
:10AC90002330052B7FF41EADBDE7D8F80410042245
:10ACA0000B68CDE90102894A0092D3F800A05A4608
:10ACB0001E2309A8D047D0E7D4F8083313F4805AEC
:10ACC00021D15FFA85FB0D2259462046FFF71AF97C
:10ACD0000646F0B1CDE909AA0A9B0022CDE90A2374
:10ACE000012108220BA804F077FA01462046FFF75D
:10ACF000F9F80BA8FCF7F8FF0AA8FCF7F5FF16B166
:10AD000009A8FCF7F1FF94F82330052B7FF4F3AC8E
:10AD100081E7D8F8041004220B68CDE901026B4AE0
:10AD20000092D3F800A05A460D230AA8D047D3E7D3
:10AD3000D4F8083313F480773FD15FFA85F90C22F9
:10AD400049462046FFF7DEF80646002800F08480DA
:10AD5000CDE90677079B0A934FF0000A692249461E
:10AD60002046CDF81CA0FFF7CDF80746002800F0DC
:10AD70008180CDE908AA099B0B9300221A2309922E
:10AD80000BA901220AA801F005F801462046FFF7A9
:10AD9000A9F80BA8FCF7A8FF09A8FCF7A5FF17B1B5
:10ADA00008A8FCF7A1FF0AA8FCF79EFF07A8FCF77C
:10ADB0009BFF16B106A8FCF797FF94F82330052BEC
:10ADC0003FF429AFD4F8083313F480777FF4A5ACAF
:10ADD0005FFA85F90C2249462046FFF793F80646AC
:10ADE000002856D0CDE90677079B0A934FF0000A5A
:10ADF000682249462046CDF81CA0FFF783F8074695
:10AE0000002854D0CDE908AA099B0B9300221A23ED
:10AE100009920BA901220AA800F0BCFF01462046B6
:10AE2000FFF760F80BA8FCF75FFF09A8FCF75CFFD1
:10AE300017B108A8FCF758FF0AA8FCF755FF07A8A8
:10AE4000FCF752FF16B106A8FCF74EFF94F823302A
:10AE5000052B7FF462ACDEE6D8F8041004220B6800
:10AE6000CDF800B0CDE901024A461F6807A80C23BF
:10AE7000B8476FE7D8F8041004220B68CDF800B08B
:10AE8000CDE901024A46D3F800A009A86923D047BA
:10AE900071E7D8F8041004220B68CDF800B0CDE9B2
:10AEA00001024A461F6807A80C23B8479CE7D8F858
:10AEB000041004220B68CDF800B0CDE901024A4627
:10AEC000D3F800A009A86823D0479DE7801A0600A0
:10AED000D4F8083313F480773DD15FFA85F90C225A
:10AEE00049462046FFF70EF80646002800F081800C
:10AEF000CDE90677079B0A934FF0000A692249467D
:10AF00002046CDF81CA0FEF7FDFF074600287ED0A6
:10AF1000CDE908AA099B0B9300221A230BA90AA8C2
:10AF2000099200F037FF01462046FEF7DBFF0BA831
:10AF3000FCF7DAFE09A8FCF7D7FE17B108A8FCF762
:10AF4000D3FE0AA8FCF7D0FE07A8FCF7CDFE16B189
:10AF500006A8FCF7C9FE94F82330052B3FF45BAE3E
:10AF6000D4F8083313F480777FF4E9AB5FFA85F9FE
:10AF70000C2249462046FEF7C5FF0646002855D05C
:10AF8000CDE90677079B0A934FF0000A68224946ED
:10AF90002046CDF81CA0FEF7B5FF0746002853D089
:10AFA000CDE908AA099B0B9300221A230BA90AA832
:10AFB000099200F0EFFE01462046FEF793FF0BA832
:10AFC000FCF792FE09A8FCF78FFE17B108A8FCF762
:10AFD0008BFE0AA8FCF788FE07A8FCF785FE16B1D1
:10AFE00006A8FCF781FE94F82330052B7FF4A7AB6D
:10AFF00011E6D8F8041004220B68CDF800B0CDE9B2
:10B0000001024A461F6807A80C23B84772E7D8F820
:10B01000041004220B68CDF800B0CDE901024A46C5
:10B02000D3F800A009A86923D04773E7D8F8041023
:10B0300004220B68CDF800B0CDE901024A461F6832
:10B0400007A80C23B8479DE7D8F8041004220B6822
:10B05000CDF800B0CDE901024A46D3F800A009A816
:10B060006823D0479EE7D4F8083313F0200A24D190
:10B070005FFA85FB1C2259462046FEF743FF064631
:10B0800008B3CDE908AA0022099B0B9311460BA82F
:10B09000CDE9092203F030FC01462046FEF722FFED
:10B0A0000BA8FCF717FE0AA8FCF714FE09A8FCF78A
:10B0B0001BFE16B108A8FCF717FE94F82330052BE9
:10B0C0007FF44EABA7E5D8F8041004220B68CDE955
:10B0D0000102B84A0092D3F800A05A461C2309A8DE
:10B0E000D047D0E7D4F8083313F0200A24D15FFA10
:10B0F00085FB1E2259462046FEF704FF064608B38C
:10B10000CDE908AA0022099B0B9311460BA8CDE9B3
:10B11000092203F0F1FB01462046FEF7E3FE0BA8EF
:10B12000FCF7D8FD0AA8FCF7D5FD09A8FCF7DCFD63
:10B1300016B108A8FCF7D8FD94F82330052B7FF44E
:10B1400020AB68E5D8F8041004220B68CDE90102B1
:10B15000984A0092D3F800A05A461E2309A8D04767
:10B16000D0E7D4F8083313F0200A25D15FFA85FB25
:10B170001C2259462046FEF7C5FE064610B3CDE90F
:10B1800008AA099A0B920023022201210BA8CDE9FB
:10B19000093303F0B1FB01462046FEF7A3FE0BA8DE
:10B1A000FCF798FD0AA8FCF795FD09A8FCF79CFDA3
:10B1B00016B108A8FCF798FD94F82330052B7FF40E
:10B1C000F1AA28E5D8F8041004220B68CDE90102A1
:10B1D000784A0092D3F800A05A461C2309A8D04709
:10B1E000CFE7D4F8083313F0200A25D15FFA85FBA6
:10B1F0001E2259462046FEF785FE064610B3CDE9CD
:10B2000008AA099A0B920023022201210BA8CDE97A
:10B21000093303F071FB01462046FEF763FE0BA8DD
:10B22000FCF758FD0AA8FCF755FD09A8FCF75CFDE2
:10B2300016B108A8FCF758FD94F82330052B7FF4CD
:10B24000C2AAE8E4D8F8041004220B68CDE9010290
:10B25000584A0092D3F800A05A461E2309A8D047A6
:10B26000CFE7D4F8083313F0400A21D15FFA85FB09
:10B270000C2259462046FEF745FE0646F0B1CDE9C0
:10B2800009AA0A9B0022CDE90A23012106220BA864
:10B2900000F046FD01462046FEF724FE0BA8FCF711
:10B2A00023FD0AA8FCF720FD16B109A8FCF71CFD38
:10B2B00094F82330052B7FF497AAACE4D8F8041057
:10B2C00004220B68CDE901023A4A0092D3F800A0AB
:10B2D0005A460C230AA8D047D3E7D4F8083313F012
:10B2E000400A20D15FFA85FB0C2259462046FEF722
:10B2F00009FE0646E8B1CDE909AA00220A9B1146DB
:10B300000BA8CDE90A2300F00BFD01462046FEF70D
:10B31000E9FD0BA8FCF7E8FC0AA8FCF7E5FC16B170
:10B3200009A8FCF7E1FC94F82330052B7FF46DAA03
:10B3300071E4D8F8041004220B68CDE901021D4A1B
:10B340000092D3F800A05A460C230AA8D047D4E7AD
:10B35000D4F8083313F0800A26D13B78F1B21A46AC
:10B360002046CDE90413FEF7CDFDDDE90413814647
:10B3700010B3CDE909AA0A9B0022CDE90A230121D5
:10B380000C220BA803F086F901462046FEF7AAFD21
:10B390000BA8FCF7A9FC0AA8FCF7A6FCB9F1000F62
:10B3A00002D009A8FCF7A0FC94F82330052B7FF409
:10B3B00040AA30E4801A0600D8F80400B84AD0F851
:10B3C00000E000924FF0040CCDE9019C0A46DEF843
:10B3D00000A001460AA8D047CDE7D4F8083313F0FF
:10B3E000800A26D13B78F1B21A462046CDE90413F3
:10B3F000FEF788FDDDE90413814608B3CDE909AA0B
:10B400000A9B0022CDE90A2300210C220BA803F09D
:10B4100041F901462046FEF765FD0BA8FCF764FCE8
:10B420000AA8FCF761FCB9F1000F02D009A8FCF7EB
:10B430005BFC94F82330052B7FF40BAAFFF7EBBBE2
:10B44000D8F80400964AD0F800E000924FF0040CBF
:10B45000CDE9019C0A46DEF800A001460AA8D047C3
:10B46000CEE7D4F8083313F4004A20D15FFA85FB05
:10B470000C2259462046FEF745FD0646F0B1CDE9BF
:10B4800009AA0A9B002201210BA8CDE90A2302F098
:10B4900077FF01462046FEF725FD0BA8FCF724FCAC
:10B4A0000AA8FCF721FC16B109A8FCF71DFC94F8CA
:10B4B0002330052B7FF4E3A9FFF7ADBBD8F80410C8
:10B4C00004220B68CDE90102754A0092D3F800A06E
:10B4D0005A460C230AA8D047D3E7D4F8083313F40C
:10B4E000004A20D15FFA85FB0C2259462046FEF720
:10B4F00009FD0646F0B1CDE909AA00220A9B1146D2
:10B500000BA8CDE90A2302F03BFF01462046FEF7D7
:10B51000E9FC0BA8FCF7E8FB0AA8FCF7E5FB16B171
:10B5200009A8FCF7E1FB94F82330052B7FF4B8A9B8
:10B53000FFF771BBD8F8041004220B68CDE90102B3
:10B54000574A0092D3F800A05A460C230AA8D047C5
:10B55000D3E7D4F8083313F4007A20D15FFA85FBDF
:10B56000302259462046FEF7CDFC0646F0B1CDE923
:10B5700009AA0A9B002201210BA8CDE90A2303F0A6
:10B5800087FC01462046FEF7ADFC0BA8FCF7ACFBA0
:10B590000AA8FCF7A9FB16B109A8FCF7A5FB94F8CB
:10B5A0002330052B7FF48DA9FFF735BBD8F80410A5
:10B5B00004220B68CDE90102394A0092D3F800A0B9
:10B5C0005A4630230AA8D047D3E7D4F8083313F4F7
:10B5D000007A20D15FFA85FB302259462046FEF7DB
:10B5E00091FC0646F0B1CDE909AA00220A9B11465A
:10B5F0000BA8CDE90A2303F04BFC01462046FEF7D9
:10B6000071FC0BA8FCF770FB0AA8FCF76DFB16B1E8
:10B6100009A8FCF769FB94F82330052B7FF462A995
:10B62000FFF7F9BAD8F8041004220B68CDE901023B
:10B630001B4A0092D3F800A05A4630230AA8D047EC
:10B64000D3E7D8F8041004200A68CDE90160144853
:10B650000090D2F800A009A84A46D047FFF774B975
:10B66000D8F8041004200A68CDE901600C48009065
:10B67000D2F800A009A84A46D047FFF7ADB9D8F8DC
:10B68000041004220B68CDE90102054A0092D3F8A8
:10B6900000B04A462B460AA8D847FFF7E1B900BFD9
:10B6A000801A0600D8F8041004220B68CDE90102C4
:10B6B0000C4A0092D3F800B04A462B4609A8D84756
:10B6C000FFF70FBAD8F8041004220B68CDE9010285
:10B6D000044A0092D3F800B04A462B4609A8D8473E
:10B6E000FFF743BA801A060073B50446FEF7CCFF95
:10B6F00094F82330052B32D0002594F83F33EB40EB
:10B70000DA07E9B216D40135082DF6D194F82330C2
:10B71000052B24D094F8203013B194F82230F3B9DB
:10B72000104B11491B68986903681B6802B0BDE89B
:10B7300070401847D4F808339B030CD42C20019197
:10B74000FEF714FA064610B1019903F019FC3146D0
:10B750002046FEF7C7FB94F82330052BD3D102B067
:10B7600070BD00BFCC250020D43009082DE9F04F72
:10B7700090F9213089B00446002B00F004810123A8
:10B7800000F50C7580F84133024600F50F712B4629
:10B790002E46D06E002859D0002384F8413394F906
:10B7A0004030642B5BD094F9BC30642B00F08D806A
:10B7B00094F93831642B00F08A80D4F830722FBBB2
:10B7C00001A9204629F0D4FE00B30C2305930123E0
:10B7D00006978DF81830714B07936946BDF8043011
:10B7E000049704A8ADF810308DF800702AF092F894
:10B7F0009DF9001051B1022908DC38B1C9B27C238F
:10B8000003FB01416C3128462BF090FA94F841B3C8
:10B81000BBF1000F5DD0E36E6367D4F8E830C4F885
:10B82000F030D4F86431C4F86C3194F8233003F16B
:10B83000C30204EB82020021042B7CD852F8040BD3
:10B840001061013342F8041CDBB2F5E753F8040B36
:10B850000028A1D18B4202F17C029AD19FE70020FF
:10B8600066238DF810307C2303FB004004A9403090
:10B870002BF0A0F904A9204629F07AFE00289CD0DC
:10B8800004238DF818300023CDE9013303933123CD
:10B890000593694604A82AF03DF8059B28B108AA3B
:10B8A00002EB8302009942F8E01C0133332B05932D
:10B8B000EFD94AF025FC9DED031ADDED020A9DED5E
:10B8C000010A66214AF0DAFB77E70120C8E7022087
:10B8D000C6E70127A94655F8043B23B1AB60013701
:10B8E000042FF7D197E7AA46B8465FFA88F3022BF0
:10B8F000F5D8DAF8002055F8043C9A4205D104A99D
:10B900005046CDF810B02BF011FA5AF8043B08F16C
:10B9100001020BB99046E8E704A906EB8800019301
:10B92000CDF810B02BF002FA019BAB6001A948469C
:10B930002BF0FCF9D3E794F8413313B92046FEF716
:10B94000DDF994F822300BB3154B1B68986A036835
:10B9500064215B6898472046FEF7A0FD94F83E30CE
:10B9600003B9E36694F8BA300BB9C4F8E83094F838
:10B9700036310BB9C4F86431F9F7DEFDF9F766FE2C
:10B980000123A4F8403309B0BDE8F08F2046FFF74B
:10B99000ABFE94F82230002BE0D0D5E788C509082B
:10B9A000CC2500207047000001207047012070471F
:10B9B000436898687047000010B5054B0360044663
:10B9C000806A10B103685B689847204610BD00BFCD
:10B9D00098350908406803685B6A184733B46C46B9
:10B9E000406884E80C0003689D6A94E80C00AC464B
:10B9F00002B030BC6047000010B50446FFF7DCFF22
:10BA00002046FEF7BBF8204610BD000040680AF053
:10BA1000A5BC0000406801230AF0A0BC40680AF001
:10BA200079BC000040680A220AF01EBC40680AF097
:10BA300033BC000040680AF0B5BC000090F82E202E
:10BA400022B190F82D10002201F06EB9704700006D
:10BA500073B5044605250026A06A8DF807600368C3
:10BA60000DF10702DB680121984778B19DF8073096
:10BA70000C2B09D0102B05D0092B07D184F83030BE
:10BA800002B070BD1523F9E71423F7E7013DE3D1B8
:10BA90002846F5E710B4806A03681C690822A446AA
:10BAA00001235DF8044B31216047000010B4806A27
:10BAB00003681C690122A44600235DF8044B32216F
:10BAC00060470000F0B50446806A036885B05B6992
:10BAD00098470546002800F08480A06A03685B69E7
:10BAE000984703689B689847A06A03689B699847D2
:10BAF00060B93D4B3D491B68986903681B689847CE
:10BB00002B682846DB689847002667E02046FFF749
:10BB1000CDFF0028F4D02046FFF79AFF0028EFD091
:10BB2000A06A03680121DB6A98472046FFF7B2FF4D
:10BB300030B92D4B2E491B68986903681B68DEE7F6
:10BB4000A06A0368DB69984730B9274B29491B680D
:10BB5000986903681B68D2E7A06A94F8301001273F
:10BB600084F82E7003685B6A9847A06A03689B6A32
:10BB7000984704F12D020146204601F023F90646BC
:10BB80000028BDD0A06A94F82D10036801919B6A2B
:10BB9000984701990246204601F018F994F82C3094
:10BBA0002BB194F82D103A46204601F023F994F871
:10BBB0002F2094F82D10204601F03EF92B682846DE
:10BBC000DB689847A06A029403681D6A0A4B0393D6
:10BBD00004AB13E90C0042F21071A847304605B0DF
:10BBE000F0BD0646FAE700BFCC2500200435090861
:10BBF0002A35090849350908F1BC010870B5002546
:10BC000086B0CDE9005500230446806A8DF80850BF
:10BC100005930393049303686A469E6810210923E1
:10BC2000B047A0B19DF8003013F0010615D194F88B
:10BC300031300133DBB2052B84F8313007D1204697
:10BC4000FFF734FF2046FFF725FF84F83160A06A34
:10BC500003681B6B984706B070BD9DF8083084F8E8
:10BC600031501B07F3D4BDF901309FED1F6A06EE7A
:10BC7000903ABDF9033007EE103ABDF90530F8EE01
:10BC8000E66A07EE903ACDED036AF0EEE66AB8EEAA
:10BC9000C77AF8EEE77AF4EEC66AF1EE10FA8DEDA7
:10BCA000047ACDED057A0DD5B0EEC77AB4EEC67A3A
:10BCB000F1EE10FA06D5F0EEE77AF4EEC67AF1EE80
:10BCC00010FAC4D49FED090A03A810F0D9F9B2EE16
:10BCD000040A03A810F0D4F994F82D200A2303A92C
:10BCE000204601F00FF9B2E7000000349A99193E9E
:10BCF000FFF784BF10B5044B044640F8043BFBF744
:10BD0000F3FF204610BD00BFB035090810B504464A
:10BD1000FFF7F0FF2046FDF731FF204610BD000081
:10BD2000F7B503680F4616461BB90024204603B03A
:10BD3000F0BD0024046008200193FDF717FF0546BD
:10BD400020B1124B0360019B4360019401A8FBF7F3
:10BD5000CBFF002DE9D03420FDF708FF0446002872
:10BD6000E3D000F0E1FE0A4BA562236084F82C705A
:10BD700084F82F602046FFF7A5FE05460028D5D1A0
:10BD8000236820465B6898472C46CFE7B035090802
:10BD9000983509082DE9F74F046806460D46904688
:10BDA0009946002C6CD00B68002B49D023682046A4
:10BDB0005B6A984703689B689847012328680DEBE6
:10BDC000030200210AF0CAFA98B39DF80130EA2B69
:10BDD0002FD1DFF8F0B04FF0060A28680023802248
:10BDE00006210AF097FA20B3DBF80070B86A0368FE
:10BDF0000A215B689847002328681A4606210AF042
:10BE000089FAB0B1B86A03680A215B6898470123D0
:10BE100028680DEB030206210AF0A0FA48B19DF84C
:10BE2000014014F040042FD00AF1FF3A1AF0FF0A43
:10BE3000D3D1306803685B6A98470368DB6898472A
:10BE400000241DE0022223460F2128680AF062FA2E
:10BE5000B86A036801215B689847306803685B6AC9
:10BE600098470368DB689847336834604A46414620
:10BE700001A80193FFF754FF044601A8FBF734FF24
:10BE8000204603B0BDE8F08F224623460F212868E4
:10BE90000AF040FAB86A036801215B6898470223F8
:10BEA000214630680DEB03020AF058FA04460028D8
:10BEB000C8D0B869024903681B689847B9E700BF52
:10BEC00070350908CC25002090F82C10002200F0D5
:10BED0002BBF000070B504468CB00426013E76B23C
:10BEE000731C4AD0A06A15236A465D210AF036FA0F
:10BEF0000028F3D0A06A152306AA5D210AF02EFAC5
:10BF000005460028EAD0152206A968466EF068F9B1
:10BF10000028E3D19DF8003084F82E309DF80730DA
:10BF200084F830309DF8143084F83A309DF813309E
:10BF30009DF8102084F83B309DF80F3043EA02232F
:10BF4000A3879DF8013084F82F309DF8083084F8DD
:10BF50003130039B9DF80C20C3F30F2363869DF8BB
:10BF60000B3043EA0223A386049BC3F30F23E3862B
:10BF7000019BC3F30F23238707E0054B05491B688B
:10BF8000986903681B689847002528460CB070BD67
:10BF9000CC250020E43509082DE9FF4104460023A3
:10BFA000806A8DF807300368DFF868815B6A98471C
:10BFB00003689B689847A06A03680A219B6C9847AE
:10BFC000A06A0A2204210AF04FF90425013D6DB24E
:10BFD0006B1C32D000234B21A06A82220AF09AF90E
:10BFE000D8F800600746B06A036802215B6898478A
:10BFF000002FEBD001231A464B21A06A0AF08AF9E0
:10C000000746B06A036802215B689847002FDDD0BD
:10C01000A06A01230DF1070240210AF09FF90028D0
:10C02000D4D09DF80720322A10D0002DCED1B0698F
:10C03000364903681D683223A847A06A03685B6A13
:10C0400098470368DB68984700255BE02046FFF7C8
:10C0500041FF0028F1D0A06A0123172251210AF0E4
:10C0600059F90028E9D05222A06A012311460AF0AA
:10C0700051F90028E1D0A06A012338224C210AF0AE
:10C0800049F90028D9D0A06A03685B6A9847036819
:10C09000DB689847A06A05210AF0FEF8A36A04F15C
:10C0A0002C029968204600F08DFE054650B3A36A25
:10C0B00094F82C109A68204600F088FE94F84420EA
:10C0C00094F82C10204600F0B7FE94F845302BB1C0
:10C0D00094F82C100122204600F08CFEA06A036820
:10C0E00002219B6C9847A06A029403689E6A084BE1
:10C0F000039304AB13E90C0044F21B11B0474CF05E
:10C10000D9F82064284604B0BDE8F0810C3609084F
:10C1100081C20108CC25002070B5858F90F93B6065
:10C12000AD03B5FBF2F2A2F5804404FB04F2D51195
:10C1300090F83A200498D201624306FB052252127D
:10C14000A03002F58012424312134A43DB0003EB96
:10C15000623000B270BD000010B5448E53005C43E5
:10C16000B0F93830C91A838FD31AB0F93620B0F934
:10C170003400534304F500449B10C3EBC13300EB80
:10C180002440044993FBF0F04FF400420DF02CFFE3
:10C1900000B210BD0080FFFF10B52DED028B8AB0FC
:10C1A00004460823806A05AA42210AF0D7F818B18C
:10C1B000BDF81A20D30719D4A06A0AF0F3F84CF09E
:10C1C00079F8236CC31AFA2B0CD92064002382223D
:10C1D0004B21A06A0AF09EF80123A06A1A464B215F
:10C1E0000AF098F80AB0BDEC028B10BDBDF914102E
:10C1F00094F930300093920894F92E300392C910CC
:10C200002046FFF789FFBDF9161094F93130039AE3
:10C21000009308EE900A94F92F30C9102046FFF7DA
:10C220007BFFBDF91810039A491008EE100A20464A
:10C23000FFF792FF07EE900AF8EEE88AF8EEE77A49
:10C24000B8EEC88AB3EE000A07A8CDED097ACDEDA5
:10C25000078A8DED088A0FF027FFB2EE040A07A8BF
:10C260000FF00EFF4CF026F894F82C2020640A23DF
:10C27000204607A900F046FEA06A0AF093F8B1E74D
:10C28000FFF78ABFF7B503680D4616461BB90024B1
:10C29000204603B0F0BD002707604820CDE90073B9
:10C2A000FDF764FC044650B100F03EFC0E4B2360E9
:10C2B000019BA362019784F8446084F8455001A86B
:10C2C000FBF708FD6846FBF705FD002CDFD0204694
:10C2D000FFF762FE05460028DAD1236820465B6836
:10C2E00098472C46D4E700BF4436090810B5044BE4
:10C2F000044640F8283BFBF7EDFC204610BD00BF8C
:10C300004436090810B50446FFF7F0FF2046FDF754
:10C3100035FC204610BD000090F82C10002200F0E3
:10C3200003BD0000F8B504460D4617461E4600F052
:10C33000FBFB094B23602B68A362002200232A60C9
:10C3400084F82D7084F82E6023656365A365E3652A
:10C35000236663662046F8BD5C360908F8B51C46BE
:10C3600009331646DB086A46A2EBC30300AF9D46BD
:10C37000806AA31C6A4609F0F1FF054628B12246EF
:10C380000DF1020130466DF03BFF2846BD46F8BD79
:10C390002DE9F34106460F4614464BF08BFF114B37
:10C3A000D3F800800546D8F82800036801215B68AF
:10C3B000984701230DF1070207213046FFF7CEFF12
:10C3C00060B19DF80730DA0702D4B7EB531F05D0F0
:10C3D0004BF070FF431BA342E5D3002002B0BDE841
:10C3E000F08100BFCC2500202DE9F041DFF860820C
:10C3F00092B0044602AF002646F02002A06A002355
:10C40000D2B2502109F086FF002800F00C810325EC
:10C41000013D6DB26A1C00F00681D8F80030986AC0
:10C4200003684FF496719B68984701230DF106024B
:10C4300055212046FFF792FF002800F0F4809DF878
:10C44000063013F0E00F40F0EE80DB07E0D502236A
:10C450000DF1060252212046FFF780FF002800F070
:10C46000E280BDF8063001365BBA202E27F8023B89
:10C47000C2D1BDF824309DF826109FED6D7ADFED16
:10C480006D6A9FED6D6A43F30B0207EE902A1B095C
:10C4900003F47063BDF82620F8EEE77A0B4343F30C
:10C4A0000B03C4ED0C7A07EE903A02F470639DF82A
:10C4B0002820F8EEE77A134343F30B03C4ED0D7A1B
:10C4C00007EE903A9DF92230F8EEE77AC4ED0E7A45
:10C4D00007EE903A9DF92930F8EEE77A67EE877A11
:10C4E00007EE103AB8EEC77A9DF92A30C4ED0F7AFC
:10C4F00027EE267ADFED517A84ED107A07EE103AB6
:10C50000B8EEC77A9DF92B30E7EE267AC4ED117AA2
:10C5100007EE903AF8EEE77A9DF9233067EEA67AB7
:10C52000DFED476AC4ED127A07EE903A9DF92C30A0
:10C5300007EE103AB8EEC77A9DF92E3027EE267A2C
:10C54000F8EEE77A84ED147A67EE867A07EE103A11
:10C550009DF93030C4ED137A07EE903AF8EEE77AA1
:10C560009DF92D3067EEA67AB8EEC77AC4ED167A3B
:10C5700027EE267A07EE903A84ED157AF8EEE77A00
:10C580009FED307A9DF92F3067EE877AC4ED177AE8
:10C5900007EE903A9DF93130F8EEE77A06EE903AE0
:10C5A00067EE877AF8EEE66AC4ED187ADFED267A50
:10C5B000BDF93830E6EE877A07EE103A9DF9323051
:10C5C000C4ED197AB8EEC77AF3EE077AE7EE067A89
:10C5D00007EE103ADFED1D6AC4ED1A7AB8EEC77A9D
:10C5E00027EE267A84ED1B7A9DF9333007EE103A58
:10C5F000B8EEC77A9DF9343027EE267A84ED1C7A9E
:10C6000007EE103A9DF9353007EE903AB8EEC77A4A
:10C61000F8EEE77A27EE267A67EEA67A84ED1D7AA1
:10C62000C4ED1E7A00E0002012B0BDE8F08100BF2A
:10C63000CDCC4C3E0000803B0000003B0AD7233CA1
:10C640000000003D0000803817B7D1B80AD7A33AE0
:10C65000CC25002073B501230E460DF107020621FB
:10C660000446FFF77BFE18B90025284602B070BDCE
:10C670009DF80730013B012B0CD80023A06A1A4615
:10C68000062109F047FE0028EED0062200212046B0
:10C69000FFF77EFEA06A00233246062109F03AFE2B
:10C6A00005460028E0D0262231462046FFF770FEDE
:10C6B000DBE7000013B501230DF107020721044653
:10C6C000FFF74CFE10B9002002B010BD9DF80730F6
:10C6D0001B070CD50023A06A1A46062109F01AFE92
:10C6E0000028F0D0062200212046FFF751FEA06A64
:10C6F00000230722062109F00DFE0028E3D01322B3
:10C7000007212046FFF744FE0028DCD0A06A002362
:10C710000522062109F0FEFD0028D4D017220521AC
:10C720002046FFF735FE0028CDD001212046FFF737
:10C7300091FFC9E7F7B50446806A5B4F03685B6AFF
:10C74000984703689B689847A06A03680A219B6C16
:10C750009847A06A0A22042109F086FD0525013DBB
:10C760006DB26B1C00F09680A06A0023B6227E2179
:10C7700009F0D0FD0028F2D03B68986A03681821C0
:10C780005B686E4698470123324600212046FFF73A
:10C79000E5FD0028E3D09DF80030332BDFD12046A3
:10C7A000FFF722FE002875D0A06A002380225021C6
:10C7B00009F0B0FD00286DD02046FFF77BFF002870
:10C7C00068D0A06A002386222E2109F0A3FD00284C
:10C7D00060D0A06A00232422042109F09BFD0028D8
:10C7E00058D0A06A00230222062109F093FD0028F8
:10C7F00050D0142202212046FFF7CAFDA06A002370
:10C800000722052109F086FD002843D0012120469A
:10C81000FFF720FF00283DD0A06A036803219B6C2E
:10C820009847A06A03685B6A98470368DB68984783
:10C83000A06A172109F030FDA36A04F12C0299685F
:10C84000204600F0BFFA054608B3A36A94F82C10FE
:10C850009A68204600F0BAFA94F82E2094F82C102A
:10C86000204600F0E9FA94F82D302BB194F82C1002
:10C870000122204600F0BEFAA06A03689F6A0B4BB3
:10C880000094019396E80C0042F21071B8472846D4
:10C8900003B0F0BDA06A03685B6A98470368DB6871
:10C8A00098470025F3E700BFCC250020A5CA010862
:10C8B00010B586B00C236A4631210446FFF74EFDC1
:10C8C000002800F0DF809DF801309DF80020DFEDAA
:10C8D000717ADFED715A1B0403EB02239DF80220ED
:10C8E00003EB02631B1206EE903A9DF804309DF8AC
:10C8F00003201B0403EB02239DF8052003EB0263D6
:10C900001B1207EE103A9DF807309DF806201B0415
:10C9100003EB02239DF8082003EB02631B1206EED3
:10C92000103A9DF80A309DF809201B0403EB0223FE
:10C93000F8EEE66AB8EEC77A9DF80B2066EEA76AB5
:10C9400027EE277AB8EEC66ADFED547A03EB02636E
:10C950001B1226EE276A07EE903AF8EEE77A67EEAA
:10C96000A57AF5EEC07AF1EE10FA40F38D80DFED96
:10C970004C5A77EEE57AD4ED134A94ED0F5A94EDC4
:10C980001C4AD4ED1D3A94F82C20F7EE005A74EEB0
:10C99000A54AF0EE632AA4EEA75A0A2303A9D4ED10
:10C9A000107AD4ED0C4A77EEA57A2046E7EEA64A37
:10C9B000D4ED1A7A75EE677A94ED145AF0EE646A43
:10C9C000D4ED174AE5EE276AB0EE655AA7EEA45AF1
:10C9D000C6EE854A94ED115AD4ED0D6A35EE255A0E
:10C9E000E5EE076A94ED157AE7EE876A94ED187A1A
:10C9F000B0EE655AA7EE875A86EE857A94ED125A04
:10CA0000D4ED0E6A35EE255AE5EE066A94ED166A07
:10CA100094ED195AE7EE866AB0EE656AA7EE856A6C
:10CA2000F0EE657A86EE863A94ED1B6AF0EE646A63
:10CA3000E6EE447AE6EE476A86EEA75AF0EE476ADB
:10CA4000E4EE646AC6EEA75AD4ED1E6AD4EE262A36
:10CA5000E6EE636AB2EE046A27EE667A65EE066A6F
:10CA6000A2EEA47ACDED036A65EE866ACDED046A86
:10CA7000C7EE276A76EE837A67EE867ACDED057A81
:10CA800000F040FA06B010BD44BFDFED055A77EE66
:10CA9000A57A70E747ABE73B5B9E803AF61BEB3B22
:10CAA00085EBCB41FFF704BF30B51346026885B074
:10CAB0000D461AB90024204605B030BD00210160A2
:10CAC0007C2001930392FDF751F8044620B1019BAD
:10CAD0002A4603A9FFF726FC03A8FBF7FBF8002C66
:10CAE000E8D02046FFF726FE05460028E3D123685C
:10CAF00020465B6898472C46DDE7000010B5044BE4
:10CB0000044640F8283BFBF7E5F8204610BD00BF7F
:10CB10005C36090810B50446FFF7F0FF2046FDF724
:10CB20002DF8204610BD0000064B10B503600446EA
:10CB3000FDF7A4FD606004F108004AF071FD204695
:10CB400010BD00BF7436090873B5064614467568F3
:10CB50007C2303FB0253C4EB441405EB8404084616
:10CB600093F8A41001900FF021FB94F93C30019848
:10CB70003BB9736893F8251002B0BDE870400FF020
:10CB800015BB94F84010F7E737B5446801917C2550
:10CB900005FB024595F83F3004EB8304D4F84C3292
:10CBA0005BB14BF087FBC5F89C000199D4F84C02AF
:10CBB00003B0BDE8304003F079BE03B030BD0000E3
:10CBC0002DE9F04FC2EB421447684FEA84088146D2
:10CBD0000E4607F13C0B08F108018BB0154659448D
:10CBE00030460FF019FAD9F8040029460BEB8404FB
:10CBF000FDF7EAFC38B17C2303FB057393ED1A0AB9
:10CC000030460FF03DFA7C2303FB057393ED146A65
:10CC1000DFED3A7AD3ED156AB0EEC67AB4EEE77A74
:10CC2000F1EE10FA0FD5B0EEE67AB4EEE77AF1EE57
:10CC300010FA08D594ED077AB0EEC77AB4EEE77A29
:10CC4000F1EE10FA1BD47C2303FB0573D86D196E2B
:10CC50005A6E9B6D029003910490079101A8314692
:10CC60008DED016ACDED056A0692089209930DF0EB
:10CC700085FB86ED000AC6ED010A86ED021A7C23CB
:10CC800003FB05770023C7F88C30C7F88830C7F856
:10CC90008430D9F8040090F95C3208F13C0A08F1BC
:10CCA0004808DA44D84463B15DB9414600F51670CE
:10CCB00004F0B4FA414630460BB0BDE8F04F0FF037
:10CCC000ABB990F93430012B0BD190ED0E0A5046E0
:10CCD0000FF082F984ED120AC4ED130A84ED141AE0
:10CCE000E8E7022BE6D1FBF75DFD002201A9FBF787
:10CCF00059FA0028DED09DED010AE8E70000003473
:10CD000010B543687C2404FB023407C904F1900386
:10CD100083E807004BF0CEFAC4F89C004BF0BEFA53
:10CD2000C4F8A00010BD0000F0B5074685B00D4660
:10CD3000164600F10801A92203A809F069FD7C68E4
:10CD40007C2303FB0543D3F8B42022B903A809F0E0
:10CD500081FD05B0F0BDBEB196ED007AD3ED2A7A23
:10CD600067EE877AC3ED2A7A96ED017AD3ED2B7AB6
:10CD700067EE877AC3ED2B7A96ED027AD3ED2C7AA3
:10CD800067EE877AC3ED2C7A7C2607EE902A06FBA5
:10CD90000541A831B8EE670A084601910FF084F901
:10CDA00001992A463846FFF7ABFF06FB05410023F1
:10CDB000C1F8B030C1F8AC30C1F8A8300023C1F8D8
:10CDC000B430C3E74068FCF7E9BF0000F7B506469A
:10CDD000406801927C2707FB01000D466C3001A9D9
:10CDE000144629F083FF716807FB05152C6703B013
:10CDF000F0BD000007B540687C2303FB010393F9F5
:10CE00003C30022B0BD000F13C03C1EB411003EB93
:10CE100080000DF107018DF8072029F0C1FE03B055
:10CE20005DF804FB43687C2202FB013191F93C0070
:10CE3000003818BF0120704743687C2000FB013197
:10CE400081F8A42070470000F8B5054608460F4653
:10CE50000FF088F910B100242046F8BD38460FF0D5
:10CE600067F904460028F6D16B6893F934637EB104
:10CE700038460FF0AFFC95ED087ADFED1F7AF0EE43
:10CE8000C76AF4EEE76AF1EE10FA03D585ED080AF9
:10CE90000124E1E777EE407A30EE076AF0EEE77AB8
:10CEA000C7EE866AF6B207EE906A9FED146AF8EE56
:10CEB000677A26EE866AF4EEC67AF1EE10FA48BF7B
:10CEC000B2EE046ADFED0E7A45BF6B6A66EE866AE3
:10CED000B0EE676A87EEA66A46BF01336B62012433
:10CEE000F7EE007A77EEC67A20EE060AA7EE270A5A
:10CEF00085ED080AB0E700BF000000340000484399
:10CF0000CDCCCC3D2DE9F74304460E4615461F46D1
:10CF1000FFF71AFE2A4631462046FFF735FE314616
:10CF200020462A46FFF74CFE31462046FFF78CFF8D
:10CF300028B39B2204F1080101A809F069FC646888
:10CF40004FF07C0909FB054808F1A8083146404626
:10CF50000FF062F809FB0542D2F8B4100131C2F8B3
:10CF6000B4104FB1B94207D34908C2F8B410B0EEBB
:10CF7000000A40460FF098F801A809F06BFC03B0D6
:10CF8000BDE8F08310B50446FCF792FFC0B23C3414
:10CF9000C0EB401004EB800010BD0000F8B50A4E55
:10CFA000044600F5167704F5137555F8040B08B11F
:10CFB00003F0B0FFBD42F8D13368986A03680121DD
:10CFC0005B689847EFE700BFCC25002008B5FFF766
:10CFD000E5FF0000F0B5144E00EB810773780446BE
:10CFE000D7F84C026FF3410387B00D467370C8B198
:10CFF00002F07EFB68B1737843F0100373702C4429
:10D000000023A372D7F84C0207B0BDE8F04002F04D
:10D01000F3BAD7F84C12684602F09AFB009B012B3A
:10D02000EDD1E8E707B0F0BD945A002070B5064690
:10D030000D46002445FA04F3DB07E1B202D5304681
:10D04000FFF7C8FF0134032CF4D170BDFF21FFF7B7
:10D05000EDBF000030B500F5137587B000F516740C
:10D0600055F8041B21B9A542FAD1002007B030BD04
:10D07000684602F06DFB009B013B022BF3D80120B8
:10D08000F4E700002DE9F0472DED028B88B004464F
:10D090000D469046B0EE408AFDF7DEF930B9002625
:10D0A000304608B0BDEC028BBDE8F087294620462B
:10D0B000FDF74CF806460028F1D004EB8507D7F8B9
:10D0C0003C22D7F830329A4206D035F0F9FC5C4A5F
:10D0D00003212EF025FFE2E7D7F84C3283B94FF455
:10D0E0009870FCF743FD814608B103F017F8C7F8C4
:10D0F0004C92B9F1000F03D135F0E2FC514AE7E759
:10D10000B4F84A32D90711D505F078FE90F8082313
:10D1100090F8C43232B9B02202FB030090F8A1307B
:10D12000012B03D835F0CCFC474AD1E72046FFF766
:10D1300091FF20B9454A537843F00203537094F9A4
:10D14000353053B329462046FFF71CFF90F90030D5
:10D15000002B53D029462046FFF714FF90F8049087
:10D16000B9F12B0F19D829462046D7F84CA2FFF762
:10D1700009FF94F9353090F90020022BD4BF00212B
:10D180000121012BD4BF00230123003A009118BFD5
:10D1900001224946504602F043FA631900229A726E
:10D1A00075B3D4EDC10AB4F84822D7F84C0270EE3A
:10D1B000A00A2B46B0EE480A414602F051FA94F814
:10D1C0003E33002B31D1224A069412680127E773BF
:10D1D000906A0268156D1F4A0792029309224FF464
:10D1E0000063CDE9003208AA12E906001A4BA847ED
:10D1F000C8B935F065FC194A02216AE79946B2E7D9
:10D2000029462046FFF7BEFE90F90030002BC8D01B
:10D21000D4EDC10AB4F84822D4F84C022B46B0EE43
:10D22000480A4146C9E784F83E7300230DF117010F
:10D2300004F124008DF8173029F0BCFC30E700BF62
:10D2400084360908B6360908D9360908945A0020E8
:10D25000CC250020CDCF0108F73609080237090890
:10D260002DE9F0412DED028B002443739DF8203011
:10D27000837305460F469046B0EE408A264647FA2D
:10D2800004F3DB07E1B210D5B0EE480A4246284667
:10D29000FFF7F8FE064640B939462846FFF7C6FEB6
:10D2A000BDEC028B3046BDE8F0810134032CE6D1A1
:10D2B000F6E70000F8B500242DED028B05460F4679
:10D2C000B0EE408A427383732646E1B2B0EE480A5C
:10D2D0003A462846FFF7D6FE0134002818BF064616
:10D2E000032CF2D1BDEC028B3046F8BDF0B500EB5B
:10D2F00081030D46D3F84C129BB0044611B90020AF
:10D300001BB0F0BD0BA802F007FA6319987A002849
:10D31000F6D10B9A002A48D0042AF0D101229A7241
:10D320000DAA07CA02AB83E8070010AA07CA05AF17
:10D3300087E8070013AA07CA9DED180A08AE86E819
:10D3400007001A46294620468DED010AFCF792FE99
:10D350003A4629462046FCF739FE32462946204601
:10D36000FCF746FE9DED010A29462046FCF752FED9
:10D370009DF8643083B129462046FFF703FE90F9FB
:10D3800000304BB194F93530012B05DD9DF85D205F
:10D3900029462046FCF786FE2046FFF75BFE20B9B3
:10D3A000034A537843F0040353700120A8E700BFF9
:10D3B000945A00202DE9F0410546884600F5137780
:10D3C0000024012657F8043BE1B26BB148FA04F39C
:10D3D000DB0709D52846FFF789FF002857F8040C1A
:10D3E00008BF002602F008F90134032CEAD13046C8
:10D3F000BDE8F0812E4B2DE9F04F1F68FB6A93F8D2
:10D400009C8087B00446B8F1000F38D1DFF8A8A09F
:10D4100000F5137600F1030B054656F8040BA5EB57
:10D4200004095FFA89F9E8B102F04EF928B19AF8D7
:10D43000013043F008038AF8013056F8040C02F07A
:10D4400057F9F8B9637B6BB1AB7A5BB956F8041C3A
:10D45000684602F07DF9009B042B03D14946204623
:10D46000FFF744FF01355D45D7D1124B204683F8C5
:10D470001280FFF7EFFD054630B10123237407B09A
:10D48000BDE8F08F8046EDE7237C002BF7D0A37B2F
:10D49000002BF4D0B86A03684FF47A715B68984740
:10D4A000B86A03689B6B294607B0BDE8F04F184780
:10D4B000CC250020755A0020945A0020F0B5002594
:10D4C00087B000F513762C46012756F8041B41B1AE
:10D4D000684602F03DF9009B1BB107FA05F31C43B7
:10D4E000E4B20135032DF0D1204607B0F0BD0000B5
:10D4F0002DE9F04F2DED028B03270E7C9FED348A32
:10D5000091B005468846B946AC5D0134E4B2B4FB3F
:10D51000F9F303EB4303E41AE4B205EB8403D3F815
:10D520004C1209B9AC554CE003A802F011F9DDF832
:10D530000CB00BF1FF33022BF4D830462FF07EFCF9
:10D540008246304630F07EFB00F11B039A4508D23C
:10D5500030462EF0EFFE002011B0BDEC028BBDE88E
:10D56000F08FAC55284698F810A0FFF7A7FFDDED27
:10D57000057A8DF83100FCEEE77A9DF810208DF8E1
:10D58000332017EE903A8DF8343006AB03CB1B886E
:10D59000ADF83D305C221B23CDE90032CDF83500DB
:10D5A000CDF8391009AABF2150468DED098A8DEDBD
:10D5B0000A8A8DED0B8A8DF830408DF832B02FF04D
:10D5C000A7FC013F17F0FF079ED10120C4E700BF71
:10D5D000000000002DE9F04F0F7CA1B00646884600
:10D5E000032500EB070999F805400134E4B2032351
:10D5F000B4FBF3F303EB4303E41AE4B206EB840356
:10D60000D3F84C1211B989F805400AE011A802F0CC
:10D6100083F8DDF844A0BAF1030F08DCBAF1000F7B
:10D62000F1DA013D15F0FF05DDD1012012E0AAF18C
:10D630000402032AF5D838462FF000FC834638460A
:10D6400030F000FB00F13602934506D238462EF04A
:10D6500071FE002021B0BDE8F08F89F8054030460A
:10D6600098F810B0FFF72AFFDDF848E0CDF80CE09D
:10D67000DDF84CE0CDF810E0DDF850E0CDF814E036
:10D68000DDF854E0CDF818E0DDF858E0CDF81CE006
:10D69000DDF85CE0CDF820E0DDF860E0CDF824E0D6
:10D6A0003219DDF864E01C9BCDF828E0DDF868E075
:10D6B00092F80AC09DF874109DF87520CDF82CE002
:10D6C0000E93DDF86CE01E9B8DF835008DF83C1054
:10D6D0008DF83D20CDF830E08DF834408DF836A03F
:10D6E0008DF837C02422CDF83E303623CDE9003204
:10D6F000C0212C2303AA58462FF00AFC91E7000012
:10D700007FB58A8B0B464AF2B9518A4205465FD0F3
:10D710004AF2BA518A4274D04AF2B8518A420BD1C5
:10D72000474A1268D26A92F89C203AB135F0C8F99B
:10D73000444A05212EF0F4FB042479E0D3ED007A6D
:10D74000F5EEC07AF1EE10FAF6D49FED3F7AF4EEE2
:10D75000C77AF1EE10FAEFDC93ED017ADFED3B6A68
:10D760001C6993ED030AB0EEC77AB4EEE67A93ED46
:10D77000027AFCEEE77AB0EEC77AF1EE10FAB4EE78
:10D78000E67A17EE903A54BF01260026F1EE10FA21
:10D7900054BF01220022003C18BF012413F0FF01F6
:10D7A00010D18DED030A0292FCF7CCFB9DED030A2C
:10D7B000029A234631462846FFF77CFD0028BBD05D
:10D7C000002435E0134600943246FFF749FDF5E7A3
:10D7D000D3ED007AF5EEC07AF1EE10FAACD49FEDFD
:10D7E0001A7AF4EEC77AF1EE10FAA5DCFCEEE77ACD
:10D7F00017EE903A13F0FF0108BFFF21FFF7DAFDA3
:10D80000DCE7D3ED007AF5EEC07AF1EE10FA93D4AE
:10D810009FED0D7AF4EEC77AF1EE10FA8CDCFCEE97
:10D82000E77A17EE904A14F0FF0404D1FFF70EFCDC
:10D83000204604B070BD2146FFF7F8FBC0E700BFEB
:10D84000CC2500203437090800007F430000003455
:10D85000F0B58BB00E4614460746FFF793FB5430E5
:10D8600007C884E8070031463846FFF78BFB90ED88
:10D87000057ADFED267AB0EEC77AB4EEE77AF1EEFC
:10D8800010FA054611D590ED067AB0EEC77AB4EEDF
:10D89000E77AF1EE10FA08D590ED077AB0EEC77A84
:10D8A000B4EEE77AF1EE10FA24D431463846FFF7A9
:10D8B00069FB016A426A836AE869D5F814E0D5F821
:10D8C00018C0099001A8CDF804E0029103920491D8
:10D8D000CDF814C00693079208930CF0FBFE98B1A4
:10D8E000214601A80CF04AFD84ED000AC4ED010AAE
:10D8F00084ED021A31463846FFF744FB00F1080177
:10D9000020460EF0A3FB01200BB0F0BD0000003458
:10D910002DE9F0472DED048BACB0B0EE608A0546E2
:10D92000B0EE409A0F46F0EE418A9046FCF70AFBB3
:10D93000DFED8B7AB0EEC87AB4EEE77AF1EE10FA4A
:10D940004BD5B0EEE87AB4EEE77AF1EE10FA44D5B2
:10D9500023AC2046FBF76EFEF7F7EEFD2146F7F706
:10D96000CDFB064658BB05F049FA90F8083390F80D
:10D97000C42233B1B02303FB020393F8A130012B7F
:10D9800007D84FF0B00909FB020090F8A130022B34
:10D990000BD835F095F8734A03212EF0C1FA3046C2
:10D9A0002CB0BDEC048BBDE8F08705F027FA90F8A9
:10D9B000C43209FB0300AC300FC884E80F00DDED72
:10D9C000257A9FED691AB8EEE78ADDED267AF8EE42
:10D9D000E78A28EE018A68EE818A04AA03A902A8D0
:10D9E000F0EE680AB0EE480A03F0D4FC064618B917
:10D9F00035F066F85D4ACFE79FED5D7ADDED027A9E
:10DA00009FED5C8ADFED5C8A8DED068A67EE877A92
:10DA10002422002111A8CDED057A8DED078A6CF046
:10DA200039FC9DED031ADDED040ADFF858A121EE63
:10DA3000281A68EEE00AB0EE480A11A80CF06AFE57
:10DA400005A911A80CF09AFC242200211AA8CDEDFA
:10DA5000060A8DED071A8DED050A6CF01BFCF7F731
:10DA60006BFD90ED810A8DED010AF7F765FD29EE5A
:10DA7000281AD0ED820A9DED010A1AA80CF04AFE80
:10DA80001AA923A80CF068FD05A923A80CF076FCC0
:10DA90004FF000098DED050ACDED060A8DED071A50
:10DAA00095F822305FFA89F4A3427FF678AF1FB170
:10DAB00027FA04F3DB071AD52B1993F92C32B3B1EB
:10DAC000B8F1000F0DD021462846FCF7C5FC88B9F7
:10DAD00034F0F6FF294A234603212EF021FA0026CE
:10DAE0005DE721462846FCF731FB0028EBD109F120
:10DAF0000109D5E708AA214628468DED088A8DED53
:10DB0000098A8DED0A8AFFF7A3FE20B934F0D8FF09
:10DB10001B4A2346E0E708A905A80EF047FA0BAA1E
:10DB2000214628468DED0B0ACDED0C0A8DED0D1A20
:10DB3000FCF7A0FA9AE807000EAB83E807001A4644
:10DB400021462846FCF742FA23AA214628468DEDB5
:10DB5000238A8DED248A8DED258AFCF749FAC6E7E4
:10DB6000000000345837090895BFD63373370908C9
:10DB700000007A440000000035FA8E3C883709081E
:10DB80009C370908E4E3080801207047012070472A
:10DB90004368986870470000406803689B6C1847AA
:10DBA00010B5054B03600446806A10B103685B68DA
:10DBB0009847204610BD00BF8438090840680368B4
:10DBC0005B6A184733B46C46406884E80C0003680D
:10DBD0009D6A94E80C00AC4602B030BC604700007F
:10DBE00010B50446FFF7DCFF2046FBF7C7FF2046D1
:10DBF00010BD0000406808F04FBB0000406808F00E
:10DC0000ADBB00004068012308F0A8BB40680023BA
:10DC100008F080BB90F84420D20705D590F8421058
:10DC200000F12C02FFF780B870470000F8B50446F9
:10DC30001E460F461546FEF777FF084B236000236C
:10DC4000E3622363636394F84430A76265F341039E
:10DC500084F8436084F844302046F8BD84380908CD
:10DC600010B50D4B83630446806A036898221B69D4
:10DC70000021984770B1A06A036820221B69012126
:10DC8000984738B1A06A0368BDE810401B690122BB
:10DC900002211847002010BDC5DC6A3F37B5044695
:10DCA000806A03686A469D6803210623A847D0B1AD
:10DCB000BDF80020BDF8041052BA95B249BAB5F5C6
:10DCC000704F0BB211D013F5805F0ED0BDF802304B
:10DCD0005BBA9DB2B5F5704F07D052425B42A28746
:10DCE000E187A4F8403003B030BD0020FBE700001E
:10DCF000806A036801221B690221184730B585B08C
:10DD00000446FFF7CBFF05462046FFF7F1FF6DB352
:10DD1000B4F93C3094ED0E0A06EE903AB4F93E3078
:10DD200007EE103AB4F9403007EE903AF8EEE66AA2
:10DD3000B8EEC77AF8EEE77A01A8CDED016A8DED6D
:10DD4000027ACDED037A0EF09BF994F8421020464A
:10DD5000FFF768F818B1022101A80EF027FA94F82D
:10DD600042200E2301A92046FFF7CCF805B030BDB4
:10DD7000FFF7C4BF13B5806A036801AA9C680A2133
:10DD80000323A04738B10549032201A86CF028FA03
:10DD9000B0FA80F0400902B010BD00BFBC370908DE
:10DDA0002DE9F84300252DED028BDFF888819FEDEA
:10DDB0005D8A04462E462F46A06A036811221B691D
:10DDC00000210137984700287BD0D8F80090D9F877
:10DDD0002800036832215B689847A06A03686022C4
:10DDE0001B690121984700286BD0A06A03680122B3
:10DDF0001B6902219847002863D0D9F828000368DE
:10DE000032215B6898472046FFF748FF002858D02A
:10DE10000135022FEDB256DDB4F93C309FED425A88
:10DE20009FED426A07EE903AF8EEE77AC5EE276A70
:10DE3000F0EEE66AF4EEC66AF1EE10FA41DDF4EEB9
:10DE4000C86AF1EE10FA3CD5B4F93E30DFED385A2D
:10DE500007EE903AF8EEE77A85EEA77AB0EEC77A49
:10DE6000B4EEC67AF1EE10FA2BDDB4EEC87AF1EE1C
:10DE700010FA26D5B4F9403005EE903AF8EEE55A9E
:10DE8000C5EE257AF0EEE77AF4EEC67AF1EE10FAF6
:10DE900017DDF4EEC87AF1EE10FA12D594ED0B6AA4
:10DEA00076EE266A0136C4ED0B6AD4ED0C6A36EEC6
:10DEB000877A84ED0C7A94ED0D7A77EE277AC4EDAB
:10DEC0000D7A192F02D0052E7FF476AFA06A036871
:10DED00010221B6900219847052E18D1D4ED0B6A3A
:10DEE000F1EE047A86EEA77A0120D4ED0C6A84ED77
:10DEF0000B7A86EEA77AD4ED0D6A84ED0C7A86EE65
:10DF0000A77A84ED0D7ABDEC028BBDE8F8834FF063
:10DF10007E53052DE3622363636394BF00200120D9
:10DF2000F1E700BFCDCCAC3F00002E443333333F8C
:10DF300000002244CC250020F0B50446806A036826
:10DF400085B05B699847054648B9504B50491B68F6
:10DF5000986903681B689847284605B0F0BD0368B8
:10DF60009B689847A06A03680A21DB6A9847A06A01
:10DF700003689B69984760B9444B46491B68986998
:10DF800003681B6898472B682846DB68984700257C
:10DF9000E2E72046FFF7EEFE0028F4D02046FFF728
:10DFA000FFFE30B9394B3C491B68986903681B6810
:10DFB000E8E72046FFF754FE0028E4D0A06A036893
:10DFC000DB69984730B9314B34491B68986903685D
:10DFD0001B68D7E794F84430A06A43F0010384F843
:10DFE000443003680321DB6A98472B682846DB68C6
:10DFF0009847236820469B689847A06A03680721D2
:10E000005B6A9847A06A03689B6A984704F14202DA
:10E0100001462046FEF7D6FE054600289CD0A06AA1
:10E0200094F84210036801919B6A9847019902464F
:10E030002046FEF7CBFE94F8432094F84210204689
:10E04000FEF7FAFE94F844309B0705D594F8421089
:10E0500001222046FEF7CEFEA06A029403681E6AE3
:10E060000F4B039304AB13E90C0043F21541B04787
:10E07000064BA06A1B689E6933681F6803689B6A29
:10E080009847084902463046B84765E7CC25002046
:10E09000C0370908E63709080C380908313809087B
:10E0A00071DD01085F38090810B5084B03600446AC
:10E0B0000023086860600B60037A03F00703022BFB
:10E0C00002D1C02108F016FA204610BD9C3809087C
:10E0D00010B5044B044640F8043BF9F7FBFD20461D
:10E0E00010BD00BF9C38090810B50446FFF7F0FFCB
:10E0F0002046FBF743FD204610BD0000F7B503683E
:10E100000E4617461BB90024204603B0F0BD00227E
:10E11000026008200193FBF729FD054610B101A913
:10E12000FFF7C2FF01A8F9F7D5FD002DEBD048207D
:10E13000FBF71CFD04460028E5D029463B46324645
:10E14000FFF774FD2046FFF7F7FE05460028DBD1F8
:10E15000236820465B6898472C46D5E790F82D1039
:10E160000022FEF7E1BD0000F0B50446806A0368B6
:10E1700089B05B6A984703689B689847A06A036800
:10E180000A219B6C9847A06A01230DF11702002118
:10E1900008F0E4F8002838D09DF81730082B34D167
:10E1A0004E4F052500230122A06A322108F0B2F863
:10E1B0003B689B6A1A68526840B90A211846904722
:10E1C000013D15F0FF05EDD145481CE0184614212E
:10E1D000904706AEFF238DF81830A06A012332461F
:10E1E000322108F0BBF80028EAD09DF8183013F06F
:10E1F0000103E5D1A06A03930822322108F08AF8CE
:10E20000039B58B9374849F099FAA06A03685B6ADA
:10E2100098470368DB68984700255CE0A06A039391
:10E220001A46342108F076F80028EBD0039BA06A48
:10E230002422412108F06EF80028E3D0039BA06A55
:10E240000822312108F066F80028DBD0A06A0368B4
:10E2500003219B6C9847A06A03685B6A9847036830
:10E26000DB689847A06A102108F016F8A36A04F149
:10E270002D0299682046FEF7A5FD054658B3A36A0E
:10E2800094F82D109A682046FEF7A0FDA36A164860
:10E290001A7A597A00919B681449D20849F04EFACB
:10E2A00094F82C2094F82D102046FEF7C5FD94F824
:10E2B0002E302BB194F82D1001222046FEF79AFD46
:10E2C000A06A03689F6A0A4B0694079396E80C00BD
:10E2D00042F21071B847284609B0F0BDCC250020A5
:10E2E0002C390908CC38090803390908FB38090812
:10E2F0007DE3010810B586B004460123806A0DF164
:10E300000302102108F02AF898B39DF80330DB07C8
:10E310002FD5A06A062301AA112108F01FF840B3E7
:10E32000BDF904309FED146A94F82D2006EE903A62
:10E33000BDF9063007EE103ABDF808305B421BB25B
:10E3400007EE903AF8EEE66AB8EEC77AF8EEE77AAA
:10E3500066EE866A27EE067A67EE867A0A2303A9B6
:10E360002046CDED036A8DED047ACDED057AFEF7FA
:10E37000C9FD06B010BD00BF85EBC13FFFF7BABFB6
:10E38000F7B503680D4616461BB90024204603B0B6
:10E39000F0BD002707603020CDE90073FBF7E6FBF6
:10E3A000044650B1FEF7C0FB0E4B2360019BA362F5
:10E3B000019784F82C6084F82E5001A8F9F78AFCA4
:10E3C0006846F9F787FC002CDFD02046FFF7CCFE2B
:10E3D00005460028DAD1236820465B6898472C461A
:10E3E000D4E700BF5839090810B5044B044640F87B
:10E3F000283BF9F76FFC204610BD00BF58390908CB
:10E4000010B50446FFF7F0FF2046FBF7B7FB2046A8
:10E4100010BD000090F831100022FEF785BC00000E
:10E4200010B5002304460122806A0A2107F072FF1A
:10E4300010B9012384F8323010BD0000F0B5044655
:10E44000806A036889B05B6A984703689B6898474D
:10E45000A06A03680A219B6C9847012200230B21C4
:10E46000A06A07F057FF514B1F68B86A03680A217A
:10E470005B689847A06A01230DF11702002107F09D
:10E480006DFF002835D09DF81730102B31D10525B0
:10E49000002301220B21A06A07F03CFFBB6A1A6827
